:020000040000FA
:1000000000040020E508000079050000C508000094
:10001000830500008D05000097050000000000002A
:1000200000000000000000000000000009090000BE
:10003000A105000000000000AB050000B5050000B0
:10004000BF050000C9050000D3050000DD05000064
:10005000E7050000F1050000FB05000005060000B3
:100060000F06000019060000230600002D06000000
:1000700037060000410600004B0600005506000050
:100080005F06000069060000730600007D060000A0
:1000900087060000910600009B060000A5060000F0
:1000A000AF060000B9060000C3060000CD06000040
:1000B000D7060000E1060000EB060000F506000090
:1000C000FF06000009070000130700001D070000DD
:1000D00027070000310700003B070000450700002C
:1000E0004F07000059070000630700006D0700007C
:1000F00077070000810700008B07000095070000CC
:100100009F0700001FB500F003F88DE80F001FBD2A
:1001100000F0DEBB1FB56FF00100009040100390AF
:10012000029001904FF010208069000B420900F00E
:100130001F045DF822300120A04083434DF8223097
:10014000684600F044F91FBDF0B54FF6FF734FF459
:10015000B4751A466E1E11E0A94201D3344600E080
:100160000C46091B30F8027B641E3B441A44F9D14B
:100170009CB204EB134394B204EB12420029EBD17E
:1001800098B200EB134002EB124140EA0140F0BD8F
:10019000DD4992B00446D1E90001CDE91001FF220A
:1001A0004021684600F03AFB94E80F008DE80F000C
:1001B000684610A902E004C841F8042D8842FAD12B
:1001C00010216846FFF7C0FF1090AA208DF8440068
:1001D000FFF7A0FF00F0F2F84FF01024A069102202
:1001E0006946803000F001F9A069082210A900F0EA
:1001F000FCF800F0D7F84FF080510A6949690068AF
:100200004A43824201D8102070470020704710B541
:10021000D0E900214FF0805002EB8103026944696C
:100220006243934209D84FF01022536903EB8103D4
:100230000169406941438B4201D9092010BD5069D1
:10024000401C01D0002010BD0F2010BD70B501680A
:100250000446AE4D4FF01020062951D2DFE801F0E0
:10026000320318283B1DD4E90265646829463046EC
:1002700000F0CDF82A462146304600F0B6F8AA0034
:100280002146304600F09EFA002800D0032070BDC1
:1002900000F050FB4FF4805007E0201DFFF7ABFF4C
:1002A0000028F4D100F046FB60682860002070BD93
:1002B000241D94E80700920000F084FA0028F6D08C
:1002C0000E2070BD8069401C12D0201DFFF79FFFDB
:1002D0000028F6D109E08069401C09D0201DFFF7F5
:1002E0008AFF0028EDD1606820B12046FFF750FF5B
:1002F000042070BDFFF70EFF00F060F800F052F828
:10030000072070BD10B50C46182802D001200860E7
:1003100010BD2068FFF79AFF206010BD4FF0102439
:10032000A069401C05D0A569A66980353079AA2846
:1003300008D06069401C2DD060690068401C29D03D
:1003400060692CE010212846FFF7FEFE31688142EB
:100350001CD1A16901F18002C03105E030B108CAA9
:1003600051F8040D984201D1012000E000208A429A
:10037000F4D158B1286810B1042803D0FEE728460C
:1003800000F057F861496868086008E000F016F866
:1003900000F008F84FF480500168491C01D000F0CB
:1003A000A3FAFEE7BFF34F8F59480168594A01F499
:1003B000E06111430160BFF34F8FFEE74FF0102063
:1003C0008169491C02D0806900F0ADB87047524A7B
:1003D00001681160121D416811604F4A8168103236
:1003E0001160111DC068086070472DE9F041174683
:1003F0000D460646002406E03046296800F0A6F8BF
:10040000641C2D1D361DBC42F6D3BDE8F08170B5CD
:100410000C4605464FF4806608E0284600F083F855
:10042000B44205D3A4F5806405F58055002CF4D1C1
:1004300070BD4168044609B1012500E000254FF078
:1004400010267069A268920000F0BCF9C8B120467D
:1004500000F01AF89DB17669A56864684FF4002031
:1004600084420AD2854208D229463046FFF7CFFFA0
:100470002A4621463046FFF7B8FFFFF79FFFFFF7F8
:1004800091FFFFF747FEF8E72DE9FF414FF01024F9
:10049000616980680D0B01EB800000F6FF70010BB5
:1004A00000200090019002900246039068460123CC
:1004B0000BE0560902F01F0C50F8267003FA0CFCF2
:1004C00047EA0C0740F82670521CAA42F1D30AE012
:1004D0004A0901F01F0650F8225003FA06F6354388
:1004E00040F82250491C8029F2D3A169090B4A091E
:1004F00001F01F0150F822408B409C4340F82240FD
:10050000FFF765FFBDE8FF815809000000000020EB
:100510000CED00E00400FA050006004014480168F4
:100520000029FCD07047134A0221116010490B6862
:10053000002BFCD00F4B1B1D186008680028FCD056
:100540000020106008680028FCD07047094B10B5E7
:1005500001221A60064A1468002CFCD00160106861
:100560000028FCD00020186010680028FCD010BDC6
:1005700000E4014004E5014008208F49096809585A
:10058000084710208C4909680958084714208A49EF
:100590000968095808471820874909680958084711
:1005A0003020854909680958084738208249096878
:1005B000095808473C2080490968095808474020E5
:1005C0007D4909680958084744207B49096809584A
:1005D0000847482078490968095808474C20764957
:1005E000096809580847502073490968095808479D
:1005F0005420714909680958084758206E4909680C
:10060000095808475C206C49096809580847602068
:100610006949096809580847642067490968095801
:100620000847682064490968095808476C206249EE
:1006300009680958084770205F4909680958084740
:1006400074205D4909680958084778205A490968A3
:10065000095808477C2058490968095808478020EC
:1006600055490968095808478420534909680958B9
:100670000847882050490968095808478C204E4986
:1006800009680958084790204B49096809580847E4
:10069000942049490968095808479820464909683B
:1006A000095808479C204449096809580847A02070
:1006B0004149096809580847A4203F490968095871
:1006C0000847A8203C49096809580847AC203A491E
:1006D000096809580847B020374909680958084788
:1006E000B4203549096809580847B82032490968D3
:1006F00009580847BC203049096809580847C020F4
:100700002D49096809580847C4202B490968095828
:100710000847C8202849096809580847CC202649B5
:10072000096809580847D02023490968095808472B
:10073000D4202149096809580847D8201E4909686A
:1007400009580847DC201C49096809580847E02077
:100750001949096809580847E420174909680958E0
:100760000847E8201449096809580847EC2012494D
:10077000096809580847F0200F49096809580847CF
:10078000F4200D49096809580847F8200A49096802
:1007900009580847FC2008490968095808475FF4C8
:1007A0008070054909680958084700000348044952
:1007B000024A034B70470000000000206809000057
:1007C0006809000040EA010310B59B070FD1042A15
:1007D0000DD310C808C9121F9C42F8D020BA19BA0C
:1007E000884201D9012010BD4FF0FF3010BD1AB171
:1007F000D30703D0521C07E0002010BD10F8013BC6
:1008000011F8014B1B1B07D110F8013B11F8014BEC
:100810001B1B01D1921EF1D1184610BD02F0FF033F
:1008200043EA032242EA024200F005B870477047EB
:1008300070474FF000020429C0F0128010F0030C42
:1008400000F01B80CCF1040CBCF1020F18BF00F8C3
:10085000012BA8BF20F8022BA1EB0C0100F00DB872
:100860005FEAC17C24BF00F8012B00F8012B48BFD0
:1008700000F8012B70474FF0000200B51346944674
:100880009646203922BFA0E80C50A0E80C50B1F1E8
:100890002001BFF4F7AF090728BFA0E80C5048BFFC
:1008A0000CC05DF804EB890028BF40F8042B08BF9A
:1008B000704748BF20F8022B11F0804F18BF00F896
:1008C000012B7047014B1B68DB68184700000020B4
:1008D00009480A497047FFF7FBFFFFF713FC00BD0B
:1008E00020BFFDE7064B1847064A1060016881F3F8
:1008F0000888406800470000680900006809000097
:100900001D030000000000201EF0040F0CBFEFF3D9
:100910000881EFF30981886902380078182803D12B
:1009200000E00000074A1047074A12682C3212689C
:100930001047000000B5054B1B68054A9B589847B7
:1009400000BD000005030000000000205409000065
:1009500004000000001000000000000000FFFFFF86
:040960000090D00330
:10100000E8110020ADE00100452F00001BE00100C9
:10101000452F0000452F0000452F00000000000074
:1010200000000000000000000000000005E10100D9
:10103000452F000000000000452F0000452F000054
:101040006DE1010073E10100452F0000452F000014
:10105000452F0000452F0000452F0000452F0000C0
:1010600079E10100452F0000452F00007FE10100DC
:10107000452F000085E101008BE1010091E10100B5
:10108000452F0000452F0000452F0000452F000090
:10109000452F0000452F0000452F0000452F000080
:1010A000452F000097E10100452F0000452F00006B
:1010B000452F0000452F0000452F0000452F000060
:1010C0009DE10100452F0000452F0000452F000045
:1010D000452F0000452F0000452F0000452F000040
:1010E000452F0000452F0000452F0000452F000030
:1010F000452F0000452F0000452F0000452F000020
:10110000452F0000452F000000F002F81CF0BBFF47
:101110000AA090E8000C82448344AAF10107DA4552
:1011200001D11CF0B0FFAFF2090EBAE80F0013F0C6
:10113000010F18BFFB1A43F0010318473CD601000A
:101140005CD601000A4410F8014B14F00F0508BFEB
:1011500010F8015B240908BF10F8014B6D1E05D083
:1011600010F8013B6D1E01F8013BF9D1641E03D05C
:10117000641E01F8015BFBD19142E4D3704700008B
:101180000023002400250026103A28BF78C1FBD890
:10119000520728BF30C148BF0B6070471FB500F031
:1011A0003DF88DE80F001FBD1EF0040F0CBFEFF3DC
:1011B0000880EFF30980014A104700009F2E0000CD
:1011C0008269034981614FF00100104470470000BB
:1011D000D511000001B41EB400B511F009F901B435
:1011E0000198864601BC01B01EBD0000F0B4404627
:1011F000494652465B460FB402A0013001B506488D
:10120000004700BF01BC86460FBC80468946924617
:101210009B46F0BC70470000091100001CF030BF75
:1012200070B51A4C054608202070A01C00F05FF82D
:101230005920A08029462046BDE8704008F010B82B
:1012400008F019B870B50C461149097829B1A0F118
:101250006001512908D3012013E0602804D06928D7
:1012600002D043F201000CE020CC0A4E94E80E00BC
:1012700006EB8000A0F58050241FD0F8806E284631
:10128000B047206070BD01207047000008000020BA
:101290001C000020E8E1010010B5044600210120F7
:1012A00000F03BF800210B2000F037F80421192052
:1012B00000F033F804210D2000F02FF804210E2057
:1012C00000F02BF804210F2000F027F80421C84378
:1012D00000F023F80721162000F01FF80721152041
:1012E00000F01BF82046FFF79BFF002010BD98215F
:1012F00001807047FFF7A4BF10487047104A10B52F
:1013000014680F4B0F4A08331A60FFF79BFF0C4815
:10131000001D046010BD704770474907090E002882
:1013200006DA00F00F0000F1E02080F8141D70478D
:1013300000F1E02080F800147047000003F900423B
:101340001005024001000001FE48002101604160DB
:10135000018170472DE9F743044692B091464068F9
:1013600011F0FAFA40B1606811F0FFFA20B9607824
:1013700000F00300022801D0012000E00020F14E1F
:101380004D463072484611F0A3FA18B1102015B03E
:10139000BDE8F0832946012001F02FFF0028F6D197
:1013A00001258DF842504FF4C050ADF840000022A6
:1013B00010A9284606F0F9FB0028E8D18DF8425024
:1013C0004FF428504FF00008ADF8400047461C216C
:1013D0006846CDF81C801CF0F8FD9DF81C0008AA9A
:1013E00020F00F00401C20F0F00010308DF81C00A1
:1013F00020788DF81D0061789DF81E0061F3420091
:1014000040F001008DF81E009DF800000AA940F090
:1014100002008DF800002089ADF83000ADF8327080
:10142000608907AFADF834000B97606810AC0E9080
:101430000A94684606F0ACF90028A8D1BDF820004F
:1014400030808DF8425042F60120ADF840009DF802
:101450001E0008AA20F00600801C20F001008DF874
:101460001E000220ADF83000ADF8340013A80E9035
:101470000AA9684606F08CF9002888D1BDF820003A
:101480007080311D484600F033F9002887D18DF86F
:10149000425042F6A620ADF840001C216846CDF827
:1014A0001C801CF092FD9DF81C00ADF8345020F01B
:1014B0000F00401C20F0F00010308DF81C009DF84B
:1014C0001D0008AA20F0FF008DF81D009DF81E00E9
:1014D0000AA920F0060040F00100801C8DF81E00D3
:1014E0009DF800008DF8445040F002008DF8000097
:1014F000CDE90A4711A80E90ADF83050684606F0C5
:1015000047F9002899D1BDF82000F08000203EE77F
:101510003EB504460820ADF80000204611F0D8F989
:1015200008B110203EBD2146012001F066FE0028D2
:10153000F8D12088ADF804006088ADF80600A088D6
:10154000ADF80800E088ADF80A007E4801AB6A46B5
:101550008088002106F026FDBDF800100829E1D0A2
:1015600003203EBD1FB50446002002900820ADF8C0
:101570000800CDF80CD0204611F0AAF910B11020C7
:1015800004B010BD6F4802AA81884FF6FF7006F0C4
:10159000A5FF0028F4D1BDF80810082901D00320C8
:1015A000EEE7BDF800102180BDF802106180BDF8A3
:1015B0000410A180BDF80610E180E1E701B582B01A
:1015C0000220ADF800005F4802AB6A464088002167
:1015D00006F0E8FCBDF80010022900D003200EBD83
:1015E0001CB5002100910221ADF80010019011F00E
:1015F00095F908B110201CBD52486A4641884FF643
:10160000FF7006F06BFFBDF800100229F3D0032035
:101610001CBDFEB54B4C06461546207A0F46C0074A
:1016200005D0084611F054F918B11020FEBD0F2066
:10163000FEBDF82D01D90C20FEBD304611F048F951
:1016400018BB208801A905F0A8FD0028F4D1307846
:101650008DF80500208801A906F082FC0028EBD156
:1016600000909DF800009DF8051040F002008DF8F4
:101670000000090703D040F008008DF80000208822
:10168000694606F00AFC0028D6D1ADF8085020883B
:101690003B4602AA002106F085FCBDF80810A942CD
:1016A000CAD00320FEBD7CB5054600200090019005
:1016B0000888ADF800000C462846019511F04CF959
:1016C00018B9204611F02AF908B110207CBD15B1D7
:1016D000BDF8000050B11B486A4601884FF6FF7004
:1016E00006F0FCFEBDF8001021807CBD0C207CBD06
:1016F00030B593B0044600200D460090142101A897
:101700001CF063FC1C2108A81CF05FFC9DF8000085
:10171000CDF808D020F00F00401C20F0F000103071
:101720008DF800009DF8010020F0FF008DF8010009
:101730009DF8200040F002008DF8200001208DF877
:10174000460001E0C601002042F60420ADF8440046
:1017500011A801902088ADF83C006088ADF83E00EB
:10176000A088ADF84000E088ADF842009DF8020086
:1017700006AA20F00600801C20F001008DF802006F
:101780000820ADF80C00ADF810000FA8059001A9D5
:1017900008A805F0FDFF002803D1BDF81800288037
:1017A000002013B030BD0000F0B5007B059F1E4641
:1017B00014460D46012800D0FFDF0C2030803A206F
:1017C0003880002C08D0287A052806D0287B0128EC
:1017D00000D0FFDF17206081F0BDA889FBE72DE96D
:1017E000F04786B0144691F80C900E9A0D46B9F168
:1017F000010F0BD01021007B2E8A8846052807D0C8
:10180000062833D0FFDF06B0BDE8F0870221F2E7FB
:10181000E8890C2100EB400001EB400018803320E8
:101820001080002CEFD0E889608100271AE0009634
:10183000688808F1020301AA696900F0B2FF06EBAB
:101840000800801C07EB470186B204EB4102BDF89B
:10185000040090810DF1060140460E320FF0E4F9CC
:101860007F1CBFB26089B842E1D8CCE73420108039
:10187000E889B9F1010F11D0122148430E301880C8
:10188000002CC0D0E88960814846B9F1010F00D032
:101890000220207300270DF1040A1FE00621ECE767
:1018A0000096688808F1020301AA696900F079FFCF
:1018B00006EB0800801C86B2B9F1010F12D007EBCD
:1018C000C70004EB4000BDF80410C18110220AF1EA
:1018D000020110301CF0E0FA7F1CBFB26089B842F0
:1018E000DED890E707EB470104EB4102BDF80400A6
:1018F000D0810AF10201404610320FF095F9EBE772
:101900002DE9F0470E4688B090F80CC096F80C8090
:10191000378AF5890C20109902F10C044FF0000A67
:10192000BCF1030F08D0BCF1040F3ED0BCF1070F8F
:101930007DD0FFDF08B067E705EB850C00EB4C00BE
:10194000188031200880002AF4D0A8F1060000F0A9
:10195000FF09558125E0182101A81CF036FB0097EE
:101960007088434601AA716900F01BFFBDF80400AE
:101970002080BDF80600E080BDF808002081A21C90
:101980000DF10A0148460FF04FF9B9F1000F00D0F0
:1019900018B184F804A0A4F802A007EB080087B2ED
:1019A0000A346D1EADB2D6D2C4E705EB850C00EB50
:1019B0004C00188032200880002ABBD0A8F1050016
:1019C00000F0FF09558137E000977088434601AA6F
:1019D000716900F0E6FE9DF80600BDF80410E18094
:1019E0002179420860F3000162F34101820862F349
:1019F0008201C20862F3C301020962F304114209C1
:101A000062F34511820962F386112171C009607188
:101A1000BDF80700208122460DF1090148460FF06C
:101A200003F918B184F802A0A4F800A000E007E0D0
:101A300007EB080087B20A346D1EADB2C4D279E755
:101A4000A8F1020084B205FB08F000F10E0CA3F827
:101A500000C035230B80002AA6D0558194810097C1
:101A600083B270880E32716900F09BFE62E72DE947
:101A7000F84F1E460A9D0C4681462AB1607A00F551
:101A80008070D080E089108199F80C000C274FF00D
:101A900000084FF00E0A0D2873D2DFE800F09E0711
:101AA0000E1C28303846556A737373002146484629
:101AB0000095FFF779FEBDE8F88F207B9146082856
:101AC00002D0032800D0FFDF378030200AE000BFBB
:101AD000A9F80A80EFE7207B9146042800D0FFDFB9
:101AE000378031202880B9F1000FF1D1E3E7207B66
:101AF0009146042800D0FFDF37803220F2E7207BB8
:101B00009146022800D0FFDF37803320EAE7207BB0
:101B10001746022800D0FFDF3420A6F800A0288056
:101B2000002FC8D0A7F80A80C5E7207B17460428F5
:101B300000D0FFDF3520A6F800A02880002FBAD003
:101B40004046A7F80A8012E0207B1746052802D0FD
:101B5000062800D0FFDF1020308036202880002F9C
:101B6000A9D0E0897881A7F80E80B9F80E00B88175
:101B7000A1E7207B9146072800D0FFDF3780372080
:101B8000B0E72AE04FF0120018804FF0380017003D
:101B9000288090D0E0897881A7F80E80A7F810807F
:101BA00099F80C000A2805D00B2809D00C280DD074
:101BB000FFDF80E7207B0C2800D0FFDF01200AE058
:101BC000207B0D2800D0FFDF042004E0207B0E28BE
:101BD00000D0FFDF052038736DE7FFDF6BE770B5DE
:101BE0000C46054601F07CFA20B10078222804D288
:101BF000082070BD43F2020070BD052128460DF09B
:101C0000A3FB206008B1002070BD032070BD38B573
:101C10000546DDE905011446049A72B10B460090B1
:101C20000422214628460AF02DFE032C06D1214627
:101C30002846BDE838400AF0F5BF198038BD2DE9C7
:101C4000FF4F85B0002003900898904689461230D7
:101C500008F0BFFA401D20F00306089828B908A92B
:101C60000598FFF7BCFF002861D1B9F1000F06D03D
:101C70000898017B00295FD10525046829E098F8C0
:101C80000000092803D00F2820D0FFDF54E0089A75
:101C900003255168527B48887243824246D901F13C
:101CA000040B098897B20C181FFA86FABC4200D3BD
:101CB000E41B5044B84200D9FFDF04EB0A00B842ED
:101CC00000D9FFDF5C440020208002E0089C04254E
:101CD00008340CB1208810B1032D27D02CE00898CF
:101CE0000121123008F0ADFAADF81000024603AB46
:101CF000294605980AF0B7FC070001D1A01C039003
:101D000008983A461230C8F804000598A8F802006E
:101D100004A94046039B08F0A1FAC0B1072814D2D9
:101D2000DFE800F0080A1313110C0E00132009B0AD
:101D3000BDE8F08F0020FAE71120F8E70820F6E769
:101D400043F20300F3E70720F1E70320EFE7BDF8D4
:101D5000100003990097CDE9011023462A460899FF
:101D60000598FFF754FFC7B9032D16D10898B7B2ED
:101D70004568407B704384B2298868880E18A64263
:101D800000D3361B3844A04200D9FFDFF019A0422F
:101D900000D9FFDF688838446880B9F1000FC9D0E6
:101DA000089981F80C90C5E72DE9FF4791461A88FC
:101DB0001C468A4680460AB303AB49460AF053FCE8
:101DC00005001BD04046A61C27880DF0DAFB3246E2
:101DD000072629463B4600960DF060F820880399B7
:101DE0000095CDE9011023464A4651464046FFF78B
:101DF0000EFF00202080012004B005E50020FBE755
:101E000010B586B01C46AAB104238DF800301388A3
:101E1000ADF808305288ADF80A208A788DF80E2087
:101E20000988ADF80C1000236A462146FFF707FF2A
:101E300006B010BD1020FBE770B50D4605210DF072
:101E400083FA040000D1FFDF294604F11200BDE847
:101E5000704008F0DFB92DE9F8430D4680460026B2
:101E600007F0B1FA0446287812287BD2DFE800F0A8
:101E70007A54543C355632321332323209323232CD
:101E800032322879001FC0B2022801D0102810D1A8
:101E900014BBFFDF35E004B9FFDF052140460DF03C
:101EA00053FA007B032806D004280BD0072828D03B
:101EB000FFDF072657E02879801FC0B2022820D014
:101EC00050B1F6E72879401FC0B2022819D0102877
:101ED00017D0EEE704B9FFDF13E004B9FFDF28797C
:101EE00001280ED1172139E0052140460DF02CFACA
:101EF000070000D1FFDF07F11201404608F061F949
:101F00002CB12A462146404600F05BFC2BE0132111
:101F1000404602F04DFC26E0FFDF24E004B9FFDF7D
:101F2000052140460DF010FA060000D1FFDF69469A
:101F300006F1120008F04FF9060000D0FFDFA98873
:101F4000172901D2172200E00A46BDF8000082429C
:101F500002D9014602E005E01729C3D3404600F04C
:101F600046FCCEE7FFDF3046BDE8F883401D20F099
:101F70000300021D01FB0020704708B1FE4A1060FB
:101F80000CF08ABB2DE9F0470E4615462421304659
:101F90001CF01BF805B9FFDFA87870732888DFF8FC
:101FA000D8A3401D20F0030195F802900C46DAF802
:101FB00000000CF088FB070000D1FFDF4FF00008A5
:101FC0003760A7F8008004FB09F4211DDAF800004F
:101FD0000CF079FB040000D1FFDF7460C4F80080CE
:101FE000298806F11200BDE8F04708F0DCB82DE9B9
:101FF000F047804601F112000D46814608F0E9F8ED
:10200000401DDD4E20F003046F7B224629683068B6
:102010000CF082FB7C43221D696830680CF07CFB6D
:1020200005200DF03BF9044605200DF03FF9201A7C
:10203000012802D130680CF037FB49464046BDE824
:10204000F04708F0C5B870B5054605210DF07CF9DC
:10205000040000D1FFDF04F112012846BDE8704002
:1020600008F0AFB82DE9F04F91B04FF0000BADF88C
:1020700034B0ADF804B047880C46054692460521B9
:1020800038460DF061F9060000D1FFDF24B1A780CA
:10209000A4F806B0A4F808B0297809220B20B2EB06
:1020A000111F297A7DD104F110023827C91E4FF083
:1020B0000C094FF0010803920F2973D2DFE801F0F9
:1020C000F4F3F28108D48A8FA13DDDF5F0B8B800B1
:1020D000307B022800D0FFDFA88909EBC001ADF8F2
:1020E00004103021ADF83410002C25D06081B5F8F3
:1020F0000E9000271DE004EBC708317C88F80E1015
:10210000F189A8F80C10CDF800906888042304AA7F
:10211000296900F046FBBDF81010A8F8101009F16D
:102120000400BDF812107F1C1FFA80F9A8F81210E5
:10213000BFB26089B842DED80CE1307B022800D003
:10214000FFDFE98909EBC100ADF804003020ADF8EC
:102150003400287B0A90001FC0B20F90002CEBD0F7
:102160006181B5F81090002727E000BFCDF80090FE
:102170006888696903AA0A9B00F013FB0A9904EBBB
:10218000C70809EB01001FFA80F908F10C0204A945
:102190000F980EF049FD18B188F80EB0A8F80CB0F1
:1021A00001E0D4E0D1E0BDF80C10A8F81010BDF8A3
:1021B0000E107F1CA8F81210BFB26089B842D5D8A3
:1021C000C8E00DA8009001AB224629463046FFF733
:1021D00006FBBFE0307B082805D0FFDF03E0307B43
:1021E000082800D0FFDFE8891030ADF80400362061
:1021F000ADF83400002C3FD0A9896181F189A1811B
:1022000027E0307B092800D0FFDFA88900F10C010E
:10221000ADF804103721ADF83410002C2CD06081BB
:10222000E8890090AB89688804F10C02296956E0BE
:10223000E8893921103080B2ADF80400ADF83410CF
:10224000002C74D0A9896181287A10280AD0022133
:102250002173E989E181288A0090EB89688869699E
:10226000039A3CE00121F3E70DA8009001AB224660
:1022700029463046FFF744FB6CE0307B0A2800D04B
:10228000FFDF1220ADF80400ADF834704CB3A9891B
:102290006181A4F810B0A4F80EB084F80C8059E065
:1022A00020E002E031E039E042E0307B0B2800D052
:1022B000FFDF288AADF834701230ADF8040084B125
:1022C00004212173A9896181E989E181298A218217
:1022D000688A00902B8A688804F11202696900F00C
:1022E00060FA37E0307B0C2800D0FFDF1220ADF819
:1022F0000400ADF834703CB305212173A4F80AB092
:10230000A4F80EB0A4F810B024E00DA8009001AB22
:10231000224629463046FFF747FA1BE00DA80090F9
:1023200001AB224629463046FFF7A1FB12E035E01B
:102330003B21ADF80400ADF834107CB3A4F806805E
:10234000A4F808B084F80AB004E0FFDF02E0012935
:102350001BD0FFDFBDF80400AAF8000094B1BDF85F
:1023600034002080BDF804006080BDF834003928B6
:1023700008D03B2806D001E0100000203C2801D006
:1023800086F80CB0002011B0D2E43C21ADF8040076
:10239000ADF8341014B1697AA172DBE7FFE7AAF84F
:1023A0000000EFE72DE9F84356880F4680461546B2
:1023B000052130460CF0C8FF040000D1FFDF1234C5
:1023C00000943B46414630466A6808F001F9CBE587
:1023D00070B50D4605210CF0B7FF040000D1FFDFFA
:1023E000294604F11200BDE8704007F0FFBE70B549
:1023F0000D4605210CF0A8FF040000D1FFDF29469F
:1024000004F11200BDE8704007F023BF70B5054627
:1024100005210CF099FF040000D1FFDF04F108034F
:1024200021462846BDE870400422BDE470B505464B
:1024300005210CF089FF040000D1FFDF214628466A
:102440002368BDE870400522AEE42DE9F0478246DE
:1024500005210CF079FF040000D1FFDF04F1120028
:1024600007F0B7FE401D20F0030626E0011D00889E
:102470000322431821465046FFF796FC002820D03F
:10248000607B656870431FFA80F82888B7B2814680
:1024900010FA86F080B22880404502D3A0EB0800F5
:1024A00028806888B84200D2FFDF09EB0701414568
:1024B00000D9FFDF6888C01B6880606841880029F8
:1024C000D4D1BDE8F08770B50E46054606F07BFF17
:1024D000040000D1FFDF0120207266726580207841
:1024E00020F00F00C01C20F0F00030302070BDE85C
:1024F000704006F06BBF2DE9F0438BB00D461446DB
:10250000814606A9FFF76BFB002814D14FF6FF7632
:1025100001274FF420588CB103208DF800001020C3
:10252000ADF8100007A8059007AA204604A90EF0F0
:102530009AFB78B107200BB0BDE8F0830820ADF816
:1025400008508DF80E708DF80000ADF80A60ADF8F7
:102550000C800CE00698A17801742188C1818DF867
:102560000E70ADF80850ADF80C80ADF80A606A4600
:1025700002214846069BFFF762FBDCE708B5012213
:102580008DF8022042F60202ADF800200A4603232D
:102590006946FFF735FC08BD08B501228DF8022019
:1025A00042F60302ADF800200A4604236946FFF70D
:1025B00027FC08BD00B587B079B102228DF8002054
:1025C0000A88ADF808204988ADF80A1000236A4649
:1025D0000521FFF734FB07B000BD1020FBE709B170
:1025E00007230DE40720704770B588B00D461446E8
:1025F000064606A9FFF7F3FA00280ED17CB10620A3
:10260000ADF808508DF80000ADF80A40069B6A4608
:102610000821DC813046FFF712FB08B070BD0520B1
:102620008DF80000ADF80850F0E700B587B059B15B
:1026300007238DF80030ADF80820039100236A4687
:102640000921FFF7FCFAC6E71020C4E770B588B08F
:102650000C460646002506A9FFF7C1FA0028DCD182
:1026600006980121123007F0ECFD9CB12178062973
:1026700021D2DFE801F0200505160318801E80B284
:10268000C01EE28880B20AB1A3681BB1824203D99E
:102690000C20C2E71020C0E7042904D0A08850B95C
:1026A00001E00620B9E7012913D0022905D0042949
:1026B0001CD005292AD00720AFE709208DF800009B
:1026C0006088ADF80800E088ADF80A00A0680390C3
:1026D00023E00C208DF800006088ADF80800E08849
:1026E000ADF80A00A0680A25039016E00D208DF8C9
:1026F00000006088ADF80800A088ADF80A00E08806
:10270000ADF80C00A0680B25049006E00E208DF8B3
:10271000000060788DF808000C256A46294630468E
:10272000069BFFF78CFA78E700B587B00F228DF88B
:102730000020ADF8081000236A461946FFF77FFA1B
:1027400049E700B587B071B102228DF800200A88F0
:10275000ADF808204988ADF80A1000236A46062122
:10276000FFF76DFA37E7102035E770B586B00646FB
:1027700001200D46ADF808108DF800000146002339
:102780006A463046FFF75BFA040008D12946304616
:1027900005F022FC0021304605F03CFC204606B046
:1027A00070BDF8B51C4615460E46069F0CF0D7FEC8
:1027B0002346FF1DBCB231462A4600940CF035FB7F
:1027C000F8BD10B548800878144620F00F00C01CF2
:1027D00020F0F00090300B4608701822214603F1DB
:1027E00008001BF09EFBBDE8104006F0EFBD70B581
:1027F0000C460546FFF720FB2146284605F0FBFB6B
:102800002846BDE87040012105F004BC4FF0E022ED
:102810004FF400410020C2F880112049087020497F
:1028200090020860704730B51C4D04462878A042DD
:1028300018BF002C02D0002818BFFFDF2878A04264
:1028400008BF30BD2C701749154A0020ECB1164D59
:10285000DFF858C0131F012C0DD0022C1CBFFFDF66
:1028600030BD086003200860CCF800504FF4000031
:102870001060186030BD086002200860CCF800507D
:102880004FF040701060186030BD086008604FF075
:102890006070106030BD00B5FFDF00BD1800002083
:1028A00008F5014000F500400403002014F5004045
:1028B00070B50B2000F0B5F9082000F0B2F9002146
:1028C0000B2000F0C4F90021082000F0C0F9EC4C06
:1028D00001256560A5600020C4F84001C4F84401EA
:1028E000C4F848010B2000F0A7F9082000F0A4F973
:1028F0000B2000F08BF9256070BD10B50B2000F0A7
:1029000090F9082000F08DF9DD48012141608160D7
:10291000DC490A68002AFCD10021C0F84011C0F847
:102920004411C0F848110B2000F086F9BDE81040B2
:10293000082000F081B910B50B2000F07DF9BDE84A
:102940001040082000F078B900B530B1012806D059
:10295000022806D0FFDF002000BDCB4800BDCB48D9
:1029600000BDCA48001D00BD70B5C9494FF0004008
:102970000860C84DC00BC5F80803C74800240460B0
:10298000C5F840410820C43500F04BF9C5F83C417A
:10299000C248047070BD08B5B94A002128B10128A9
:1029A00011D002281CD0FFDF08BD4FF48030C2F8E0
:1029B0000803C2F84803B3483C300160C2F8401134
:1029C000BDE80840D0E74FF40030C2F80803C2F871
:1029D0004803AC4840300160C2F84411AB480CE0F9
:1029E0004FF48020C2F80803C2F84803A5484430D9
:1029F0000160C2F84811A548001D0068009008BD9C
:102A000070B516460D460446022800D9FFDF0022A5
:102A10009B48012304F110018B4000EB8401C1F8B5
:102A2000405526B1C1F84021C0F8043303E0C0F896
:102A30000833C1F84021C0F8443370BD2DE9F0419E
:102A40001C46154630B1012834D0022839D0FFDFAA
:102A5000BDE8F081891E002221F07F411046FFF77A
:102A6000CFFF012C24D000208C4E8A4F012470709F
:102A70003C61894900203C3908600220091D08603A
:102A8000854904203039086083483D350560C7F822
:102A90000042082000F0D0F82004C7F80403082002
:102AA00000F0B4F87A49E007091F08603470CFE7F6
:102AB0000120D9E7012B02D00022012005E00122EC
:102AC000FBE7012B04D000220220BDE8F04197E78C
:102AD0000122F9E76B480068704770B500F0C7F84D
:102AE000674C0546D4F840010026012809D1D4F8E6
:102AF0000803C00305D54FF48030C4F80803C4F8B8
:102B00004061D4F8440101280CD1D4F808038003B3
:102B100008D54FF40030C4F80803C4F8446101201C
:102B20000EF030FFD4F8480101280CD1D4F8080386
:102B3000400308D54FF48020C4F80803C4F8486166
:102B400002200EF01FFF5648056070BD70B500F002
:102B50008EF8524D0446287858B1FFF705FF687883
:102B600020B1002085F801000EF00CFF4C480460F5
:102B700070BD0320F8E74FF0E0214FF40010C1F8DA
:102B800000027047152000F057B842490120086143
:102B9000082000F051B83F494FF47C10C1F80803F9
:102BA0000020024601EB8003C3F84025C3F8402112
:102BB000401CC0B20628F5D37047410A43F60952BB
:102BC0005143C0F3080010FB02F000F5807001EBE8
:102BD0005020704710B5430B48F2376463431B0C19
:102BE0005C020C602F4C03FB04002F4B4CF2F724CB
:102BF00043435B0D13FB04F404EB402000F58070AD
:102C00004012107008681844086010BD00F01F02E0
:102C1000012191404009800000F1E020C0F800113E
:102C2000704700F01F02012191404009800000F12F
:102C3000E020C0F88011704700F01F020121914090
:102C40004009800000F1E020C0F880127047490779
:102C5000090E002806DA00F00F0000F1E02080F8ED
:102C6000141D704700F1E02080F8001470470C48F4
:102C7000001F00680A4A0D49121D116070470000CC
:102C800000B0004004B500404081004044B1004025
:102C900008F5014000800040408500402C000020E5
:102CA00014050240F7C2FFFF6F0C01000100000194
:102CB0000A4810B5046809490948083108600EF04F
:102CC000FEFE0648001D046010BD06490020086095
:102CD0004FF0E0210220C1F8800270471005024049
:102CE00001000001FC1F004010B50D2000F06FF83E
:102CF000C4B26FF0040000F06AF8C0B2844200D0A1
:102D0000FFDF3A490120086010BD70B50D2000F0CA
:102D100048F8374C0020C4F800010125C4F80453DA
:102D20000D2000F049F825604FF0E0216014C1F853
:102D3000000170BD10B50D2000F033F82C480121C2
:102D400041600021C0F80011BDE810400D2000F0E6
:102D500033B8284810B50468264927480831086068
:102D60002349D1F80001012804D0FFDF2148001DCC
:102D7000046010BD1D48001D00680022C0B2C1F8EB
:102D800000210FF06EFAF1E710B51948D0F80011E4
:102D90000029FBD0FFF7DDFFBDE810400D2000F05B
:102DA0000BB800F01F02012191404009800000F1A2
:102DB000E020C0F88011704700F01F02012191400F
:102DC0004009800000F1E020C0F880127047002820
:102DD00006DA00F00F0000F1E02090F8140D03E097
:102DE00000F1E02090F800044009704704D500404D
:102DF00000D00040100502400100000110B5202065
:102E000000F075F8202000F07DF84449202081F87A
:102E10000004434900060860091D42480860FEF7A7
:102E20006BFA3F49C83108603F48D0F8041341F0BD
:102E30000101C0F80413D0F8041341F08071C0F808
:102E40000413364901201C39C1F8000110BD10B52A
:102E5000202000F04CF8324800210160001D016084
:102E60002F4A481EE83A10602F4AC2F808032C4B3C
:102E7000C8331960C2F80001C2F860012B4908602C
:102E8000BDE81040202000F03DB825492848EC3925
:102E90000860704722492648E8390860704770B5D5
:102EA0001F4A8069E83A224911601F49D1F8006140
:102EB0000023204D1D4A5C1E1EB1A84206D30021EE
:102EC0000FE0D1F8606186B1A84209D2C1F80031A3
:102ED000C1F860311460BDE87040202000F012B8E5
:102EE0001168BDE870401BF097B8FFDF70BD00F0BF
:102EF0001F02012191404009800000F1E020C0F84C
:102F00008011704700F01F020121914040098000AC
:102F100000F1E020C0F880127047000020E000E0DF
:102F2000000602406412002000000240000402403B
:102F30000100000100F001000F4A12680D498A42A9
:102F40000CD118470C4A12680A4B9A4206D101B5B7
:102F50000FF040FAFFF799FFBDE801400749096803
:102F60000958084706480749054A064B70470000BC
:102F700000000000BEBAFECAA0000020040000202D
:102F8000E8110020E811002070B50C46054607F056
:102F9000BCFC21462846BDE8704008F0AEBD10B527
:102FA0000FF02EFEFFF732FC0FF0FEFCBDE81040E4
:102FB0000FF0B0BD0548064A0168914201D10021D9
:102FC000016004490120086070470000A000002053
:102FD000BEBAFECA40E5014070477047704770476F
:102FE000704702F0FF0343EA032242EA02421AF06A
:102FF000CCBF70477047704770470004050601005A
:1030000018FFFFFFDBE5B15100F001009800FFFF62
:103010008400000002093D0030B5FF4D0446102831
:103020000AD0112C06D02846122CC17806D0132CB9
:1030300008D0FFDFEC7030BDFFDFFBE71129F9D0CE
:10304000FFDFF7E71129F5D0FFDFF3E770B50DF0EB
:1030500075FF04460EF094FF201AC4B206200CF04F
:103060001DF9054606200CF021F92E1A07200CF058
:1030700015F9054607200CF019F9E749281A321806
:10308000C87812280DD000231A4413280BD0002032
:1030900002440878022808D000201044201AC0B248
:1030A00070BD0123F0E70120F2E70120F5E7DA48DF
:1030B00000B58079D849420897B051F8070F898840
:1030C0000CD017228DF80020CDF80200ADF80610C4
:1030D0000BA9684609F0B0F917B000BD4022F1E72E
:1030E00002210CF031B92DE9F04196B01D46904611
:1030F0000E460746FFF7F4FF04000BD02078222885
:1031000004D3A07FC0F34010A84206D1082016B017
:10311000BDE8F08143F20200F9E745208DF8000098
:10312000ADF802703DB101208DF804008DF8056006
:103130008DF8068002E000208DF804000BA9684697
:1031400009F07AF9A07F65F34510A0770020DEE74B
:1031500030B50446A1F120000D460A284AD2DFE826
:1031600000F005070C1C2328353A3F44FFDF42E0FE
:10317000207820283FD1FFDF3DE0A74801780329D0
:1031800039D0C078132836D02078242833D0252889
:1031900031D023282FD0FFDF2DE0207822282AD01D
:1031A000232828D8FFDF26E02078222823D0FFDF3D
:1031B00021E0207822281ED024281CD026281AD0CE
:1031C000272818D0292816D0FFDF14E020782528DA
:1031D00011D0FFDF0FE0207825280CD0FFDF0AE0B8
:1031E0002078252807D0FFDF05E02078282802D0A6
:1031F000FFDF00E0FFDF257030BD30B50B8840F603
:103200007B444FF6FF72022801D0934204D09D1FE9
:10321000A54224D2022802D04D88954203D04D8881
:10322000AD1FA5421BD24C88A34218D88B88B3F59A
:10323000FA7F14D2022802D0C888904205D0C888EC
:1032400040F677450A38A84209D2C888904208D08B
:10325000944206D05B1C6343B3EB800F01DB072075
:1032600030BD002030BD70B514460D4606460FF047
:103270002FFB60B90DB1A54201D90C2070BD00240F
:1032800009E000BF56F824000FF022FB08B110201F
:1032900070BD641CE4B2AC42F4D3002070BDF0B544
:1032A0000024059D10B1A94203D850E009B90020BF
:1032B000F0BD0920F0BD055DD5B1071997F801C033
:1032C000BCF1150F2DD03BDCBCF1150F38D2DFE877
:1032D0000CF037122020262628282F2F3737373793
:1032E0003737373737372000025D22BB641CE4B222
:1032F0008C42F9D3DBE7022DDBD1BD781D70072DA1
:1033000001D26D0701D40A20F0BD157845F0010502
:1033100015E0EF43FF0707E0012D07D010E006207E
:10332000F0BD2F07A7F18057002FF5D03046F0BD34
:103330001578AF0701D50B20F0BD45F002051570DB
:10334000055D641C2C44E4B28C4202D9B1E74FF411
:1033500048568C42AFD3AAE710B50278540809D07A
:10336000012243F20223012C07D0022C0DD0032CA2
:1033700013D10FE00020087005E080790324B4EB3E
:10338000901F0AD10A70002010BD8079B2EB901F07
:1033900003D1F7E780798009F4D0184610BD1E4AA2
:1033A000117C39B1517C022908D0032908D043F29D
:1033B000022070470146901D01F08ABC032100E005
:1033C000012101700020704738B50C46054669465A
:1033D00001F07EFC00280DD19DF80010207861F3EB
:1033E0004700207055F8010FC4F80100A888A4F820
:1033F0000500002038BD38B51378E8B102281BD08D
:1034000006A46D46246800944C7905EB9414247846
:1034100064F34703137003E0B00100200302FF01CF
:1034200003280ED003F0FE0010700868C2F80100F7
:103430008888A2F8050038BD23F0FE031370022827
:10344000E9D1D8B240F00100EEE730B50C4609787A
:1034500097B0222902D2082017B030BD28218DF85C
:103460000010ADF80200132A03D03B2A01D0072038
:10347000F2E78DF804200BA9684608F0DDFF05008F
:1034800003D121212046FFF763FE2846E4E700B57B
:1034900097B023218DF80010ADF802001088ADF828
:1034A00004005088ADF80600D088ADF80A00908876
:1034B000ADF808000020ADF80C00ADF80E000BA927
:1034C000684608F0B9FF07E62DE9FF470220FB4EEA
:1034D0008DF804000027B08AADF80600B84643F224
:1034E00002094DE001A80BF098FE050006D0B08A55
:1034F000A8B3A6F81480ADF806803FE0039CA07F37
:1035000001072DD504F124000090A28EBDF808001B
:10351000214604F1360301F0E4FD050005D04D45D8
:103520002BD0112D3DD0FFDF3BE0A07F20F0080025
:10353000A077E07F810861F30000C10861F34100DA
:10354000E07794F8210000F01F0084F82000207834
:10355000282827D129212046FFF7FAFD22E015E08F
:1035600040070BD5BDF80800214604F10E02FFF715
:103570008EFF05000DD04D4510D100257F1CFFB2F8
:1035800002200BF08BFE401CB842ABD8052D12D0A8
:1035900008E0A07F20F00400A07703E0112D00D008
:1035A000FFDF0025BDF80600B082052D05D02846B6
:1035B00004B0BDE8F087A6F814800020F8E72DE9F4
:1035C000FE43040000D1FFDF2078002720F00F0029
:1035D000801C20F0F000703020706068B74E0178D9
:1035E000091F15290DD2DFE801F0FD0B0C49FC0C79
:1035F0000EFCFC36FD0C0CFD6BFD0C0CFDFDFB0008
:10360000FFDFBDE8FE8385882846FFF769FD0400DB
:1036100000D1FFDF05F0DAFEB07C212140F004008C
:10362000B0742046FFF794FD284609F0F9F82846C3
:10363000FEF709FD284603F0D5FF294602200FF0CA
:1036400003F9A07F20F01000A077FFF73DFF0028CE
:10365000D7D0FFDFD5E785882846FFF741FD00B9C1
:10366000FFDF60688078012800D0FFDF6068817923
:1036700003B02846BDE8F04309F036BA86883046E4
:10368000FFF72EFD050000D1FFDF05F09FFE60680B
:103690003146C088288160680089688160684089F7
:1036A000A88102200FF0D0F8AF75A87F00F00300CA
:1036B0000228A6D1FFF708FF0028A2D0FFDFA0E76D
:1036C00080783C281CD0002502280ED08DF8007090
:1036D00000B1FFDF05F07AFEB07C40F00800B07466
:1036E00095B1B07801F0D4FA01208DF8000000BF48
:1036F0009DF80000012876D0022875D0FFDF80E712
:1037000001258DF80070E5E76568B5F80490A879A3
:10371000AD1C012806D03079804605F009FC070071
:1037200003D101E0B078F7E7FFDF0022022148462D
:103730000BF001FE040000D1FFDF22212046FFF73D
:1037400007FD2879012800D002208DF80000A17F14
:103750006A4660F30101A177288B2081688B608124
:10376000A88BA08184F82280032148460BF0E3FD5A
:1037700000B9FFDFB888ADF80800B8788DF80A0006
:1037800002AA052148460BF0D6FD00B9FFDFB88834
:10379000ADF80400F8788DF8060001AA0421484627
:1037A0000BF0C9FD00B9FFDF062105F1120001F0A1
:1037B000BAFA30B36879800700D5FFDF6979E07D18
:1037C00061F34700E075D5F80600A0616889A08321
:1037D000062105F10C0001F0A6FAE0B1B07904E091
:1037E00041E03BE046E021E02CE04108607861F3F5
:1037F00047006070D6F80700C4F80200B6F80B0066
:1038000012E0E07D20F0FE00801CE075D5F812008B
:10381000A061E88ADBE7607820F0FE00801C607021
:10382000E868C4F80200288AE08061E7307803285D
:1038300000D0FFDF002108460FF006F8012001F05C
:10384000F6F9DEE6F078132800D0FFDF002107202C
:103850000EF0FAFF1120FFF7DFFBD2E62046BDE8AD
:10386000FE4301F0FFBE05F0B1FDB07C40F040002A
:10387000B074C6E6BDE8FE4305F0A8BD2DE9F05FD3
:10388000054600780C4600270109DFF830A0914674
:103890003E4601296FD000234FF6FF7002296BD0FE
:1038A00007290DD00A2968D0FFDF00BFA9F8006002
:1038B0000CB1278066800020BDE8F09FB001002099
:1038C000D5F804C004F108029CF80010122973D046
:1038D0000EDC04F118080A2913D004DC042969D08D
:1038E000072968D14AE00E295AD01129F9D1C6E03A
:1038F00013297CD0162949D0172979D01829F0D15D
:1039000003E111270926002C73D0BCF8048040463F
:10391000FFF7E6FB90F822B0A4F80480686880798D
:1039200020729AF81210404621F004018AF8121011
:1039300004210BF01BFD052140460BF017FD002173
:1039400040460BF013FD012140460BF00FFD032113
:1039500040460BF00BFD022140460BF007FD06210F
:1039600040460BF003FD072140460BF0FFFC584694
:1039700001F08EF99AE7E7E012E1DFE01227102666
:10398000BCF80400214601F0BBF98FE71C2709268B
:103990007CB3BCF80200A08068680079207285E7DB
:1039A0001B2709262CB30420207268684088A08059
:1039B0007CE701E037E0C0E09CF802003C2828D01A
:1039C000102718260CF1020C9CB1BCF80200A08054
:1039D000BCF818006082BCF818002082BCF81A00FD
:1039E000A082BCF81C00E0829CF8050002E078E0B0
:1039F00067E00BE00CF10601FFF7FDFC9CF804000A
:103A000010B10120E07309E00220FBE7A9F8006093
:103A100051E71B270926002CF8D023729AF81210C0
:103A200021F00801CFE01D273726002CEED0A08022
:103A30006968481D0B7901461846FFF7DCFC686889
:103A400090F82B00A0756868C0780428E07D13D03A
:103A500020F00100E07569681F22C97861F3420017
:103A6000E0756968C97A61F3C700E0756968404626
:103A70000C311AF011FA19E740F00100EAE71D27AE
:103A80003726002CC2D0A08069680879491DFFF74D
:103A9000B2FC686804F10F0200F10C01C07AFFF774
:103AA000AAFC6868807CA0756868C178E07D61F3D5
:103AB000420020F0F900E0751F2140461AF085FA17
:103AC000F4E620271026002CA0D0A080686804F11E
:103AD0000902407A20726868C11C8078FFF78BFC6D
:103AE000E4E622271026002C90D0BCF80200A0802B
:103AF0006868007920816868007A60816868C08899
:103B0000A08168684089E081D0E621271026002C3A
:103B10008CD0BCF80200A08068688088208168682A
:103B2000C088608168680089A08168684089E081F8
:103B30009AF8121021F0400145E04A4621462846F5
:103B4000BDE8F05F01F02ABF287A012803D00228DF
:103B500014D0FFDFAAE61F271026002C92D0688819
:103B6000A08068892081A8896081E889A081288A4D
:103B7000E0819AF8121021F0200124E0122710268B
:103B80006888214601F0BCF8002C9DD0687800F0D0
:103B90000700052894D19AF8121021F0020112E0D2
:103BA000297A062923D2DFE801F004111103030367
:103BB000C3E71B270926002C86D0A08023729AF821
:103BC000121021F001018AF812106FE61B27092656
:103BD000002C89D0A080287A012806D003202072EA
:103BE0009AF8121021F01001EDE70220F7E7FFDF4D
:103BF0005CE630B5F74D97B0E878132801D008207F
:103C00002AE422208DF800000BA9684608F014FC75
:103C1000040002D1287901F03BF8002107200EF0C2
:103C200013FE204618E400B5EA4897B0C078122881
:103C300001D0082047E41E208DF8000000208DF8F8
:103C400002008DF803000BA9684608F0F5FB002878
:103C5000F0D1002107200EF0F7FD1120FFF7DCF96D
:103C6000002030E410B5DB4C96B02078012813D04A
:103C70001B208DF8000000208DF802000BA968467B
:103C800008F0DAFB002808D1002108460EF0DCFD20
:103C90002078032803D005E0082016B010BDA078D6
:103CA00000F0F6FF012000F0C2FF0020F5E72DE94B
:103CB000F041C84C002740B102281DD0072842D04F
:103CC000082800D0FFDFBDE8F081FFF7CBFF002818
:103CD000F9D105F078FB0028F5D0017821F00F012B
:103CE000891C21F0F00120310170077205F06EFB94
:103CF000A07C40F001001DE08EB23046FFF7F0F9E5
:103D0000050000D1FFDF28782128DCD005F05BFB1F
:103D100090B1017821F00F01891C21F0F0011031E0
:103D20000170022101724680AF7505F04FFBA07C47
:103D300040F00200A074C6E729463046BDE8F041D5
:103D40001322FFF782BBE578122D03D0132D04D088
:103D5000FFDFB8E7FFF767FF01E0FFF74AFF002842
:103D6000B1D105F030FB0028ADD0017821F00F0172
:103D7000891C21F0F00120310170122D07D00221A1
:103D8000017205F023FBA07C40F01000D2E7012176
:103D9000F6E72DE9F04116460C00074600D1FFDF9B
:103DA000307820F00F00801C20F0F00010303070D0
:103DB0002078012803D0022817D0FFDF83E7384698
:103DC000FFF78EF9050000D1FFDF0320A87505F08D
:103DD000FDFA2068B0606068F060208930827D481C
:103DE000817C41F0200181746DE73846FFF778F956
:103DF000050000D1FFDF61884FF6FF70814209D1D5
:103E0000A288824206D129463846BDE8F0411322F5
:103E1000FFF71BBB814201D1A08848B105F0D6FA5B
:103E20002068B0606068F06020893082002009E07E
:103E3000A87D0128C2D178230022394602200EF045
:103E400063FC0220A8753EE730B5054697B00C46E6
:103E500008460EF03DFD78BB00210120203D082DD5
:103E600070D2DFE805F004254C505A6772400021FB
:103E700008200EF0BFFC08B11120C1E624208DF807
:103E80000000D4F80200CDF80200A0798DF80600F9
:103E90000BA9684608F0D0FA050054D10823002287
:103EA000114618460EF030FC08284CD0FFDF4AE0DF
:103EB00060680EF051FD08B11020A1E646208DF893
:103EC00000002088ADF802006088ADF804000BA95E
:103ED000684608F0B1FA050035D1606848B3BDF80E
:103EE000301001802FE048208DF800002088ADF8C8
:103EF0000200A07800F001008DF8040014E02068B2
:103F000001F0EDFF14E0472208E000BF8DF8020049
:103F10000AE000BF8DF8021006E042228DF8002072
:103F20002278D207F6D0F1E70BA9684608F084FAA8
:103F3000054608E02178C90704D050218DF800100B
:103F4000E4E7FFE7072528465AE638208DF8000009
:103F50002088ADF802006088ADF80400E4E730B5D1
:103F6000054697B00C4608460EF0D8FC08B1102064
:103F700046E6203D082D27D2DFE805F0042424245E
:103F8000262626242088FFF7ABF820B100782228C7
:103F900004D2082034E643F2020031E625208DF8F1
:103FA00000002088ADF802000BA9684608F044FA2A
:103FB0000028DDD1DDF83210C4F802109DF836106B
:103FC000A1711DE606201BE6072019E60148801DA9
:103FD00070470000B001002038B51621FE4819F0E6
:103FE000D2FF012000F023FE1120FFF715F8FA4C54
:103FF0006846E11D05F048F99DF80010A07961F3CD
:10400000470020F00100A071002020744FF461707F
:10401000E08102206074FFF74AF800B1FFDFFDF78E
:1040200093F901F0DAFA38BD10B50C463E2120466E
:1040300019F0A9FFA07F20F00300A07720202070B6
:104040000020A07584F8230010BDC1E77CB50546AB
:104050000EF03EFC08B110207CBDDF4CA11DD4F851
:1040600006000090D4F80A0001902846FFF7ACF94A
:104070000028F1D1FFF71BF80028EDD00099C4F813
:104080000610BDF8041061819DF8061021737CBDF7
:1040900010B504460EF042FC08B1102010BDCE4908
:1040A00022468879C91D4008FFF7A5F9002010BDF8
:1040B0002DE9F0479CB00D4604004FF0000812D0E7
:1040C0000822FFF7D0F800281CD1002609E000BF25
:1040D00054F8260004A9FFF73FF9002812D1761CF6
:1040E000F6B2AE42F4D32F460A2006AD0DF1440AD3
:1040F0008DF8180026465146284608F09DF920B153
:1041000043F203201CB0BDE8F0874046DFF8C882C8
:1041100088F805002EB300244FF00B091DE000BF06
:1041200056F8240005A9FFF717F900B1FFDF9DF845
:104130001400A87056F8240050F8011FC5F80310A9
:104140008088A5F8070085F800905146284608F0B9
:1041500073F900B1FFDF641CE4B2BC42E0D388F81D
:1041600005700020CEE72DE9F0479EB01546894640
:1041700004001ED00F4608222946FFF774F80028D5
:1041800011D1002613E000BF54F8260005A9103015
:1041900000F09EFD002806D13FB157F826000EF032
:1041A00097FB10B110201EB0ADE7761CF6B2AE4200
:1041B000EAD30026A5F101081CE000BF06F1010AC0
:1041C0000AF0FF0712E000BF54F82600017C4A08FD
:1041D00054F827100B7CB2EB530F05D10622113097
:1041E000113119F02DFE78B17F1CFFB2AF42EBD335
:1041F0000AF0FF064645E1DBC8462E4607AD0DF145
:10420000480924B1012003E043F20520CBE7002058
:104210008DF81E0031208DF81C004946284608F014
:104220000BF938B934208DF81C004946284608F0AF
:1042300003F910B143F20420B5E77CB300272BE06B
:1042400054F82700A91C103000F042FD00B1FFDF38
:1042500054F82700102250F8111FC5F80310808869
:10426000A5F8070054F8271005F1090019F014FE0D
:10427000B8F1000F14D058F82710102205F11900DA
:1042800019F00AFE322028704946284608F0D4F872
:1042900000B1FFDF7F1CFFB2B742D1D3002082E71D
:1042A00005F1190001F00FFEECE770B596B0044679
:1042B0000EF00EFB18B960680EF057FB10B110201D
:1042C00016B070BD60884AF2B811884205D82078CF
:1042D000414D6E4618B1012804D00720F0E7FEF7E3
:1042E000E6FE1AE06078022804D0032802D043F2E8
:1042F0000220E5E7687417208DF80000697C002033
:10430000CDF80200ADF80600022932D003292DD0E5
:10431000FFDF0BA9684608F08FF80028D0D160684D
:1043200001F0C4FD207870B101208DF80200F01C6E
:1043300001F0C9FD4A208DF800000BA9684608F07D
:104340007BF800B1FFDF6088A8B1E88180B2ADF8EA
:10435000020030208DF800000BA9684608F06CF8C8
:1043600000B1FFDF207828740020A9E78DF807004E
:10437000CFE74020FAE74FF46170E6E710B5044656
:104380000EF0CCFA20B9606838B10EF0E5FA08B149
:10439000102010BD606801F096FD0F48C189618052
:1043A000417C6170007C2070002010BD2DE9F0413F
:1043B0009CB0054600208DF864008DF860008DF8F3
:1043C00030008DF868001E461446884628460EF0D8
:1043D000CCFA30B9204601E0B00100200EF0C5FA59
:1043E00010B110201CB06EE455EA040018D01F274D
:1043F0000CAB19AA414628460097FEF750FF00284B
:10440000F0D11AAB18AA314620460097FEF747FFB5
:104410000028E7D19DF86000C00703D00A20E1E73B
:104420000720DFE701AF7DB11A208DF804008DF879
:10443000068042462946F81C19F02EFD0DA901A858
:1044400007F0FAFF0028CDD17CB120208DF80400C0
:104450008DF8066032462146F81C19F01DFD0DA9A5
:1044600001A807F0E9FF0028BCD1FF499DF8300002
:1044700048700020B6E72DE9F0479CB08A464FF01F
:104480000008FAA104468DF83480D1E90001CDE995
:10449000190120460EF01CFA90B92078012803D1AA
:1044A00060680EF015FA58B9EF4D4FF00109287CFD
:1044B00040B1687C022805D160680EF056FA08B158
:1044C00010201FE62878012801D008201AE60720CE
:1044D0000AF0ECFE18B9207848B1012807D0FEF7A1
:1044E000B5FD30B1A87C10F00C0F08D103E012200C
:1044F00008E6132006E6C10701D1800701D5112087
:1045000000E6608943F6E172A0F120019142217832
:1045100007D301297ED100287CD1A189002979D136
:104520000FE0022901D0032901D1A02872D301296B
:1045300007D06978C90704D0A18900296AD0B429B5
:1045400068D8217831B1012908D0022904D0032983
:1045500060D10AE0002609E0022607E008B9A08938
:1045600008B1042609E0012607E00326287C50B1A3
:10457000687C022807D1606828B10DA96068FEF741
:10458000EBFE00289DD1207A30B1012806D0022808
:1045900006D0032878D105E0002704E0012702E0D7
:1045A000022700E003270EB1022E0ED16FB1687909
:1045B00080B36878800702D043F20120A2E5022E82
:1045C00003D1022F60D0032F5ED0207808B10128DC
:1045D00006D1504600F03FFB002889D185F802A0A3
:1045E00018208DF838006089ADF83A006089ADF880
:1045F0003C008DF83E600DF13F00FEF7D0FE00B1AB
:10460000FFDF9DF834008DF840002078012808D0A5
:10461000287C00E038E058B1687C022808D1606846
:1046200030B1606850F8011FCDF84110808802E079
:104630004046CDF84180ADF845008DF84870A07B2C
:10464000C0F34002014662F35F01C0F3800041EA1B
:10465000800019A9085C8DF84700A8B169460EA82A
:1046600007F0EAFE0028A9D11B208DF838008DF84C
:104670003A9069460EA807F0DFFE00289ED19DF80B
:1046800001001B281CD101E007203BE5052E0CD2C0
:10469000DFE806F0030308080300A87800F0EBFA4F
:1046A000032000E0022000F0C2FA012E0AD0A08907
:1046B00040B100228300114610460EF025F808B1E3
:1046C00003201FE500201DE52DE9FC4107460D46AE
:1046D000032608460EF049F9002867D13846FEF750
:1046E000FFFC040005D02078222805D20820BDE870
:1046F000FC8143F20200FAE7A07F00F0030C2DB129
:1047000029466046FEF779FD0600F0D15648BCF117
:10471000010F05D0BCF1020F1AD0FFDF3046E6E7EB
:10472000A27D2946022A02D0807C800701D5112073
:10473000DDE729B96846FCF715FF0028D7D169469F
:10474000384608F07FF90600E8D10120A075E5E7BA
:10475000A17D032914D1807C800611D425B1A07FCE
:1047600040070BD4002100E00121384608F095F9FC
:104770000600D3D1A075002DD0D002E01126CDE7E0
:10478000A5B12A4621463846FEF781FE0646112885
:10479000C4D1A07F4107C1D4296844F80E1F6968BD
:1047A000616040F0040020740026B7E710209EE707
:1047B00070B50C460546FEF793FC010005D0224675
:1047C0002846BDE87040FEF740BE43F2020070BDCF
:1047D00000B597B03F218DF800108DF802000BA9AD
:1047E000684607F029FE17B000BD0123FEF77BBC29
:1047F00000231A461946FEF776BC30B597B004463A
:104800000EF066F810B1102017B030BD204600F051
:1048100049FA0028F8D1144DE878112801D0082071
:10482000F2E7FEF713FC20B1A87CC00603D51120E7
:10483000EAE71320E8E72078800701D56879E8B334
:104840001D208DF800002078022200F001008DF874
:1048500002006088ADF80400A088ADF8060020785A
:10486000C0F3400106E00000B00100200706050487
:104870000302010002EA500001438DF8091002A86A
:10488000FEF78DFD00B1FFDF0BA9684607F0D4FDF0
:104890000028B9D11E208DF8000001208DF80200FB
:1048A00000208DF803000BA9684607F0C5FD00281D
:1048B000AAD1E08800F016FA040000E005E0A3D1D8
:1048C0001220FEF7A9FB20469EE707209CE72DE972
:1048D000F041FC4C074696B0E078984616460D46E7
:1048E000122803D1FFF79FF900280ED128460DF0BA
:1048F000EFFF70BB30460DF0EBFF50BBA07C10F01B
:10490000180F01D1400703D5112016B0BDE8F08182
:10491000284600F0C7F90028F7D131460220FEF7FB
:104920006CFC0028F1D1E078112801D00820ECE7D8
:1049300006200AF0BBFC50B12878800701D56079C9
:1049400040B1FEF783FB022806D21320DDE71220D8
:10495000DBE716E00720D8E721208DF80000688803
:10496000ADF80200A888ADF804002878C0F3400034
:104970008DF80600287880071CD438460DF0A8FF73
:1049800008B11020C1E73878420808D0012A18D0B1
:1049900043F20221022A18D0032A18D115E0C007D9
:1049A00000D002208DF8070057F8010F0290B88858
:1049B000ADF80C000DF10E00FEF7F1FC58B103202C
:1049C000A3E7C00705D00320ECE7C00701D00846E5
:1049D0009BE70120E6E73088ADF810007088ADF85D
:1049E0001200B088ADF81400F088ADF81600002071
:1049F000ADF81800ADF81A00404600F02CF9002878
:104A000083D184F804800BA9684607F015FD0028BF
:104A10008DD1207900F02FF9E88800F063F90400C7
:104A200085D11320FEF7F8FA20466EE730B505462B
:104A300097B00C4608460DF071FF08B11020E3E670
:104A40002846FEF74DFB38B10178222902D3807F3A
:104A5000800604D40820D7E643F20200D4E61320EF
:104A60008DF80000ADF802500BA9684607F0E4FC91
:104A70000028E4D19DF932107F2901D02170C3E6CE
:104A80000520C1E62DE9F043B1B015460C460646B7
:104A9000FEF726FB070006D03878222806D2082029
:104AA00031B0BDE8F08343F20200F9E720460DF093
:104AB0005CFF30B94FF000084DB128460DF04CFFB7
:104AC00008B11020ECE7C5F80080A5F804807D4807
:104AD000807C400601D51120E2E797F8220004F01F
:104AE00027FA8088011DFB2901D2001D00E0FB2070
:104AF000C0B2210007D0D1F8009064681FFA89F194
:104B0000002909D00AE060F30F0960F31F4900F0A3
:104B10008AF860F30F0411E060F30F095FEA1941AE
:104B200001D160F31F492004000C05D11FFA89F060
:104B300000F079F860F30F04200C05D14FEA19401A
:104B400000F071F860F31F442C225F490EA819F0A1
:104B5000E8F94FEA1940ADF83C00200CADF83E00F2
:104B6000ADF84090ADF83A60ADF842401BA90EA8F0
:104B700007F062FC00B1FFDFBDF87000ADF8640023
:104B8000BDF87200ADF86600BDF87400BDF876108F
:104B90000844ADF868001FFA89F107201B2984D367
:104BA0004FEA19421B2A8DD3FB298BD8FB2A89D8BF
:104BB000062791420CD1084600F035F8A1B2884290
:104BC00006D14FEA194000F02EF8210C884201D09E
:104BD000384665E7BDF8640028B9BDF8660010B92D
:104BE000BDF8680038B125B119982860BDF8680093
:104BF000A880132054E734492C222C3102A819F044
:104C000090F94FEA1940ADF80C00200CADF80E00F9
:104C1000ADF81090ADF80A60ADF8124026A902A8D0
:104C200007F00AFC3CE7C000703080B2704730B536
:104C3000244D040008D0012C04D0022C06D0032CF3
:104C400004D0FFDF2C7030BDFFDFFBE728780128A0
:104C5000F8D0FFDFF6E710B5044604F069F930B18B
:104C6000407830B1204604F06AFC002010BD0720D7
:104C700010BD122010BD10B504F05AF9040000D187
:104C8000FFDF607800B9FFDF6078401E607010BD04
:104C900010B504F04DF9040000D1FFDF6078401C2E
:104CA000607010BD418843F6FD730A1F9A420DD211
:104CB000808804280AD3B0F5804F07D8884205D8E9
:104CC00000207047B00100202CE301000720F8E726
:104CD0000278520804D0012A02D043F20220F0E701
:104CE000FEF73ABB10B548B18300002211460720F9
:104CF0000DF00AFD072801D0032010BD002010BDD3
:104D000070B50C0006460DD0FEF7EAF9050000D19B
:104D1000FFDFA68028892081288960816889A08199
:104D2000A889E08170BD10B500231A4603E0845CB9
:104D30002343521CD2B28A42F9D30BB1002010BDDA
:104D4000012010BD2DE9F0418846064601884088C3
:104D500015460C181F46AC4200D3641B3844A842C9
:104D600000D9FFDFE019A84200D9FFDF708838447E
:104D7000708008EB0400BDE8F08110B504460DF02A
:104D8000A7FD08B1102010BD2078C0F30210042840
:104D900007D86078072804D3A178102901D8814268
:104DA00001D2072010BDE078410706D421794A07D7
:104DB00003D4000701D4080701D5062010BD002048
:104DC00010BD10B513785C08C37F64F30003C3778C
:104DD0001478A40864F34103C3771078C3094878B2
:104DE00063F34100487013781C090B7864F3471390
:104DF0000B701378DB0863F300004870507848713B
:104E000010BD10B5C4780B7864F300030B70C47840
:104E1000640864F341030B70C478A40864F382034C
:104E20000B70C478E40864F3C3030B700379117842
:104E300063F30001117003795B0863F341011170A2
:104E400003799B0863F3820111700079C00860F355
:104E5000C301117010BD70B514460D46064604F02E
:104E6000B2FA80B10178142221F00F01891C21F0DF
:104E7000F001A03100F8081B214619F052F8BDE8F6
:104E8000704004F0A3BA29463046BDE870401322B2
:104E9000FEF7DBBA70B514460E46054604F093FAE9
:104EA00070B1017821F00F01891C21F0F00120314F
:104EB0000170458021688160BDE8704004F086BAC9
:104EC00031462846BDE870401322FEF7BEBA10B541
:104ED000FE4C94F8300000280CD104F120014FF66C
:104EE000FF72A1F110000BF026FE00B1FFDF0120E0
:104EF00084F8300010BD2DE9F047064608A8894621
:104F000090E830041F4690461421284619F05DF8B9
:104F10000021CAF80010B8F1000F03D0B9F1000F5A
:104F200003D114E03878C00711D020680DF0F6FCEA
:104F3000F0BBB8F1000F07D120681230286020685C
:104F4000143068602068A8602168CAF800103878BA
:104F5000800728D560680DF0FFFC48BBB9F1000F51
:104F60002DD0FFF733F80168C6F8C8118188A6F87C
:104F7000CC11807986F8CE01FFF7A9FFDFF84C83CA
:104F800008F12008C5F80C80626862B196F8C80183
:104F900006F2C91140081032FEF72DFA10224146E0
:104FA000606818F079FF3878400712D5A06800E0F3
:104FB00002E00DF0B3FC50B11020BDE8F08760684E
:104FC0000028F9D0E8606068C6F8C401EBE7A06883
:104FD00028610020F1E730B5054608780C4620F03E
:104FE0000F00401C20F0F001103121700020607093
:104FF00095F8230030B104280FD0052811D00628D9
:1050000014D0FFDF20780121B1EB101F04D295F8F6
:10501000200000F01F00607030BD21F0F000203053
:1050200002E021F0F00030302070EBE721F0F000DA
:105030004030F9E710B510B190F8BD4044B1A34835
:1050400090F83540002064B108601060186010BD11
:1050500000F1BC040C6000F1E40100F58670116001
:10506000F4E79A4C34340C60EFE700B58BB00723BB
:10507000CDE902128DF80130019194490023643189
:105080000591099301468DF8103068460BF02BFD11
:10509000002800D0FFDF0BB000BD70B590B0154602
:1050A0000C4602220646ADF80820082103AB07F0A3
:1050B000DAFA0490002812D00C208DF801000420A8
:1050C0008DF8040004F59A74099605948DF818502B
:1050D0000AA968460BF007FD00B1FFDF012010B000
:1050E00070BD30B597B00C462C251A998DF800503C
:1050F000ADF80200B3B11868019058680290ADF89D
:105100000C2010220DF10E0018F0C6FE0BA9684607
:1051100007F092F9002803D1A17F41F01001A17797
:1051200017B030BD00200190E8E72DE9F0470646B2
:10513000008A8CB080B20D468246FDF7D1FF04464E
:10514000624F3078283FDFF884814FF00009122841
:1051500073D2DFE800F072EF350936777E98A5F05C
:10516000EDECEBEAE95BE9E9A07F00F00300012840
:1051700006D0002150460AF0E7F8050003D101E00F
:105180000121F7E7FFDF98F85C10090602D5D8F88F
:1051900060000BE0032105F121000DF043F8D5F884
:1051A00021004B49B0FBF1F201FB1200C5F82100D0
:1051B0007068A867B068E8672078252800D0FFDF0E
:1051C000EAE0A07F00F00300012806D0002150464D
:1051D0000AF0BAF8060003D101E00121F7E7FFDF8A
:1051E0003078810702D52178252904D040F00100CC
:1051F00030700CB0E1E60220287096F8200028718B
:1052000006F121003136C5E90206F2E7A07F00F081
:105210000300012806D0002150460AF095F804004A
:1052200003D101E00121F7E7FFDF2078C10605D5B2
:105230001320287041346C60DBE7CCE140F00800BB
:105240002070D6E72148082128380CF0EBFF032016
:1052500016E02A208DF8000010220DF1020071687E
:1052600018F01AFE10220DF11200B16818F014FEA9
:10527000164968462C3907F0DFF800B1FFDF04203B
:1052800028706F60B5E7E07FC00600D5FFDFB0682B
:105290000090B38806220821504607F0F3FAA8E7E9
:1052A00004B9FFDF716821B1102204F1240018F065
:1052B000F3FD28212046FDF74BFFA07F00F00300FF
:1052C000022813D104F12400002303E0FC01002094
:1052D00040420F0000901A4621465046FFF701FF5A
:1052E000112807D029212046FDF732FF307A84F8B3
:1052F00020007EE7A07F000700D5FFDF14F81E0F17
:1053000040F008002070A4F81690C4F81890C4F873
:105310001C906178084661F38200410861F3C30084
:105320006070307AE07064E728E050E18CE082E061
:105330005AE000E037E0A07F00F00300012806D02B
:10534000002150460AF000F8040003D101E00121D9
:10535000F7E7FFDF022104F189000CF063FF102062
:10536000287004F5E4706860B4F88910298204F1AB
:105370008000FE496861C5E902813AE7A07F00F03C
:105380000300012805D00021504609F0DDFF18B9BF
:1053900001E00121F8E7FFDF0CB03246214650461C
:1053A000BDE8F04757E504B9FFDF20782128A0D9F0
:1053B0003079012802D002280AD103E0E07F40F0D2
:1053C0001000E07798F85C1041F0010188F85C105B
:1053D000324621465046FFF73EFD0CB02046BDE860
:1053E000F0472321FDF7B4BE3279AA8005F1080306
:1053F0000821504607F037F9E86008B1112021E094
:10540000A07F00F00300012806D00021504609F0DB
:105410009BFF040003D101E00121F7E7FFDF04F166
:10542000660102231022081FFFF78CFC80F8009011
:1054300031794170DDE60821504607F0F3FB002882
:105440009BD112202870D4E6A07F00F00300012831
:1054500006D00021504609F077FF050003D101E096
:105460000121F7E7FFDF95F8880000F0030001282D
:1054700078D1A07F00F00307E07FC0F3400616B1AB
:10548000012F04D02BE095F8A400C0072AD0D5F84E
:10549000C01119B395F88720087C62F3870008745F
:1054A000E27FD5F8C01162F341000874D5F8C0114D
:1054B00066F300000874AEB1D5F8C001102204F103
:1054C00024018C3518F0E8FC287E40F00100287695
:1054D000287820F0010005F88C0900E016B1022FB1
:1054E00004D02CE095F88C00C00726D0D5F8BC116C
:1054F00019B395F88720087C62F387000874E27F6F
:10550000D5F8BC1162F341000874D5F8BC1166F3FC
:10551000000008748EB1D5F8BC01102204F12401FA
:105520008C3518F0B9FC287840F0010005F8180B0C
:10553000287820F0010005F8A409022F43D00020AC
:1055400000EB400005EBC00090F88C00800709D507
:1055500095F88000D5F8C421400805F1810110328A
:10556000FDF749FF05208DF8000095F888006A4690
:1055700000F003008DF8010095F88C108DF80210F2
:1055800095F8A4008DF8030021465046FFF782FCF1
:105590002078252805D0212807D0FFDF2078222871
:1055A00003D922212046FDF7D3FDA07F00F00300A0
:1055B00001280AD00021504609F0D8FE00283FF407
:1055C00024AEFFDF15E60120BAE70121F3E7716899
:1055D00081F801900DE6FFDF0BE670B5634C002506
:1055E000103C14F85C0F20F08000207065600BF018
:1055F00042FA5E49A1F1100003F078FE04F82C5C39
:105600000620607259487C3020615030A061103013
:10561000E06170BD70B50D46FDF762FD040000D17C
:10562000FFDF4FF4E871284618F0CFFC4F485430A4
:10563000686104F124002861A07F00F003000128C4
:1056400008D0022105F59A700BF016FA002800D058
:10565000FFDF70BD0121F5E70A46014602F59A70A9
:105660000BF02ABA70B5054640689CB0017808294D
:1056700006D00B2937D00C2933D0FFDF1CB070BD0A
:1056800046883046FDF72CFD040000D1FFDF20786E
:105690002128F3D0282821D1686802210C3001F09C
:1056A000CEF9D8B168680821001D01F0C8F9A8B189
:1056B0002D208DF80000ADF80260102204F12401C5
:1056C00001A818F0E9FB0BA9684606F0B5FE00B189
:1056D000FFDF29212046FDF73BFDCFE703F076FEF3
:1056E000CCE701218171686886883046FDF7F8FCB7
:1056F000040000D1FFDFA07F00F00301022902D1E6
:1057000020F01000A077207821280AD068688179DD
:1057100009B1807880B1A07F00F00300022859D041
:10572000FFDFA07F00F003000228A7D1FDF7CCFE29
:105730000028A3D0FFDFA1E703F048FEE07FC10708
:1057400023D0800701D5062000E0052084F823003F
:10575000207829281BD02428E3D1314606200DF0DB
:1057600073F822212046FDF7F3FC01E00C02002033
:10577000A07F00F0030001282AD00021304609F064
:10578000F5FD0028CDD0FFDFCBE70420DEE7A07FCA
:1057900000F00300012806D00021304609F0D4FDB6
:1057A000050003D101E00121F7E7FFDF25212046B5
:1057B000FDF7CEFC0F208DF8580016A905F59A705C
:1057C0000BF071F90228ACD00028AAD0FFDFA8E7BF
:1057D0000121D3E703F0FAFDA3E72DE9F0438BB0F5
:1057E0009946154688460646FDF77AFC04004FD0D8
:1057F000207822284CD323284AD0E07FC00647D403
:10580000A07F00F00300012806D00021304609F0F7
:105810009BFD070002D00CE00121F7E7A07F00F01C
:105820000300012805D101210022304609F083FD43
:10583000074601AB02AA03A93846FFF7FBFB039812
:1058400000B9FFDF4FB1039807F59A778761207899
:10585000222806D0242804D007E00399002088617C
:1058600003E025212046FDF773FC03980B214170CE
:1058700046628580C0E9028902990161019941610E
:1058800004A90BF030F9022802D0002800D0FFDF75
:105890000BB0BDE8F083F0B587B00746FDF720FCFC
:1058A000017822291DD9807F00F00300012806D04D
:1058B0000021384609F048FD04003FD101E00121F4
:1058C000F7E7FFDF3AE000BFB4F8621004F16600CA
:1058D00008440178427831B121463846FFF7DDFBB4
:1058E000B8B907B0F0BDADF804200821384602ABC6
:1058F00006F0B9FE03900028F3D011208DF80000C7
:10590000694604F59A700BF0CEF8022801D000B178
:10591000FFDF04F162052E88B01C80B228801028B9
:1059200001D3103828806888022800D2FFDFB61C17
:10593000102E00D9FFDF6888801E6880B4F86400EC
:105940000028C1D1CDE730B587B00546FDF7C8FBCB
:105950000446007822281FD90821284607F062F95A
:10596000002819D1A07F00F00300012806D00021F3
:10597000284609F0E9FC040003D101E00121F7E722
:10598000FFDF12208DF80000694604F59A700BF0D5
:105990008AF8002800D0FFDF07B030BD2DE9F05FA6
:1059A00005460C4600270078904601093E46BB4656
:1059B00004F1080A02297CD0072902D00A2909D15A
:1059C00042E068680178082905D00B292CD00C2901
:1059D0002AD0FFDFC6E114271C26002C6AD040889D
:1059E000A080FDF77DFB5FEA000900D1FFDF99F899
:1059F00017005246400809F11801FDF7FCFC6868E1
:105A00008089208268684168C4F812108068C4F8F0
:105A10001600A07E20F0060040F00100A07699F864
:105A20001E0040F040014DE01A270A26002CD5D078
:105A30008088A080FDF754FB050000D1FFDF5146B0
:105A40002846FFF7C8FA8DE10CB1288BA080287A90
:105A50000E287CD006DC01287AD0022808D0032842
:105A600004D135E0102874D0112873D0FFDF79E11C
:105A70001E270926002CB1D0A088FDF731FB5FEA74
:105A8000000900D1FFDF287B00F003000128207A05
:105A90001BD020F001002072297B890861F34100AE
:105AA0002072297BC90861F382002072297B0909D1
:105AB00001E04CE119E161F3C300207299F81E0086
:105AC00040F0800189F81E104CE140F00100E2E74F
:105AD00013270D26002CAAD0A088FDF701FB8146D4
:105AE000807F00F00300012806D00021A08809F083
:105AF0002BFC050003D101E00121F7E7FFDF99F856
:105B00001E0000F00302012A59D0E86F817801F0ED
:105B100003010129217A54D021F0010121728378F7
:105B20009B0863F3410121728378DB0863F38201F0
:105B3000217283781B0963F3C3012172037863F335
:105B400006112172437863F3C711217203E060E00C
:105B5000A6E08EE09EE084F809B0C178A172012A27
:105B600032D04279E17A62F30001E172427952085F
:105B700062F34101E1724279920862F38201E172BB
:105B80004279D20862F3C301E1720279217B62F3A8
:105B9000000121730279520862F3410121730279F5
:105BA000920862F3820121730079C00860F3C30197
:105BB000217399F8000023285AD9262168E0A86F9C
:105BC000A4E741F00101A9E70279E17A62F300015B
:105BD000E1720279520862F34101E172027992089E
:105BE00062F38201E1720279D20862F3C301E172C9
:105BF0004279217B62F3000121734279520862F3FA
:105C0000410121734279920862F382012173407944
:105C1000CBE718271026002C67D0A088FDF760FA84
:105C20008246807F00F00300012807D00021A08871
:105C300009F08AFB5FEA000903D101E00121F6E7E0
:105C4000FFDFE868A06099F8000040F0040189F8DF
:105C5000001099F80100800708D5012020739AF8F8
:105C6000000023287ED92721504663E084F80CB039
:105C700078E015270F26C4B3A088FDF731FA8146D6
:105C800006225146E86806F03FFC0120A073AEE012
:105C900048464FE0162709263CB3287B207261E076
:105CA000297BFE4802290CD019270E26ECB10129C8
:105CB0000DD003291AD004291BD0052919D0FFDFE4
:105CC00023E01B270926BCB30121217205E0012135
:105CD0002172617A21F00301617210F85C1F4A0899
:105CE000520062F3060101700FE02BE002202072E7
:105CF00007E0687B052900F00F0040F0800020726B
:105D00001BD0607A20F003006072A088FDF7E8F9EC
:105D100005460078212825D0232800D0FFDFA87F62
:105D200000F00300012810D00021A08809F01EFB1C
:105D300022212846FDF70CFA14E0607A20F00300D7
:105D4000401CE1E7A8F8006011E00121EDE70CB18B
:105D50006888A080287A03282BD004280AD0052838
:105D60004BD0FFDFA8F800600CB1278066800020D0
:105D7000BDE8F09F15270F26002CE3D0A088FDF783
:105D8000AFF9807F00F00300012806D00021A08831
:105D900009F0DAFA050003D101E00121F7E7FFDF9E
:105DA000D5F821000622514606F0AEFB84F80EB06D
:105DB000D8E717270926002CC4D0A088FDF790F952
:105DC0008146807F00F00300012806D00021A088D2
:105DD00009F0BAFA050003D101E00121F7E7FFDF7E
:105DE0006878800701D5022000E00120207299F830
:105DF00000002328B6D927214AE719270E26002CB0
:105E0000A0D0A088FDF76CF95FEA000900D1FFDFA0
:105E1000C4F808B0A4F80CB084F808B0A07A40F038
:105E20000300A07299F81F1061F38200A07299F824
:105E30001F1001EA510161F3C300A072687A00F0FB
:105E4000030001288ED1607A40F00400607299F856
:105E50001E00E97A00F00300012813D0607B61F393
:105E600000006073AA7A217B62F300012173EA7A51
:105E7000520862F341006073A87A400860F3410160
:105E800021736FE7207B61F300002073AA7A617BA6
:105E900062F300016173EA7A520862F341002073F1
:105EA000A87A400860F3410161735BE710B57B4C51
:105EB00030B10146102204F1200017F0EDFF01205F
:105EC00084F8300010BD10B50446FFF700F87349A0
:105ED00020461022BDE81040203117F0DDBF70B51C
:105EE0006E4C06004FF0000514D00CF0F1FC08B128
:105EF00010250DE00621304606F0EDFA411C06D0D3
:105F0000206614F85C0F40F08000207000E0072548
:105F1000284670BD14F85C0F20F08000F5E700788B
:105F200010F00F0204D0012A05D0022A0CD110E093
:105F3000000909D10AE00009012807D0022805D08C
:105F4000032803D0042801D00720704708700020E0
:105F500070470620704705282AD2DFE800F00307C3
:105F60000F171F00087820F0FF001EE0087820F0CF
:105F70000F00401C20F0F000103016E0087820F0F0
:105F80000F00401C20F0F00020300EE0087820F0D8
:105F90000F00401C20F0F000303006E0087820F0C0
:105FA0000F00401C20F0F0004030087000207047C7
:105FB000072070472DE9F041804688B00D46002744
:105FC00008460CF0D2FCA8B94046FDF789F8040059
:105FD00003D02078222815D104E043F2020008B053
:105FE000BDE8F08145B9A07F010603D500F00300AC
:105FF000022801D01020F2E7A07FC10601D40107DA
:1060000002D50DB10820EAE7244991F85C10C907D0
:1060100001D01120E3E7E17FC90601D50D20DEE7BD
:1060200000F00300022805D125B12846FEF7A5FEA1
:106030000700D4D1A07F00F00300012806D0002182
:10604000404609F081F9060002D00DE00121F7E792
:10605000A07F00F0030001280CD000210022404660
:1060600009F069F9060007D0A07F00F003000228BC
:1060700004D009E00121F1E70420B0E725B12A4668
:1060800031462046FEF79DFE07AB1A46694630466C
:10609000FEF7D0FF009800B9FFDF01E0FC0100200F
:1060A00000990C20487006F59A70C1F82480486168
:1060B00000200881A07F00F00300012828D0EDB364
:1060C00002200871301D88613078400908777078A7
:1060D000C0F340004877287800F00102887F62F31F
:1060E00001008877E27F62F382008877E27F5208BE
:1060F00062F3C3008877727862F304108877A87817
:10610000C87701F1210228462031FEF77AFE22E00D
:1061100001200871287800F00102087E62F3010076
:1061200008762A78520862F3820008762A78920864
:1061300062F3C30008762A78D20800E007E062F331
:106140000410087624212046FDF702F80BE0032016
:1061500008710520087625212046FCF7F9FFA07F6D
:1061600020F08000A07701A900980AF0BCFC02286A
:1061700001D000B1FFDF384631E72DE9FF4FF94A82
:106180000D4699B09A4607CA14AB002783E807006A
:106190001998FCF7A5FF060006D03078262806D00F
:1061A00008201DB0BDE8F08F43F20200F9E7B07F90
:1061B00000F00309B9F1010F03D0B9F1020F07D0C4
:1061C00008E03DB91B98FEF7D8FD0028E9D101E0B1
:1061D0001B9878BBB07F00F00300012806D0002197
:1061E000199809F0B1F8040003D101E00121F7E7A3
:1061F000FFDF852D25D007DCD5B1812D1BD0822D69
:106200001BD0832D08D11AE0862D1CD0882D1CD0E0
:10621000892D1CD08A2D1CD00F2020710F281AD058
:1062200001208DF83400201D0E902079A8B158E18E
:106230000020F2E70FE00120EFE70220EDE7032066
:10624000EBE70520E9E70620E7E70820E5E7092076
:10625000E3E70A20E1E70720A3E7B9F1010F17D030
:10626000D4E91E5080460220019001200090A878B9
:1062700098F80210C0F3C000C1F3C00108405FEA03
:10628000000B5DD050460CF023FB00286CD12DE0B4
:10629000D4E91E850120019002200090214630465D
:1062A0001B9AFEF78EFD1B98007800F00101A8787C
:1062B00061F30100A870F17F61F38200A870F17FA3
:1062C000490861F3C300A870617861F30410A870F5
:1062D0002078400928706078C0F3400068701B98EF
:1062E0008078E870002068712871C0E7DAF80C0047
:1062F0000CF0EEFAC0BBDAF81C000CF0E9FA98BB1F
:10630000DAF80C00A060DAF81C00E06098F80100F0
:10631000617800F0010041EA4000607098F80210D6
:10632000C0B2C1F30011891E08406070002084F8DB
:106330002000009906F1170002290BD001210AE084
:1063400098F80110607801F00101FD2242EA410154
:106350000840E2E7002104EB810188610199701C8B
:10636000022902D0012101E028E0002104EB810193
:106370008861A87800F00300012849D198F802004C
:1063800000F00300012843D1B9F1010F04D12A1D07
:10639000691D1B98FEF735FD297998F80400014026
:1063A0008DF82C10687998F8052010408DF8300091
:1063B00001432DD050460CF08BFA08B11020F0E6C6
:1063C0000AF1100004F5DE7104F190020490B9F1B5
:1063D000020F3CD00090CDE9012100210BAB5A46C1
:1063E0002046FEF788FD0028E9D104F5E07104F1AC
:1063F000A802B9F1010F30D004980090CDE9012135
:1064000000210CAB5A462046FEF775FD0028D6D178
:106410006078800740D4A87898F80210C0F3800014
:10642000C1F38001084337D0297898F8000014AAF6
:10643000B9F1010F17D032F810204B00DA4012F0FA
:10644000030718D0012F1ED0022F12D11DE0CDF866
:1064500000A0CDE901210121C0E7CDF800A0CDE9E0
:1064600001210121CDE732F811204300DA4002F08A
:106470000307032F07D0BBF1000F0DD0012906D071
:10648000042904D008E00227F5E70127F3E70128F3
:1064900001D0042800D10427F07F40F001006BF305
:1064A0004100F077607881074FF003000CD5A071B0
:1064B000BBF1000F15D100BF8DF85C0017AA314663
:1064C0001998FEF7E7FC0CE00221022F18D0012FEB
:1064D00018D0042F22D00020A071F07F20F00100FE
:1064E000F07725213046FCF733FE0DA904F59A70AC
:1064F0000AF0D9FA10B1022800D0FFDF002050E6E0
:10650000A171D9E7A1710D2104F1240017F05DFDFF
:10651000207840F0020020700420CDE70120A07117
:10652000DFE72DE9F04387B0904689460446002511
:10653000FCF7D6FD060006D03078272806D00820C4
:1065400007B0BDE8F08343F20200F9E7B07F00F046
:106550000300012808D00021204608F0F5FE0400C1
:1065600005D103E084E301000121F5E7FFDFA7790E
:106570005FEA090005D0012821D0B9F1020F26D128
:1065800010E0B8F1000F22D1012F05D0022F05D065
:10659000032F05D0FFDF2DE00C252BE0012529E09E
:1065A000022527E040460CF093F9B0B9032F0ED135
:1065B0001022414604F1210017F06EFC1AE0012F71
:1065C00002D0022F03D104E0B8F1000F12D007204F
:1065D000B6E740460CF07CF908B11020B0E7102176
:1065E00004F1210017F0CFFC0621404605F073FFAF
:1065F000C4F821002078252140F0020020703046A8
:10660000FCF7A6FD2078C10714D020F0010020700F
:1066100002208DF8000004F1210002908DF8045052
:10662000694604F59A700AF03EFA022804D018B1BF
:10663000FFDF01E084F82050002081E730B587B00B
:106640000D460446FCF74CFD88B1807F00F0030046
:1066500001280FD00021204608F076FE04000ED05D
:1066600028460CF035F938B1102007B030BD43F2A0
:106670000200FAE70121EEE72078400701D4082064
:10668000F3E7294604F141002022054617F004FCF7
:10669000207840F01000207001070FD520F008008E
:1066A000207013208DF80000694604F59A7001955A
:1066B0000AF0F9F9022801D000B1FFDF0020D4E789
:1066C00070B50D460646FCF70BFD18B10178272979
:1066D0001FD102E043F2020070BD807F00F0030092
:1066E000012806D00021304608F02EFE040003D118
:1066F00001E00121F7E7FFDFA079022809D16078E6
:10670000C00706D02A4621463046FEF7C6FC10B127
:106710000FE0082070BDB4F864000E280BD204F11D
:10672000660102231022081FFEF70CFB01210170F5
:106730004570002070BD112070BD70B5064686B052
:1067400014460D4608460CF0C3F818B920460CF064
:10675000E5F810B1102006B070BDA6F57F40FF38F7
:106760000ED03046FCF7BCFC38B1417822464B08CD
:10677000811C1846FCF73FFE07E043F20200EAE7FF
:106780002046FDF785FC0028E5D11021E01D0BF027
:1067900049FDE21D29466846FEF767FC102204F118
:1067A0001700019917F078FB0020D4E72DE9F0419C
:1067B000044686B015468846002708460CF0D5F8F2
:1067C00018B928460CF0D1F810B1102006B007E433
:1067D0002046FCF785FC060003D03078272818D126
:1067E00002E043F20200F1E7B07F00F0030001286D
:1067F00006D00021204608F0A7FD040003D101E0E7
:106800000121F7E7FFDF2078400702D56078800795
:1068100001D40820DAE7B07F00F00300012818D087
:10682000D4E91E01407800B1B5B1487810B1B8F193
:10683000000F11D0C5B1EA1D6846E168FEF715FCEE
:10684000102205F11700019917F0FAFA30B1042768
:106850000AE0D4E91E10E5E70720B7E71022E91D9A
:1068600004F1310017F018FBB8F1000F06D0102228
:1068700008F1070104F1210017F00EFB2078252113
:1068800040F0020020703046FCF762FC2078C1071F
:1068900016D020F00100207002208DF8000004F1D5
:1068A00021000290103003908DF80470694604F5C1
:1068B0009A700AF0F8F8022804D018B1FFDF01E05E
:1068C00084F82070002081E7F8B515460E4607468B
:1068D000FCF706FC040004D02078222804D008200D
:1068E000F8BD43F20200F8BDA07F00F003000228CB
:1068F00002D043F20400F8BD30460BF0E9FF18B9AE
:1069000028460BF0E5FF08B11020F8BD009532884D
:10691000B31C21463846FEF7E4FB112814D00028AA
:10692000F3D1297C4A08E17F62F30001E1772A7CF8
:1069300062F34101E177297C890884F82010A17F66
:1069400021F08001A177F8BDA17F0907FBD4D6F81B
:106950000200C4F83600D6F80600C4F83A003088C1
:10696000A0861022294604F1240017F095FA287C0D
:106970004108E07F61F38200E077297C61F3C30086
:10698000E077287C800884F82100A07F40F0080090
:10699000A0770020D3E770B596B00D46064613B138
:1069A000072016B070BDFCF79BFB040007D02078D1
:1069B000222802D3A07F400604D40820F1E743F246
:1069C0000200EEE7C5B12D208DF80000ADF80260A1
:1069D0001022294601A817F05FFA287C4108E07FC1
:1069E00061F30000E077297C61F34100E077287CC7
:1069F000800884F8200004E02E208DF80000ADF817
:106A000002600BA9684605F017FDA17F21F0400147
:106A1000A177C6E770B50D46FCF762FB040005D010
:106A200028460BF07BFF20B1102070BD43F202001E
:106A300070BD29462046FEF7CEFA002070BD04E066
:106A400010F8012B0AB100207047491E89B2F7D215
:106A50000120704718B18178012938D101E0102058
:106A60007047018842F60112881A914231D018DC31
:106A700042F60102A1EB020091422AD00CDC41B3A4
:106A8000B1F5C05F25D06FF4C050081821D0A0F533
:106A90007060FF381BD11CE001281AD002280AD1EF
:106AA00017E0B0F5807F14D008DC012811D002284F
:106AB0000FD003280DD0FF2809D10AE0B0F5817F5F
:106AC00007D0A0F58070033803D0012801D0002042
:106AD00070470F2070470B2826D008DC1BD2DFE858
:106AE00000F01C2025251A25292325271E00112802
:106AF0001CD008DC0C2817D00D281DD00F2815D06D
:106B0000102808D110E0822809D0842810D08528C8
:106B100010D0872812D0032070470020704705202E
:106B2000704743F203007047072070470F207047FB
:106B300004207047062070470C20704743F2020083
:106B4000704708280DD2DFE800F00406040C0C089A
:106B50000A0A00207047112070470720704708205C
:106B600070470320704738B50C46050041D0694690
:106B7000FFF7D5F9002819D19DF80010607861F36E
:106B8000020060706946681CFFF7C9F900280DD142
:106B90009DF80010607861F3C5006070A978C1F3BA
:106BA0004101012903D0022905D0072038BD2178F1
:106BB00021F0200102E0217841F0200121704107FD
:106BC00004D0A978C90861F386106070607810F06D
:106BD000380F07D0A978090961F3C710607010F069
:106BE000380F02D16078400603D5207840F040008D
:106BF0002070002038BD70B504460020088015467E
:106C00006068FFF7B0FF002816D12089A18988426B
:106C100011D860688078C0070AD0B1F5007F0AD823
:106C200040F20120B1FBF0F200FB1210288007E0D7
:106C3000B1F5FF7F01D90C2070BD01F2012129803F
:106C4000002070BD10B50478137864F3000313704E
:106C50000478640864F3410313700478A40864F3AF
:106C6000820313700478E40864F3C3031370047898
:106C7000240964F3041313700478640964F345135E
:106C800013700078800960F38613137031B10878AF
:106C9000C10701D1800701D5012000E0002060F389
:106CA000C713137010BD4278530702D002F00703D8
:106CB00006E012F0380F02D0C2F3C20300E0012355
:106CC0004A7863F302024A70407810F0380F02D01D
:106CD000C0F3C20005E0430702D000F0070000E067
:106CE000012060F3C5024A7070472DE9F04F95B05E
:106CF0000D00804615D0B8F1000F16D0122128469D
:106D000017F041F94FF6FF7B05AA0121584605F01F
:106D1000DDF90024264637464FF420596FF4205AF7
:106D200075E0102015B0BDE8F08F0720FAE700BF2E
:106D30009DF81E0001280AD1BDF81C0048450BD063
:106D400010EB0A000AD001280CD002280CD0042C29
:106D50000ED0052C0FD10DE0012400E00224BDF877
:106D60001A6008E0032406E00424BDF81A7002E06B
:106D7000052400E00624BDF81A10414547D12C74C3
:106D8000BEB34FF0000810AA4FF0070ACDE9028207
:106D9000CDE900A80DF13C091023CDF81090424632
:106DA0003146584605F045FA08BBBDF83C002A4676
:106DB000C0B210A909F038FFC8B9AE81CFB1CDE992
:106DC00000A80DF1080C0AAE40468CE841021323DE
:106DD00000223946584605F02CFA40B9BDF83C006F
:106DE000F11CC01EC0B22A1D09F01EFF10B1032005
:106DF00098E70AE0BDF82900E881062C05D19DF846
:106E00001E00A872BDF81C00288100208AE705A892
:106E100005F068F900288BD0FFF75DFE82E72DE9C9
:106E2000F0471C46DDE90978DDF8209015460E0094
:106E3000824600D1FFDF0CB1208818B1D5B11120F6
:106E4000BDE8F087022D01D0012100E0002106F10C
:106E5000140004F013F8A8F8000002463B46294647
:106E6000504605F000FCC9F8000008B9A41C3C60BD
:106E70000020E5E71320E3E7F8B50D460646144683
:106E8000DDE90710069ACAB10346009104222146A3
:106E9000304605F0F7FC5CB1022C08D1A87CC00795
:106EA00005D02146304605F0BDFE0020A874F8BD8F
:106EB00021463046BDE8F84005F0B4BE1880F8BD64
:106EC0002DE9FF4791461A881C468A4680460AB338
:106ED00003AB494605F0C7FB05001BD04046A61C86
:106EE000278808F04EFB3246072629463B46009687
:106EF00007F0D4FF208803990095CDE901102346BF
:106F00004A4651464046FFF7B7FF00202080012047
:106F100004B095E70020FBE72DE9F0478CB00D4663
:106F2000DDE9149882461C4617460226142103A860
:106F300017F04BF8012002218DF810108DF80C008D
:106F40008DF81180ADF8147064B1A178C90709D02B
:106F50008DF81600E088ADF81A00A088ADF818008A
:106F6000A06807900AAA09A908A88DE80700324678
:106F7000294650466B68FFF752FF00280ED1DDE925
:106F8000080105F114028DE807000AAB4A4603A97F
:106F9000504604F037FB18B1FFF7D3FD0CB04FE7B4
:106FA000DDE90801BDF828208DE8070032462946B2
:106FB00050466B68FFF760FF0020EFE7F0B58BB03D
:106FC00000240646069407940727089405A8099408
:106FD000019400970294CDE903400D461023224608
:106FE000304605F026F978B90AA806A90194009759
:106FF0000294CDE90310BDF8143000222946304632
:1070000004F0EEFE002801D0FFF765FD0BB0F0BDE7
:1070100004F080BD2DE9FC410C468046002602F0BC
:10702000D2F9054620780D287ED2DFE800F0B207BD
:107030000BA918B33C5C6C8FA5949A00404602F0F3
:10704000F1F9A7E00421404608F07EF9070000D1DD
:10705000FFDF07F11401404603F0A4FE6AE00421BB
:10706000404608F071F9070000D1FFDFE088ADF875
:1070700000000020B8819DF80000010704D5C0067B
:1070800002D5A088B88105E09DF80100400609D529
:10709000A088F88105B9FFDF22462946404601F065
:1070A00017FD022676E0A088694605F0A5F900B133
:1070B000FFDF9DF8020001280BD1BDF8000042F669
:1070C000011188420BD0A0F52451023907D0491E86
:1070D00005D0E079000600D5022635BB01E0042684
:1070E00058E0FFDF27E0E079000609D5042140469B
:1070F00008F02AF9060000D1FFDFA088F0810226FF
:107100009DB9FFDF17E00421404608F01DF9070094
:1071100000D1FFDF07F1140004F033FD90F0010F00
:1071200005D1E079000601E033E004E032D5022623
:10713000A7F810802DB122462946404601F0C8FC30
:1071400028E013214046FDF733FB23E00226002D03
:10715000F1D1FFDFEFE702260121404602F0AEF950
:1071600018E0606800902089ADF8040001226946AB
:10717000404602F0C4F90DE0002DDCD1FFDFDAE774
:10718000022600214046FBF732F9002DD3D1FFDF64
:10719000D1E7FFDF3046BDE8FC813EB50C0009D0E9
:1071A00001466B4601AA002005F0C5F820B1FFF7A3
:1071B00092FC3EBD10203EBD00202080A0709DF8B6
:1071C000050002A900F00700FEF7C5FE50B99DF8C2
:1071D000080020709DF8050002A9C0F3C200FEF768
:1071E000BAFE08B103203EBD9DF8080060709DF80E
:1071F0000500C109A07861F30410A0709DF8051086
:10720000890961F3C300A0709DF80410890601D5B7
:10721000022100E0012161F342009DF8001061F3BA
:107220000000A07000203EBD70B5144606460D4615
:1072300051EA040005D075B108460BF08DFB78B912
:1072400001E0072070BD2946304605F0D5F810B1A1
:10725000BDE870403FE454B120460BF07DFB08B11F
:10726000102070BD21463046BDE8704095E70020F3
:1072700070BD2DE9FE4F0C4690460546002701786B
:107280000822007A3E46B2EB111F7DD104F10A01BB
:107290000091891E02910C31821E4FF0020B4FF0BB
:1072A000010A0191092A70D2DFE802F0F5F4056FB6
:1072B000252579B8F6006888042108F045F806000D
:1072C00000D1FFDFB08910B152270726EBE051272C
:1072D0001026002C7ED06888A08084F806A0A8899B
:1072E00000220099FFF7A0FF002874D1A88920810F
:1072F000288AE081FDE0B5F81290072825D1E87BC7
:10730000000622D5512709F1140086B2002CE1D0E5
:10731000A88900220099FFF787FF00287CD16888A0
:10732000A08084F806B0A889208184F80EA0288A5D
:107330002082A4F81290A88A009068884B46A96918
:10734000DDF8042001F0A1FBD3E0502709F1120081
:1073500086B2002C3ED0A88900220299FFF764FF74
:10736000002859D16888A080A889E080287A072859
:1073700013D002202073288AE081E87BC009607363
:10738000A4F81090A88A01E0B0E0ADE00090688811
:107390004B4604F11202A969D4E70120EAE76888A4
:1073A000042107F0D1FFB5F812A05FEA000900D16F
:1073B000FFDF09F1140004F0E4FB90F0010F02D1AB
:1073C000E87B000627D50AF11400512786B2002C6D
:1073D0007FD001E072E01FE06888A080A8890022C9
:1073E0000099FFF721FF002816D184F806B0A8897C
:1073F00020810420A073288A2082A4F812A0A88AE1
:10740000009068885346A969019A01F03EFBA9895A
:10741000A9F80E106DE00320BDE8FE8F6888FBF729
:107420005FFE82466888042107F08EFF8146BAF12C
:10743000000F00D1FFDFB9F1000F00D1FFDFB9F875
:107440001010A1F57F40FF3802D05127142601E02B
:107450005027122694B36888A080502F06D084F855
:1074600006B0287B029901F020FB42E0287BA11D99
:1074700001F01BFB00219AF82300CDE900010B4627
:10748000B9F80E2068884946FFF746FD0028C3D1A9
:107490002FE001E013E01FE0FB49A889C988814281
:1074A00005D1542706264CB16888A08021E05327D7
:1074B0000CE06888A080A889E0801AE009E068886C
:1074C000042107F041FF00B9FFDF55270826002CF3
:1074D000EFD1A8F8006011E056270726002CF8D05D
:1074E0006888A080002012E0FFDF02E0012807D0BA
:1074F000FFDFA8F800600CB12780668000208BE7D2
:1075000057270726002CE4D06888A080687AA071ED
:10751000EFE7401D20F00300042202EB400201FBD4
:1075200000207047D84B00221A7008B1D74A10606B
:1075300007F0B2B870B50C46064686B015465C2119
:10754000204616F042FD05B9FFDFA878E074AA785E
:107550002988204601F0D2FA0020A081E0814FF670
:10756000FF7020822A8804F11401304603F0FFFBEB
:107570006A460121304604F0A9FD19E09DF8030098
:10758000000715D5BDF806103046FFF717FD9DF82A
:107590000300BDF8061040F010008DF80300BDF8A0
:1075A0000300ADF81400FF233046059A04F0EFFE07
:1075B000684604F097FD0028E0D006B070BD70B5B5
:1075C000064601F114000C46054603F007FC01468F
:1075D000E27C204601F0BEFA29463046BDE8704004
:1075E00003F0E7BB70B50546042107F0ADFE0400CB
:1075F00000D1FFDF04F114012846BDE8704003F01C
:10760000D1BB2DE9F0418CB00C4680460226FBF739
:1076100067FD050014D02878222829D30CB1A08852
:1076200098B101208DF8180003208DF81C0000206F
:107630008DF81D005CB1A088ADF82400206808E03A
:1076400043F202000CB0BDE8F0810920FAE7ADF882
:10765000240008900421404607F076FE040000D183
:10766000FFDF04F11400074603F0CFFBC00601D48E
:107670000820E7E705AA04A903A88DE80700324619
:10768000214640466368FFF7CAFB00B1FFDFDDE932
:1076900003018DE8830095F8232005AB06A9404639
:1076A00003F0B0FF10B1FFF74CFACBE7BDF81420A0
:1076B000DDE903018DE80700324621464046636854
:1076C000FFF7DAFB4FF6FF7020820020BAE72DE9C2
:1076D000F047B2F80290824688B015468846484680
:1076E000FBF7FEFC06460421484607F02DFE044643
:1076F0000020059002270690ADF81C0006B9FFDFB8
:1077000004B9FFDF3946484605F0A2FA60B907AA76
:1077100006A905A88DE807003A4621464846636851
:10772000FFF77DFB00B1FFDFDDE9051204F1140076
:10773000CDF80080CDE9032007ABCDE9013196F803
:107740002320514648466B6803F0A8FB06000AD088
:10775000022E04D0032E16D0042E00D0FFDF08B076
:107760003046BDE8F087BDF81C000028F7D0DDE901
:1077700005120091CDE901203A462146484663684A
:10778000FFF77AFBEBE7687840F008006870E6E7FF
:107790002DE9F04F9BB004464FF000083A48ADF891
:1077A0005480ADF83080ADF85080A0F80480ADF87A
:1077B0001480ADF81880ADF82080ADF81C800078FA
:1077C00016460D464746012809D0022807D003284F
:1077D00005D0042803D008201BB0BDE8F08F204658
:1077E0000BF076F8D0BB28460BF072F8B0BB60689F
:1077F0000BF0BBF890BB606848B160892189884272
:1078000002D8B1F5007F01D90C20E5E780460BAA2C
:1078100006A92846FFF7EFF90028DDD168688078CF
:10782000C0F34100022808D19DF8190010F0380F6C
:1078300003D028690BF090F880B905A92069FFF7FB
:1078400092F90028C8D1206950B1607880079DF86E
:10785000150000F0380002D5F0B301E011E0D8BB0C
:107860009DF81400800613D59DF8150010F0380F10
:1078700003D060680BF070F818B960680BF075F809
:1078800030B11020A8E70000F8020020140000200A
:1078900007A96069FFF767F900289DD1606940B1C9
:1078A0009DF81D0000F0070101293BD110F0380FB1
:1078B00038D008A9A069FFF756F900288CD19DF8A7
:1078C0001C0080062ED49DF8200080062AD4A069D2
:1078D00050B19DF8210000E024E000F007010129EB
:1078E00020D110F0380F1DD0E06818B10078C8B171
:1078F0001C2817D20EAA611C2046FFF7A3F901200D
:10790000B94660F30F27BA4607468DF84E0042F697
:107910000300ADF84C000DF13B0217A9286809F0EF
:10792000A2F908B1072057E79DF85C0016A9CDF829
:107930000090C01CCDE9019100F0FF0B00230BF279
:107940000122514613A804F005FBE8BBBDF858001E
:107950000990FE482A8929690092CDE901106B89B6
:10796000BDF82C202868069904F0F4FA01007DD1B6
:1079700020784FF0020AC10601D480062BD5ADF85D
:107980000C90606950B907A906A8FFF78CF99DF81B
:107990001D0020F00700401C8DF81D009DF81C0004
:1079A0008DF84E7040F0C8008DF81C0042F60210B1
:1079B000ADF84C000CA903AACDF800A0CDE9012137
:1079C000002340F2032200E01FE013A8079904F00F
:1079D000C1FA01004AD1DD484D46001F5B46808850
:1079E000ADF839000EA8CDE90290CDF80490CDF89D
:1079F00010904FF007090022CDF80090BDF8581004
:107A00004FF6FF7004F0ECF910B1FFF764F8E3E60D
:107A10009DF83800000625D52946012060F30F2186
:107A20008DF84E704FF42450ADF84C00ADF8105066
:107A300062789DF81000002362F300008DF81000BA
:107A40006278CDF800A0520862F341008DF8100072
:107A500004AACDE9012540F2032213A804F07AFA22
:107A6000010003D1606888B3206900E087E098B91D
:107A700005A906A8FFF717F96078800706D49DF8D6
:107A8000150020F038008DF8150005E09DF8140071
:107A900040F040008DF814008DF84E7042F6011051
:107AA000ADF84C00208940F20121B0FBF1F201FB5E
:107AB0001202606814ABCDF80080CDE90103002309
:107AC00013A8059904F046FA010058D12078C007A0
:107AD00029D0ADF80C50A06950B908A906A8FFF745
:107AE000E2F89DF8210020F00700401C8DF82100ED
:107AF0009DF820008DF84E7040F040008DF8200079
:107B000042F60310ADF84C0015A903AACDF800A069
:107B1000CDE90121002340F2032213A8089904F0C3
:107B200019FA01002BD1E06868B32946012060F3FF
:107B30000F218DF84E7042F60410ADF84C00E0684D
:107B4000002302788DF8602040788DF86100E068AD
:107B500018AA4088ADF86200E06800798DF86400EA
:107B6000E068C088ADF86500CDF80090CDE901254A
:107B70004FF4027213A804F0EDF9010003D0099844
:107B800001F011F828E671480321001F017056B179
:107B900080883080BDF850007080BDF83000B08023
:107BA000BDF85400F080002016E670B501258AB0BB
:107BB00016460B46012802D0022816D104E08DF8A3
:107BC0000E504FF4205003E08DF80E5042F60100A5
:107BD000ADF80C0063B10024601C60F30F2404AA0C
:107BE00008A9184609F03FF820B107200AB070BD77
:107BF0001020FBE704A99DF820205448CDE900217E
:107C0000801E02900023214603A802F2012204F004
:107C1000A1F910B1FEF75FFFE8E74C48001F0EB175
:107C20004188318005700020E0E7F0B593B0074649
:107C300001268DF83E6041F60100ADF83C0012AA25
:107C40000FA93046FFF7B1FF002848D13F4C00256F
:107C5000241FE7B31C2102A816F0B7F99DF808000D
:107C60008DF83E6040F020008DF8080042F60520B7
:107C7000ADF83C000E959DF83A00119520F00600F5
:107C8000801C8DF83A009DF838006A4620F0FF000D
:107C90008DF838009DF8390009A920F0FF008DF813
:107CA00039000420ADF82C00ADF830000EA80A9081
:107CB00011A80D900FA80990ADF82E5002A8FFF75B
:107CC00067FD00280BD1BDF80000E08000E008E06F
:107CD000BDF804002081401C60812570002013B095
:107CE000F0BDE5802581BDF84800F4E72DE9F74FA8
:107CF0001649A0B00024091F17940A78A146012A4A
:107D000004D0022A02D0082023B066E54A888242C5
:107D100001D00620F8E721988A46824201D1072047
:107D2000F2E701202146ADF848004FF6FF788DF8C4
:107D30006E0042F6020B60F30F21ADF84A80ADF8F9
:107D40006CB006918DF8724002E00000FC02002049
:107D50001CA9ADF870401391ADF8508012A804F042
:107D6000E5F900252E462F460DAB072212A9404605
:107D700004F0DFF978B182285DD195B38EB3ADF808
:107D80006450ADF866609DF85E008DF8144019AC43
:107D9000012864D06BE09DF83A001FB3012859D147
:107DA000BDF8381059451FD118A809A901940294AB
:107DB000CDE9031007200090BDF8361010230022F3
:107DC000404604F036FAB0BBBDF86000042801D08C
:107DD00006284AD1BDF82410219881423AD10F20BB
:107DE00092E73AE0012835D1BDF83800B0F5205FC0
:107DF00003D042F6010188422CD1BAF80200BDF846
:107E00003610884201D1012700E0002705B19EB15C
:107E1000219881421ED118A809AA01940294CDE9A3
:107E20000320072000900D4610230022404604F056
:107E300000FA00B902E02DE04E460BE0BDF860000C
:107E4000022801D0102810D1C0B217AA09A908F041
:107E5000EBFE50B9BDF8369086E7052054E705A93A
:107E600017A8221D08F0FFFE08B103204CE79DF87B
:107E700014000023001DC2B28DF814202298009235
:107E8000CDE901401BA8069904F064F810B902225C
:107E90008AF80020FEF71FFE36E710B50B46401E9D
:107EA00088B084B205AA00211846FEF7CBFE002058
:107EB0000DF1080C06AA05A901908CE8070007201F
:107EC00000900123002221464FF6FF7003F088FF47
:107ED0000446BDF81800012800D0FFDF2046FEF759
:107EE000FAFD08B010BDF0B5FF4F044687B03878F2
:107EF0000E46032804D0042802D0082007B0F0BDA5
:107F000004AA03A92046FEF776FE0500F6D16068B4
:107F10008078C0F3410002280AD19DF80D0010F0CE
:107F2000380F05D020690AF017FD08B11020E5E7E9
:107F3000208905AA21698DE807006389BDF8102012
:107F40002068039904F006F810B1FEF7C4FDD5E7E8
:107F500016B1BDF814003080042038702846CDE7F3
:107F6000F8B50C0006460CD001464FF6FF7500230D
:107F70006A46284604F0DFF928B100BFFEF7ABFDE2
:107F8000F8BD1020F8BD69462046FEF7ECFD00283C
:107F9000F8D1A078314600F001032846009A04F099
:107FA000F6F9EBE730B587B0144600220DF1080C66
:107FB00005AD01928CE82C00072200920A4601468A
:107FC00023884FF6FF7003F00BFFBDF814102180DB
:107FD000FEF781FD07B030BD70B50D46042107F0F6
:107FE000B3F9040000D1FFDF294604F11400BDE815
:107FF000704002F003BF70B50D46042107F0A4F9EC
:10800000040000D1FFDF294604F11400BDE87040F0
:1080100002F017BF70B50D46042107F095F9040072
:1080200000D1FFDF294604F11400BDE8704002F0E2
:108030002FBF70B50546042107F086F9040000D172
:10804000FFDF214628462368BDE870400122FEF785
:1080500037BF2DE9F0478246042107F075F9040087
:1080600000D1FFDF04F1140002F0B8FE401D20F043
:10807000030626E0011D00880022431821465046D1
:10808000FEF71EFF002820D0E07CA56870431FFA91
:1080900080F82888B7B2814610FA86F080B228802E
:1080A000404502D3A0EB080028806888B84200D27F
:1080B000FFDF09EB0701414500D9FFDF6888C01BDE
:1080C0006880A06841880029D4D1BDE8F08770B5E8
:1080D0000546042107F038F9040000D1FFDF2146EE
:1080E00028466368BDE870400222FEF7E9BE70B51D
:1080F0000E46054601F067F9040000D1FFDF0120BC
:10810000207266726580207820F00F00001D20F03C
:10811000F00040302070BDE8704001F057B910B554
:108120000446012900D0FFDF2046BDE810400121B0
:10813000FAF75DB92DE9F34F9BB04FF0000B0C003F
:10814000ADF81CB05E461BD0E06830B1A068B8B195
:108150000188ADF81C10A0F800B01B98FAF7C0FF1A
:108160005FEA000943F2020769D099F8000022286B
:1081700063D304211B9807F0E7F8050005D103E05D
:1081800010201DB0BDE8F08FFFDF05F11400109046
:1081900002F024FE401D20F00308A078012803D03F
:1081A000022801D00720ECE7208878B1401C81B27A
:1081B0000BAA1B9803F08AFF0BA803F093FF9DF80E
:1081C00036204FF45051012A0DD102E043F2030052
:1081D000D7E7BDF83420A2F52453023B03D182280F
:1081E00001D0A0B901E00846CBE7E068B0B1CDE925
:1081F00002B0072007AA0090CDF804B00492A2882C
:108200002188BDF81C301B9803F0EAFD10B1FEF781
:1082100062FCB6E7A168BDF81C0008809DF82F003D
:10822000C00602D543F20140ABE70F9838B1A17800
:108230000078012905D080072AD40820A1E7384614
:108240009FE7C007F9D00020039002208DF84C0072
:10825000A868EA7C418802FB08F28A421ED9031D05
:108260000A93008896B247181FFA88FAB74200D3DB
:10827000BF1B01EB0A00B04200D9FFDF07EB0A0089
:10828000B04200D9FFDF0A98C619A6F800B005E091
:108290000120039003208DF84C002E689DF83000DB
:1082A00010F0380F00D1FFDF9DF830000F49C0F308
:1082B000C200084410F8011C99F82300814201D93A
:1082C0000F205EE72088ADF8500008AA06A905A88F
:1082D0008DE8070033462946039A1B98FEF79FFD59
:1082E000002896D104E00000F8020020FA2F0000D8
:1082F000DDE90501109A8DE8070008AB072213A9F4
:108300001B9803F07FF910B1FEF71BFC39E7BDF8AD
:108310002020DDE905018DE8070033462946039A50
:108320001B98FEF7A9FD0598D0B9A078012817D1B0
:10833000E87CAC6800FB08F086B2218860881FFAF0
:1083400088F70D18B54200D3AD1B3844B04200D9B0
:10835000FFDFE819B04200D9FFDF60883844608051
:1083600000200EE770B5064615460C460846FEF797
:1083700071FB002805D12A4621463046BDE87040F1
:1083800013E470BDB2E470B51E4614460D0009D06A
:1083900044B1616831B138B1FE494988814203D0A6
:1083A000072070BD102070BD2068FEF753FB002829
:1083B000F9D1324621462846BDE87040FFF7E8B9BA
:1083C00070B515460C0006D038B1F2498988814253
:1083D00003D0072070BD102070BD2068FEF73AFB67
:1083E0000028F9D129462046BDE870407BE570B5EC
:1083F000064686B00D46144610460AF08FFAD0BBEA
:1084000060680AF0B2FAB0BBA6F57F40FF3803D02F
:108410003046FAF765FE80B128466946FEF765FCEE
:1084200000280CD19DF810100F2008293CD2DFE85D
:1084300001F008060606060A0A0843F2020006B022
:1084400070BD0320FBE79DF80210012908D1BDF89B
:108450000010B1F5C05FF2D06FF4C052D142EED03F
:108460009DF8061001290DD1BDF80410A1F5285181
:10847000062907D200E028E0DFE801F00303040347
:108480000303DCE79DF80A1001290ED1BDF808109E
:10849000B1F5245FD3D0A1F524510239CFD0012901
:1084A000CDD0022901D1CAE7FFDF606878B9002387
:1084B00005AA2946304603F03EFF10B1FEF70BFB3C
:1084C000BDE79DF81400800601D41020B7E761884D
:1084D000224628466368FFF765FDB0E72DE9F043C3
:1084E000814687B08846144610460AF017FA18B13C
:1084F000102007B0BDE8F083002306AA4146484695
:1085000003F019FF18B100BFFEF7E5FAF1E79DF897
:108510001800C00602D543F20140EAE7002507270C
:1085200005A8019500970295CDE9035062884FF6A2
:10853000FF734146484603F07CFE060013D1606895
:108540000AF0ECF960B960680195CDE90250009736
:108550000495238862884146484603F06AFE064631
:10856000BDF8140020803046CEE739B1894B0A8827
:108570001B899A4202D843F203007047DAE510B52E
:1085800086B0844C0423ADF81430E38843B12489C9
:108590008C4201D2914205D943F2030006B010BDCE
:1085A0000620FBE7ADF81010002100910191ADF815
:1085B000003002218DF8021005A9029104A903914F
:1085C000ADF812206946FFF7B5FDE7E72DE9FC4756
:1085D00081460F4608460AF07BF988BB4846FAF701
:1085E0007FFD5FEA00080AD098F80000222829D30E
:1085F0000421484606F0A8FE060005D103E043F238
:108600000200BDE8FC87FFDF06F1140002F0FDFB6D
:1086100005463878012803D0022804D00720F0E767
:10862000A8070FD502E015F0340F0BD0B8793C1D28
:10863000C00709D0E08838B1A0680AF049F918B13C
:108640001020DEE70820DCE73A782088002128B3F4
:10865000A0F201130721112B18D20CD2DFE803F08E
:108660000B090D0B1D0B121D100B0B1D1D1D1D0BE2
:108670001D00022A11D10846C3E7012AFBD00CE0F5
:10868000EA0600E0AA06002AF5DA06E0A0F5C072C4
:108690001F2A02D97D3A022AEDD8C1B298F82300E8
:1086A000CDE90001F289234631464846FEF734FC05
:1086B000A7E72DE9F04F8BB01F4615460C468346C1
:1086C0000026FAF70DFD28B10078222805D20820EF
:1086D0000BB057E543F20200FAE7B80801D00720D3
:1086E000F6E7032F00D100274FF6FF79CCB1022D1A
:1086F00071D320460AF039F930B904EB0508A8F126
:1087000001000AF032F908B11020E1E7AD1EAAB26B
:108710002146484603F009FF38F8021C88425AD126
:10872000ADB21C49B80702D50889401C00E0012001
:108730001FFA80F8F80701D00F8900E04F4605AA1C
:108740004146584603F0C2FC4FF0070A4FF00009BB
:10875000FCB1204608E0408810283CD8361D304443
:1087600086B2AE4237D2A01902884245F3D352E016
:108770009DF8170002074ED57CB304EB0608361DA2
:10878000B8F80230B6B2102B25D89A19AA4222D8CE
:1087900002E040E0F8020020B8F8002091421AD12F
:1087A000C0061BD5CDE900A90DF1080C0AAAA11934
:1087B00048468CE80700B8F800100022584603F03D
:1087C0000FFB10B1FEF787F982E7B8F80200BDF899
:1087D0002810884202D00B207AE704E0B8F80200A3
:1087E000304486B206E0C00604D55846FEF7E6FBE4
:1087F00000288AD19DF81700BDF81A1020F010004B
:108800008DF81700BDF81700ADF80000FF2358469B
:10881000009A03F0BCFD05A803F064FC18B9BDF88C
:108820001A10B942A4D90421584606F08DFD04005F
:1088300000D1FFDFA2895AB1CDE900A94D4600233E
:1088400021465846FEF768FB0028BDD1A5813FE7C9
:1088500000203DE72DE9FF4F8BB01E4617000D4667
:108860004FF0000412D0B00802D007200FB089E406
:10887000032E00D100265DB108460AF06DF828B934
:108880003888691E08440AF067F808B11020EDE73F
:10889000CA4AB00701D5518900E00121F0074FF61F
:1088A000FF7802D05089401E00E0404686B206AAFA
:1088B0000B9803F00BFC4FF000094FF0070B0DF184
:1088C000140A38E09DF81B00000734D5CDF8049059
:1088D000CDF800B0CDF80890CDE9039A43460022C8
:1088E0000B9803F0A6FC60BB05B3BDF814103A88E2
:1088F00021442819091D8A4230D3BDF81E2020F8D2
:10890000022BBDF8142020F8022BCDE900B9CDE9E7
:108910000290CDF810A0BDF81E10BDF81430002252
:108920000B9803F086FC08B103209FE7BDF8140004
:108930002044001D84B206A803F0D4FB20B1822895
:1089400006D0FEF7C8F891E7BDF81E10B142B9D9BC
:1089500034B17DB13888A11C884203D20C2085E750
:10896000052083E722462946404603F0DEFD014606
:1089700028190180A41C3C80002077E710B504462C
:1089800009F0CCFF08B1102010BD8C484089208030
:10899000002010BD2DE9F0438DB00D4681464FF00B
:1089A0000208142106A815F010FB01268DF81C60A2
:1089B00000208DF81D008DF81860ADF82050484655
:1089C000FAF78EFB48B10078222812D304214846DA
:1089D00006F0BAFC040005D103E043F202000DB03A
:1089E00088E5FFDF04F11400074602F00EFA4006A6
:1089F00001D40820F3E705AA04A903A88DE807001D
:108A00004246214648466368FEF709FA00B1FFDF97
:108A1000DDE903018DE8830005AB072206A948467E
:108A200002F0F0FD10B1FEF78CF8D8E7A674BDF89F
:108A30001420DDE903018DE807004246214648463F
:108A40006368FEF719FA29464846F9F7C1FC0BA9F5
:108A5000384602F0C9F900B1FFDFBDF82C40172CF1
:108A600001D2172000E02046A84201D92C4602E09E
:108A7000172C00D2172421464846FFF7BCFA21469E
:108A80004846F9F7D9F90020A9E7F8B51C4615467C
:108A90000E46069F06F063FD2346FF1DBCB231461D
:108AA0002A46009406F0C1F9F8BD70B50C4605469B
:108AB0000E21204615F067FA002020802DB1012DEF
:108AC00001D0FFDF70BD062000E00520A07170BD61
:108AD00010B548800878144620F00F00001D20F0E3
:108AE000F00080300B4608701422214603F1080084
:108AF00015F017FABDE8104000F068BC2DE9F0470A
:108B00002F4F491D064621F0030191460C46386857
:108B100005F0D9FD050000D1FFDF4FF000083560FA
:108B2000A5F800802146386805F0CDFD050000D18C
:108B3000FFDF7560A5F8008004FB09F1091D3868A6
:108B400005F0C1FD040000D1FFDFB460C4F800806F
:108B5000BDE8F0872DE9F041491D21F00304184DCF
:108B60001746064601682246286805F0D5FD2246CC
:108B70007168286805F0D0FD7C43221DB168286823
:108B800005F0CAFD042006F089FB0446042006F027
:108B90008DFB201A012804D12868BDE8F04105F0BA
:108BA00083BDBDE8F08110B50C4603F05CFA00B15E
:108BB000FFDF2046BDE81040FDF78DBFF802002022
:108BC00014000020F0B597B0054652208DF8000043
:108BD000281DADF80200ADF804101E4617460BA97B
:108BE000684603F029FC00B1FFDFBDF83040032CDC
:108BF00001D2204600E00320C1B2284600F07EFFEB
:108C00003870022C00D30224E1B2284600F076FF2F
:108C1000401C307017B0F0BD2DE9F04F0C00FC493E
:108C200099B08246D1E90201FA4ECDE90C010AF170
:108C30000300717A327A1144CDB220F00301009121
:108C4000377E07F1010704D1F8B207F093FF00B1B6
:108C5000FFDF00982A4600EB0710C01C20F003013C
:108C6000F7694FF00009009134B981F80090B8B26B
:108C700003F081F800B1FFDF0098234638440090EC
:108C8000B07A317A2A460844C1B2684600F0FEFE46
:108C90000098C01C20F003000090737A327AB17AF9
:108CA00004B1002006F042FA0099084400902146E1
:108CB000684600F02EFF00273D46B34696F8018037
:108CC0000CE0284600F0C5FE064681788088F9F75A
:108CD0004DF971786D1C00FB0177EDB24545F0D17F
:108CE0000098C01C20F00300009004B10020394619
:108CF000F9F743F900990027084400903D469BF896
:108D000001800CE0284600F0A4FE0646C178808869
:108D1000FEF7FFFB71786D1C00FB0177EDB2454556
:108D2000F0D10098C01C20F00300009004B1002096
:108D30003946FEF7F7FB00990844C01D20F00700F4
:108D40000090ECBBB54AB4491160111D401E08608B
:108D500001222C21B24806F07AF9FAF720F9B1483D
:108D60004178806804F00CF9AE4801240C30017899
:108D7000012915D13E218DF80410C0788DF8060028
:108D800010B1012803D004E08DF8064001E08DF811
:108D9000069001A805F0A5FB10B10EA804F0AFF9EC
:108DA00000211E22084601F0F7F9FBF715F903F040
:108DB00018FD98480CAA00210C30F8F7CBFA00E017
:108DC0001DE000B1FFDF9BF81900FEF72EFF00B198
:108DD000FFDF90484FF4B871443015F0F6F88D4835
:108DE0000221443080F8694180F86A1180F86B11E3
:108DF00080F86C91062180F86D11052101710099B0
:108E000019B0A1EB0A00BDE8F08F70B5814D0646A0
:108E10004435287805EB4014E8780834A0B9A8193F
:108E200090F86801002810D0A8780B2800D3FFDF45
:108E3000207820F0FF002070607866F3020020F0B8
:108E4000080060700120E870204670BD2DE9F041F7
:108E500005460C4600270078052190463E46B1EBBA
:108E6000101F00D0FFDF287A50B101280ED0FFDF9D
:108E7000A8F800600CB1278066800020BDE8F08172
:108E80000127092674B16888A08008E0022714260B
:108E900044B16888A0802869E060A88A2082287B85
:108EA0002072E5E7A8F80060E7E710B55D4C606860
:108EB000C11D21F00701814200D0FFDF554801218B
:108EC00000220170427001720323437281720273A7
:108ED000052282821F22C282417353A202610A22AA
:108EE000027641764FF4B061C1616168416010BDA6
:108EF00030B54C4C1568636808339D4202D204209B
:108F0000136030BD434B5D785A6802EBC5021070A8
:108F100051700320D080172090800120D070907075
:108F20005878401C5870606808306060002030BD80
:108F300070B5064637480024457807E0204600F023
:108F400088FD0178B14204D0641CE4B2AC42F5D192
:108F5000002070BDF7B5064608780C4650B1FFF703
:108F6000E7FF0546202E07D0232E17D0212E18D03C
:108F7000222E16D00720FEBD00F076FD0DB16978D7
:108F800000E00021401A81B2A0780144FF29F1D805
:108F90000028EFD0A088022803D2EBE760881728CA
:108FA000E8D365B9207802AA0121FFF7A1FF0028C4
:108FB000E1D12078FFF7BCFF050000D1FFDF202EB4
:108FC00008D0212E0ED0222E0FD0232E07D0FFDF67
:108FD0000020FEBDA0786870A088E880F8E760886F
:108FE000A880F5E7A078A870F2E7A078E870EFE72E
:108FF00000B597B04F218DF8001000780BA900F054
:1090000001008DF80200684603F016FA17B000BDA3
:1090100090E3010010040020000000200006024040
:10902000C40500201C0000206E5246357800000068
:1090300000B5017897B001F001018DF80210417878
:1090400001F001018DF803100178C1F340018DF8A2
:1090500004104178C1F340018DF8051001788908AA
:109060008DF80610417889088DF8071081788DF801
:109070000810C1788DF8091000798DF80A00492090
:109080008DF800000BA9684603F0D6F9BEE700B5DD
:1090900097B051218DF80010ADF802000BA9684679
:1090A00003F0CAF900B1FFDF9DF8300000F00100C5
:1090B000ACE72DE9F84FDFF8F483FD4C00271BE007
:1090C000022000F066FD0120FFF79FFE0546F948EB
:1090D00005F0E6FF686000B9FFDF686803F0F9F9A2
:1090E000A0B12846FAF76BFA284600F058FD18B9E7
:1090F000F048696805F0DDFF94F869010028DFD1C8
:10910000022006F0CBF8064600259AE0E948696897
:1091100005F0CFFFF4E7B8F802104046491C89B2C9
:10912000A8F80210B14201D3002141800221B8F811
:10913000020006F009F900285DD0B8F80200FFF738
:10914000A6FF78B1B8F8020006F01BFA5FEA000942
:1091500000D1FFDF484605F0CEFC18B1B8F8020098
:1091600003F04FFDB8F8020006F0F9F95FEA0009D4
:1091700000D1FFDF484605F0B7FCE0BB0321B8F89B
:10918000020006F0E1F85FEA000B47D1FFDF45E09F
:10919000DBF8040010B10078FF2848D0042000F06C
:1091A000F8FC0320FFF731FE8246484605F0CEFD6D
:1091B000CAF8040000B9FFDFDAF8040005F0A8FEE1
:1091C000002100900170B8F802105046AAF8021071
:1091D00003F094FB484605F09DFE00B9FFDF5046C2
:1091E00000F0DDFC18B99AF80100000704D50099D9
:1091F000CBF8041012E022E0DBF8040038B101786B
:10920000491C11F0FF01017008D1FFDF06E00022C8
:109210001146484600F01BFC00B9FFDF94F86B01D3
:1092200028B1B8F8020003F044FB0028B0D194F84C
:10923000690120B1484605F0E3FE00B101276D1C2D
:10924000EDB2B54204D294F86B0100287FF463AF0D
:10925000002F7FF433AFBDE8F84F052000F099BC34
:1092600010B5924CA0600868E060AFF2B91000F051
:1092700006FF607010BD8E480021443801708B4895
:1092800001708D494160704730B505464FF0805000
:109290000C46D0F8A41097B0491C05D1D0F8A810FE
:1092A000C9430904090C08D050F8A01F01F00101BE
:1092B00029704168216080680EE02B208DF8000045
:1092C0000BA9684603F0B8F800B1FFDF0120287051
:1092D0000C982060BDF83400A0802878002803D0C6
:1092E000607940F0C000607117B030BDF0B54FF04C
:1092F00080540746D4F8800097B00D462B26401CBA
:109300000BD1D4F88400401C07D1D4F88800401C4D
:1093100003D1D4F88C00401C0BD0D4F88000386006
:10932000D4F884007860D4F88800B860D4F88C0051
:1093300016E08DF82C6069460BA803F07DF800B1AB
:10934000FFDF01983860029878608DF82C606946DC
:109350000BA803F071F800B1FFDF0198B860029824
:10936000F860D4F89000401C0BD1D4F89400401C55
:1093700007D1D4F89800401C03D1D4F89C00401CBD
:1093800008D054F8900F286060686860A068A860F2
:10939000E06816E08DF800600BA9684603F04CF811
:1093A00000B1FFDF0C9828600D9868608DF80060B0
:1093B0000BA9684603F040F800B1FFDF0C98A860E5
:1093C0000D98E86026E43A4800791EE570B5384CFF
:1093D000E07828B3207804EB4010407A00F00700D2
:1093E000204490F8680100B9FFDF2078002504EBE5
:1093F0004010407A00F00700011991F86801401E02
:1094000081F868012078401CC0B220700B2800D180
:109410002570A078401CA07008F0F3FDE57070BDC9
:10942000FFDF70BD3EB50546032105F08DFF044604
:10943000284606F094F8054604B9FFDF606818B1C5
:109440000078FF2800D1FFDF01AA6946284600F016
:10945000FEFA60B9FFDF0AE0002202A9284600F008
:10946000F6FA00B9FFDF9DF8080000B1FFDF9DF8B4
:109470000000411E8DF80010EED26068019988420C
:1094800001D1002060600A4C94F86B01022800D3DF
:10949000FFDF94F86B0118B90448407800F00EFE25
:1094A00094F86B01401C84F86B013EBD1C00002049
:1094B00054040020C40500206812002070B5054641
:1094C000A0F57F400C46FF3800D1FFDF012C01D012
:1094D000FFDF70BDFFF777FF040000D1FFDF2078CA
:1094E00020F00F00401D20F0F0005030207065800B
:1094F0000020207201202073BDE8704066E770B53F
:1095000015460C460646FFF75EFF90B1017821F044
:109510000F01491D21F0F0015031017046800121F9
:10952000017221680161A18881820573BDE87040E4
:109530004CE73046BDE870401321FBF739B930B530
:1095400099B0FFF7F5FC040000D1FFDFA588E188A2
:109550000CAB0BAA2846FFF735FB4E208DF8000018
:109560009DF82C008DF802002D1D9DF83000ADF8FF
:1095700004508DF80300ADF80650E088ADF80800FF
:109580000DA9684602F058FF002800D0FFDF19B08F
:1095900030BD2DE9F84FF94E05464FF0000A3078FE
:1095A00010B10820BDE8F88F284609F0B7F908B1D6
:1095B0001020F7E7F24C207808B9FFF776FC617AC3
:1095C000207A0844C4B200F04FFAA04208D2201A10
:1095D000C1B22A460020FFF78BFC5FEA000AE1D106
:1095E000E6484FF00009C84641684F46C91C21F0C3
:1095F00003014160E248CDF800904E464C4690F899
:1096000001B00EE0204600F024FA4178827809F19A
:109610000109884412FB0177C07810FB0166641CC5
:10962000E4B25C45EED10098D54C00EB890000EB2C
:10963000C80000EB8700217A00EB860000EBC10038
:10964000617ADFF8388300EBC100A17A00EBC1003A
:10965000D8F80410471801213846FFF7DDFA06460E
:1096600029683844884202D8B6F5803F13D3286071
:109670000020FFF75DFC60B1D8F8041045460839BA
:10968000814200D0FFDF6078401E60706868083853
:109690006860042086E700213846FFF7BDFA0446DB
:1096A000A64200D0FFDFE119C8F8041029604FF688
:1096B000FF71A8F80210012188F80010504671E7E8
:1096C0002DE9F0410446AD4817460D46007810B12B
:1096D0000820BDE8F081084609F0FAF808B110202A
:1096E000F7E7A74E307808B9FFF7DFFB601E1E28AA
:1096F00007D8012C3FD12878FE283CD830760020AE
:10970000E7E7A4F120001F2805D8E0B23A46294631
:10971000BDE8F0411EE4A4F140004FF000081F280E
:1097200021D8402C02D0412C25D117E06878297827
:109730004418A97881421ED8FF2C08D807F0FEFBF8
:10974000074608F01DFC381A801EA04201DA1220DC
:10975000BFE728883081A878B07224E02846BDE8A9
:10976000F04100F042BAA4F1A0001F2803D8A02CB9
:1097700003D0A12C06D00720ABE7287800F0010029
:10978000707610E029680920F829A2D38A07A0D1B1
:10979000727B02F00302012A04D1F28AD73293B21B
:1097A0008B4296D8F161404693E72DE9F047074692
:1097B0000C46084609F0B2F840B9384609F0CCF832
:1097C00020B9F81C20F00300B84202D01020BDE8F8
:1097D000F0876B484FF000084430817889B14178B8
:1097E000824600EB4115B4F8009015F8080F2346A7
:1097F00000F00F000022294600F0DFF9060004D037
:1098000013E0A4F800800520E1E797B121884945DD
:1098100001D90C260DE02878234600F00F003A46C7
:10982000294600F0CAF9060005D00C2E01D0A4F894
:1098300000803046CBE79AF801005446401CC0B285
:109840008AF801000B2801D184F80180A078401E1D
:10985000A070697801F00700062827D2DFE800F041
:1098600026091E031E1E0807E3D46888FFF7DAFDE9
:10987000DFE74448696805F01CFC94F8690130B9D9
:109880003E48407800F01AFC94F8690100B1FFDF0F
:1098900094F86901401C84F86901CAE700EB0A01E9
:1098A00091F86801401C81F86801C2E7FFDFC0E75A
:1098B00070B50D46044609F00BF818B9284609F0B2
:1098C0002DF808B1102070BD29462046BDE8704033
:1098D00007F087B970B5044615460E46084608F0ED
:1098E000F7FF18B9284609F019F808B1102070BD23
:1098F000022C03D0102C01D0092070BD2A4631461D
:10990000204607F091F90028F7D0052070BD70B50A
:1099100014460D46064608F0DBFF38B9284608F025
:10992000FDFF18B9204609F017F808B1102070BDE6
:1099300022462946304607F096F90028F7D007203E
:1099400070BD10B596B0044608F0E8FF10B11020C5
:1099500016B010BD0F208DF800000BA9684602F06C
:109960006BFD0028F4D19DF834002070BDF836005E
:109970006080BDF83800A0800020E9E71C000020CE
:1099800010040020C405002070B505460C460846AA
:1099900008F0E2FF20B93CB1206808F0BFFF08B131
:1099A000102070BDA08828B121462846BDE870402F
:1099B000FDF727BE092070BD70B504460D46084668
:1099C00008F086FF30B9601E1E2814D8284608F01B
:1099D0007FFF08B1102070BD022C01D9072070BD97
:1099E00004B9FFDFA64800EB840050F8041C2846A9
:1099F000BDE870400847A4F120001F28EED8294692
:109A00002046BDE87040FAF71FBA70B504460D460F
:109A1000084608F083FF30B9601E1E280DD828467E
:109A200008F056FF08B1102070BD012C01D0022CA7
:109A300001D1062070BD072070BDA4F120001F28B1
:109A4000F9D829462046BDE87040FAF788BA05F0F3
:109A500006B830B58B4D04466878A04200D8FFDFC9
:109A6000686800EBC40030BD70B5864800252C4600
:109A7000467807E02046FFF7ECFF4078641C284456
:109A8000C5B2E4B2B442F5D1284670BD2DE9F0412B
:109A90000646022012B101EB4200401DC7B23068F9
:109AA000C01C20F0030232601BBB76483B460921F4
:109AB000203008F0F9FD002408E0092C11D2DFE87D
:109AC00004F005070509090B0B0505006E4804E0C5
:109AD0006E4802E06E4800E06E4808F005FE05465C
:109AE00000E0FFDFA54200D0FFDF641CE4B2092CD8
:109AF000E3D3306800EB07103060EAE5001D414316
:109B0000452900D24521491EB1FBF0F0401CC0B2EE
:109B100070472DE9FC5F06465A484FF000088B4617
:109B20004746454690F801901FE02846FFF791FF11
:109B3000040000D1FFDFB4F804A0E18801AB6A465D
:109B40005046FFF73FF860789DF804303844C7B2BC
:109B50000AF1040081B280B29DF8002005F04AFCB1
:109B600062786D1C00FB0288EDB24D45DDD1306896
:109B7000C01C20F003003060BBF1000F00D00020BB
:109B80004246394605F044FC316808443060BDE87F
:109B9000FC9F3C49443108710020C8707047394926
:109BA0004431CA782AB10A7801EB42110831814266
:109BB00001D001207047002070472DE9F041044694
:109BC00000201880601E1D4616460F46052800D34B
:109BD000FFDF2B482A46103000EB8400314650F856
:109BE000043C3846BDE8F041184738B50446407893
:109BF00000F00300012803D002280BD0072038BD55
:109C0000606858B108F0B1FED0B9606808F0A4FEF1
:109C100020B915E0606808F05BFE88B96946204607
:109C2000FCF77DF90028EAD1607800F003000228F3
:109C300008D19DF8000028B1606808F08DFE08B1D9
:109C4000102038BD6189F8290DD8208988420AD8AA
:109C5000607800F003020B48012A06D1D731C269AF
:109C600089B28A4201D2092038BD94E80E0000F181
:109C70000C0585E80E000AB900218182002038BD5C
:109C800090E3010010040020AF3C000029C8000050
:109C9000892F00002709010010B5EFF3108000F0B4
:109CA000010472B6E9484178491C417040780128A6
:109CB00001D108F0C5F9002C00D162B610BD70B515
:109CC000E24CE07848B90125E570FFF7E5FF08F0C0
:109CD000BFF920B1002008F09BF9002070BD4FF0C3
:109CE00080406571C0F80453F7E770B5EFF310805A
:109CF00000F0010572B6D54C607800B9FFDF6078DE
:109D0000401E6070607808B908F09EF9002D00D1FF
:109D100062B670BDCD4810B5C17821B10021417146
:109D2000C170FFF7E2FF002010BD10B5044608F037
:109D30008FF9C649C978084000D001202060002072
:109D400010BD2DE9F05FDFF804934278817889F83F
:109D50000620002689F80710074689F80860007871
:109D6000354620B101280FD002280FD0FFDF08F0C0
:109D70007CF998B108F080F9B0420FD1304608F074
:109D80007FF90028FAD047E00126F0E7FFF784FFCB
:109D900008F05EF90028FBD00226E8E701208407DE
:109DA000E060C4F80451AA490E600107D1F84412DA
:109DB000A74AC1F3423124321160A5494FF0020B8A
:109DC00034310860C4F804B3A060DFF888A2DAF880
:109DD0000010C94341F3001101F10108DAF8001045
:109DE00041F01001CAF8001000E020BFD4F80401CF
:109DF0000028FAD0304608F043F90028FAD0B8F12C
:109E0000000F05D1DAF8001021F01001CAF8001097
:109E1000C4F808B3C4F8045199F807004C4670B16F
:109E2000387860B908F014F9074608F005FB6FF0C0
:109E3000004117B1C4E9031001E0C4E9030116B100
:109E40002571BDE8F09F0127BE0727714FF0190863
:109E5000C6F80883B761C6F80051C6F80C51C6F8B9
:109E6000105108F0F5F810B1A770376100E02770C5
:109E7000FFF712FF7649A07920310860C6F8048305
:109E8000DFE770B5050000D1FFDF4FF080424FF0F3
:109E9000FF30C2F808030021C2F80011C2F8041113
:109EA000C2F80C11C2F81011684C617008F0D6F8B5
:109EB00010B10120E07060702846BDE8704040E7B6
:109EC0002DE9F041614C4FF080470125E079F0B178
:109ED000012803D0217A401E814218DA08F0B8F830
:109EE000064608F0A9FAE179012902D9217A491C2C
:109EF00021720EB1216900E0E168411A022902DAFB
:109F000011F1020F0BDC0EB1206100E0E060FFF701
:109F1000C3FE08F09DF828B13D61A57003E07D61A6
:109F2000BDE8F081257000202072F9E72DE9F05F8F
:109F30004948D0F800B0484A4849083211608406C0
:109F4000D4F8080110B14FF0010801E04FF000080B
:109F5000D4F8000100B101208146D4F8040108B111
:109F6000012600E00026D4F80C0100B10120824651
:109F7000D4F8100108B1012700E0002748EA0901E0
:109F800026EA010020EA0A00B84300D0FFDF0025DE
:109F9000B8F1000F04D0C4F80851012008F038F8D7
:109FA0005FEA0900DFF8A4804FF0010913D0C4F87C
:109FB000005198F8050020B188F80550002008F0FD
:109FC00027F898F8000030B108F042F818B188F886
:109FD0000290C4F810900EB1C4F80451BAF1000F09
:109FE0000CD0C4F80C5198F80200464600B9FFDFC7
:109FF000B5703570C4F81490FFF777FE37B1C4F828
:10A00000105198F8040008B1FFF75AFF1249091DD2
:10A01000C1F800B015E770B50C4DE87808B908F044
:10A0200013F801208407A061A87850B1D4F80C017E
:10A0300020B9002008F024F80028F7D10020C4F847
:10A040000C014FF0FF30C4F8080370BD3000002051
:10A050001805004010ED00E010050240010000016D
:10A060004FF0E0214FF00070C1F88001C1F880028C
:10A07000384B802283F80024C1F80001704700B5F6
:10A0800002460420344903E001EBC0031B792BB1E5
:10A09000401EC0B2F8D2FFDFFF2000BD41F83020E3
:10A0A00001EBC00100224A718A7101220A7100BDD0
:10A0B000294A002102EBC0000171704710B5044627
:10A0C000042800D3FFDF244800EBC40420790128D2
:10A0D00000D0FFDF6079A179401CC0B2814200D07E
:10A0E00060714FF0E0214FF00070C1F8000210BD28
:10A0F0002DE9F041194805681849194808310860E8
:10A100001448042690F80004134F4009154C042805
:10A1100018D0FFDF16E0217807EBC1000279012A91
:10A1200008D1427983799A4204D04279827157F8F2
:10A13000310080472078401CC0B22070042801D331
:10A1400000202070761EF6B2E5D20448001D05609E
:10A15000BDE8F08119E000E0F405002010050240A0
:10A160000100000144000020F8B51D46DDE9064766
:10A170000E000AD005F005FA2346FF1DBCB2314699
:10A180002A46009404F08AFEF8BDD01922461946EA
:10A1900013F082FE2046F8BDF84B586019721A8001
:10A1A000C90013F012BF70B50D460446102113F01C
:10A1B000EAFE258117206081A07B40F00A00A07391
:10A1C00070BD4FF6FF720A800146032008F03CBBC9
:10A1D000704700897047827BD30701D1920703D46F
:10A1E000808908800020704705207047827B920795
:10A1F00000D58181704701460020098847F2FE1290
:10A20000114200D00120DD49497A002901D040F0F7
:10A210000800704700B50346807BC00701D00520C9
:10A2200000BD59811846FFF7E6FFC00703D0987BB1
:10A2300040F004009873987B40F001009873002070
:10A2400000BD827B520700D509B1408970471720B5
:10A250007047827B61F3C302827370472DE9F04F30
:10A260000E46017804464FF0010B0BFA01F047F25D
:10A27000FF1100EA010961684FF6FF7887B008888E
:10A280001D469646404506D0B9F1000F07D047F26B
:10A29000FE12104203D0012007B0BDE8F08F40EA63
:10A2A000090008804FF0000A95B185F800A02278D7
:10A2B0000027052003210223102A6FD2DFE802F0D5
:10A2C0006E0D2C35546F768054CBC79CCFFEFDFCB1
:10A2D00020780B28EBD00420DEE762682089937B8E
:10A2E0009B077DD5172851D313898342FBD39289CD
:10A2F000172A01D3824249D12A7822F03F02921CC8
:10A300002A70A5F801003180616888816068817BCE
:10A3100021F00201817342E1042129702189A5F80D
:10A3200001106189A5F803108FE0208A3188C01DD3
:10A330001FFA80F84145D6D3062028702089A5F859
:10A3400001006089A5F80300A089A5F80500072190
:10A35000208ACDE9000160882A4671466369FFF7CB
:10A3600003FFA6F800801AE1082A10D008212970FE
:10A370002189A5F801106189A5F8031030806A1DB4
:10A38000694604F10C0006F06EFC10B1CCE010211F
:10A39000EDE730889DF80010084456E00EE10A20F1
:10A3A00028702089A5F801003180B2E00C212970C5
:10A3B0002189A5F801106189A5F803103080A8E073
:10A3C000218933880BEB41021FFA82FA534576D379
:10A3D000BAF1050F73D30E222A7008EA410100E09A
:10A3E0007FE0CDE9001B60882A467146E368FFF7ED
:10A3F000BBFEA6F800A0D2E06048417A002970D0E8
:10A40000491E41724068217AE26800EBC105D046DE
:10A41000A9882868D2F800C00844A0F1080140F8D3
:10A4200008CC506848608DF800308DF801A028688D
:10A430000290A888ADF8040060886946F7F70BFD24
:10A44000A5F80480002E01D040463080A7E028788F
:10A4500040F080022A70287840F040022A7060891B
:10A460003288C01C1FFA80F842455DD3287820F05E
:10A470003F00123028702289A5F801206089CDE9BB
:10A48000000160882A467146E368FFF76DFEA6F872
:10A490000080287841063CD500065ED58DF800B0D6
:10A4A0008DF801A03188CDE9025A091DADF80410DC
:10A4B0000420DFF8C88003E059E04FE02DE033E0EE
:10A4C000049098F808008DF8140060886946F7F742
:10A4D000C2FC074630880C303080022F02D0E7B330
:10A4E0006FE048E09DF81420D8F8041098F8083080
:10A4F000404601EBC2019A4216D28A88A2B9427A3A
:10A50000521C88F809200D6030888880A6F800A0C9
:10A5100057E061682089888041E0A1893288491D1F
:10A520001FFA81F8424501D204274AE029782A46D9
:10A5300021F03F01163129702189A5F801106189A8
:10A54000A5F80310A189CDE9001060887146236940
:10A55000FFF70AFEA6F80080DBE720E0287820F06D
:10A560003F0018302870207A6870338017E06068E8
:10A570000188090404D4052723E000001406002004
:10A58000C0882189884201D006271AE01E20287041
:10A59000A6F800B06068018821F400410180B9F19B
:10A5A000000F0ED0DF48618800220088830003205E
:10A5B00008F0AAF861682078887007E0A6F800A083
:10A5C00003276068018821EA09010180384663E6B3
:10A5D0002DE9F04F87B01746109C0D0083461E46AC
:10A5E0001AD03078C10703D000F03F00192801D9F4
:10A5F000012100E000212046FFF723FEA8420BD3F3
:10A600002088A0F57F41FF3906D03078410601D47B
:10A61000000603D508203FE607203DE600208DF820
:10A6200000008DF8010030786B1E00F03F0C012215
:10A63000A81E4FF0050A4FF0020999B2BCF1200F95
:10A6400076D2DFE80CF08C10755F7569758D759E9C
:10A6500075B875BD75CB75D775E4757575F475F2FC
:10A6600075F175F0758C052D79D104208DF80000F9
:10A67000A0788DF804007088ADF8060030798DF868
:10A680000100707800F03F000C2829D00ADCA0F10E
:10A690000200092863D2DFE800F0126215621A6234
:10A6A0001D622000122824D004DC0E281BD01028A4
:10A6B000DAD11BE016281FD01828D5D11FE020784A
:10A6C000800701E020784007002848DAF1E0207890
:10A6D0000007F9E72078C006F6E720788006F3E760
:10A6E00020784006F0E720780006EDE72088C005D6
:10A6F000EAE72088C004E7E720888004E4E72088B0
:10A700004004E1E72078800729D5032D27D18DF873
:10A7100000A0B6F8010083E0217849071FD5062D77
:10A720001DD381B27078012803D0022817D102E02E
:10A73000CCE0022000E0102006228DF80020727884
:10A740008DF80420801CB1FBF0F2ADF8062092B227
:10A7500042438A4203D10397ADF80890A9E07BE019
:10A760002078000778D5072198B28DF8001081086D
:10A77000ADF80410B0EB810F6ED10297ADF8062052
:10A7800097E02178C90667D5022D65D381B20820EC
:10A790008DF80000707802285ED300BFB1FBF0F2A4
:10A7A0008DF80400ADF8062092B242438A4253D19C
:10A7B000ADF808907CE0207880064DD5092003E0B4
:10A7C0002078400648D50A208DF80000A088ADF812
:10A7D0000400ADF80610ADF8082069E02078000606
:10A7E00072D50B20ADF804108DF80000ADF80620EE
:10A7F00002975EE02188C90566D5022D64D381B237
:10A800000C208DF80000707804285DD3C6E72088FE
:10A81000C00459D5012D57D10D208DF80000A08816
:10A82000ADF8040045E021E026E016E0FFE72088CF
:10A83000800449D5052D47D30E208DF80000A0884F
:10A84000ADF80400B6F803006D1FADF80850ADF880
:10A850000600ADF80AA02BE036E02088400433D58E
:10A86000012D31D10F208DF8000022E02088000456
:10A870002AD4B6F80100E080A07B000724D5032D80
:10A8800022D3307800F03F001B2819D011208DF81A
:10A890000000208840F40040A4F80000B6F8010051
:10A8A000ADF80400ED1E0320ADF80650ADF8080029
:10A8B000039769465846F7F7CEFA050008D016E028
:10A8C00010208DF80000E9E7072510E008250EE0CC
:10A8D000307800F03F001B2809D01D2807D05946CA
:10A8E000032007F0B1FF208800F400402080A07B07
:10A8F000400708D52046FFF77EFCC00703D1A07BA8
:10A9000020F00400A0732846C6E400B587B00328F1
:10A9100005D18DF8000088B26946F7F79CFA07B0B8
:10A9200000BD000014060020F8B51D46DDE906470D
:10A930000E000AD004F025FE2346FF1DBCB23146AE
:10A940002A46009404F0AAFAF8BDD0192246194606
:10A9500013F0A2FA2046F8BD2DE9FF4F8DB09B46BB
:10A96000DDE91B57DDF87CA00C46082B05D0E0691B
:10A9700001F00CF950B11020D2E02888092140F0F4
:10A98000100028808AF80010022617E0E1690120F3
:10A990008871E2694FF420519180E1698872E06921
:10A9A00042F601010181E0690021817328881121AB
:10A9B00040F0200028808AF80010042638780A9099
:10A9C0000A2038704FF0020904F118004D460C902F
:10A9D00001F0ACFBB04681E0BBF1100F0ED1022DAF
:10A9E0000CD0A9EB0800801C80B20221CDE9001038
:10A9F00005AB52461E990D98FFF796FFBDF816104D
:10AA00001A98814203D9F74800790F9004E003D1E6
:10AA10000A9808B138702FE04FF00201CDE9001913
:10AA20000DF1160352461E990D98FFF77DFF1D98F4
:10AA30000088401B801B83B2C6F1FF00984200D201
:10AA400003461E990BA8D9B15FF00002DDF878C06B
:10AA5000CDE9032009EB060189B2CDE901C10F98C8
:10AA60000090BDF8161000220D9801F0E2FB38703E
:10AA700070B1C0B2832807D0BDF8160020833AE039
:10AA80000AEB09018A19E1E7022011B0BDE8F08F55
:10AA9000BDF82C00811901F0FF08022D0DD09AF8A5
:10AAA0000120424506D1BDF82010814207D0B8F1FF
:10AAB000FF0F04D09AF801801FE08AF80180C9488E
:10AAC00000680178052902D1BDF81610818009EBD4
:10AAD00008001FFA80F905EB080085B2DDE90C10CB
:10AAE00005AB0F9A01F025FB28B91D980088411B82
:10AAF0004145BFF671AF022D13D0BBF1100F0CD141
:10AB0000A9EB0800801C81B20220CDE9000105AB51
:10AB100052461E990D98FFF707FF1D9805800020EB
:10AB200038700020B1E72DE9F8439C46089E134693
:10AB30000027B26B9AB3491F8CB2F18FA1F57F4504
:10AB4000FF3D05D05518AD882944891D8DB200E020
:10AB500000252919B6F83C800831414520D82A44FF
:10AB6000BCF8011022F8021BBCF8031022F8021BEB
:10AB7000984622F8024B914604F0F1FC4FF00C0C81
:10AB800041464A462346CDF800C004F04EF9F58709
:10AB9000B16B00202944A41D2144088003E001E09A
:10ABA000092700E083273846BDE8F88310B50B88F5
:10ABB000848F9C420CD9846BE018048844B184884B
:10ABC00024F40044A41D23440B801060002010BD19
:10ABD000822010BD2DE9F0478AB0002590468946B5
:10ABE0008246ADF8185007274BE005980688808804
:10ABF000000446D4A8F8006007A8019500970295C4
:10AC0000CDE903504FF4007300223146504601F065
:10AC100010FB04003CD1BDF81800ADF820000598E9
:10AC200004888188B44216D10A0414D4019502958F
:10AC3000039521F400410097049541F48043428834
:10AC40002146504601F0CCF804000BD105988188CC
:10AC500041F40041818005AA08A94846FFF7A6FFF4
:10AC60000400DCD0009705980295019503950495A2
:10AC70000188BDF81C300022504601F0B1F8822C4A
:10AC800006D105AA06A94846FFF790FF0400ACD0FC
:10AC9000ADF8185004E00598818821F400418180C6
:10ACA00005AA06A94846FFF781FF0028F3D0822CA9
:10ACB00003D020460AB0BDE8F0870020FAE710B5BF
:10ACC0000C46896B86B051B10C218DF80010A18F14
:10ACD000ADF80810A16B01916946FCF79BF90020C3
:10ACE0004FF6FF71A063E187A08706B010BD2DE984
:10ACF000F0410D460746896B0020069E1446002948
:10AD000011D0012B0FD1324629463846FFF762FF9A
:10AD1000002808D1002C06D0324629463846BDE826
:10AD2000F04100F042BFBDE8F0812DE9FC4114463E
:10AD3000DDE9087C0E46DDE90A15521DBCF800E08D
:10AD400092B2964502D20720BDE8FC81ACF8002003
:10AD500017222A70A5F80160A5F803300522CDE975
:10AD600000423B462A46FFF7DFFD0020ECE770B5C6
:10AD70000C4615464821204613F027F904F1080037
:10AD800044F81C0F00204FF6FF71E06161842084BD
:10AD9000A5841720E08494F82A0040F00A0084F883
:10ADA0002A0070BD4FF6FF720A800146042007F0AA
:10ADB0004BBD30B585B00C460546FFF780FFA18E30
:10ADC000284629B101218DF800106946FCF722F9C7
:10ADD0000020E0622063606305B030BDB0F8400041
:10ADE000704700004800002090F84620920703D4E6
:10ADF000408808800020F3E70620F1E790F846201D
:10AE00009207EDD5A0F84410EAE701460020098832
:10AE10000A0700D5012011F0F00F01D040F0020028
:10AE2000CA0501D540F004008A0501D540F01000A4
:10AE30004A0501D540F020000905D1D540F0400079
:10AE4000CEE700B5034690F84600C00701D00620C3
:10AE500000BDA3F842101846FFF7D7FF10F0760F99
:10AE600005D093F8460040F0040083F8460013F83C
:10AE7000460F40F001001870002000BD90F84620F9
:10AE8000520700D511B1B0F84200A9E71720A7E793
:10AE900010F8462F61F3C3020270A1E72DE9FF4FBE
:10AEA0009BB00E00DDE92B34DDE92978289D25D003
:10AEB0002878C10703D000F03F00192801D90121EB
:10AEC00000E000212046FFF7D9FFB04216D32878D2
:10AED00041060FD400F03F011E2909D0218811F44A
:10AEE0007F6F0BD13A884AB1A1F57F42FF3A05D076
:10AEF000010606D500F03F00122802D004201FB042
:10AF0000C4E5FC491D984FF0000A08718DF818A09F
:10AF10008DF830A00CAA0A60ADF81CA0ADF824A0F2
:10AF20002978994601F03F02701F5B1C04F1180C50
:10AF3000D3464FF0030ECDF828C01F2A7ED2DFE89B
:10AF400002F07D7D107D227DAE7DF77DF67DF57D65
:10AF5000F47DF77DF37D7D7DF27DF17D7D7D7D7DD1
:10AF6000F00094F84610B5F80100890767D5032E64
:10AF700065D14FF40061ADF8241060808DF830E0A9
:10AF8000ADF83400E9E2052EF2D1B5F801002083D6
:10AF9000ADF81C00B5F803106183002870D088421A
:10AFA0006ED884F80AB0A4F808B04FF6FF70208479
:10AFB0000A9801F0BBF8052089F8000002208346BA
:10AFC000029011AB1D9A0A991B9801F0B2F820B1BA
:10AFD0005EE000BF8DF81800FEE29DF84A000128EF
:10AFE00004D0022089F80100102003E0012089F834
:10AFF000010002200390002204A912A805F033FEEC
:10B00000E8BB9DF81010039888423ED13A88891C0D
:10B01000A2EB0B00884238DB02990220CDE9000147
:10B020000DF146034A4641461B98FFF77DFC029806
:10B030000BF1020B801C81B217AA01E0ACE2B1E077
:10B04000029104A912A805F00EFE02999DF81000C5
:10B05000CDE9000117AB4A4641461B98FFF764FC57
:10B060009DF8100011AB0BEB00011FFA81FB029958
:10B070001D9A084480B202900A991B9801E004E0EE
:10B0800091E001F056F80028B5D0BBF1020F03D1D2
:10B090000A208DF818005DE2A7F800B05AE2CDF85A
:10B0A0000CB0072E7ED3B5F801002083ADF81C004C
:10B0B000B5F803206283002875D0904273D84FF012
:10B0C000010B84F80AB0B5F8050020810020A073B8
:10B0D000E06900F05BFD80B9E16942F6010081F8AA
:10B0E00006B0E2694FF420519180E16981F80AB01D
:10B0F000E1690881E16900208873F01F20841E98AF
:10B100004FF0070B6062A4F822B00A9801F00EF825
:10B1100089F800B00120834604900020ADF8460075
:10B120002AE026E2B0E147E1EDE01FE2B0E088E08E
:10B130004FE000BFBBF1010F15D0E0698079012815
:10B1400003D1BDF84400ADF80E0004990420CDE908
:10B15000000103AB4A4641461B98FFF7E5FB049804
:10B16000001D80B20490BDF84600ADF80C00ADF8AB
:10B170000E0005981FFA80FB11AB1D9A0A991B98C7
:10B1800000F0D7FF28B939880BF1040005908142FF
:10B19000D0D2BBF1010F3FF41BAFE06980790128E9
:10B1A00008D001E098E023E0BDF84410A1F57F400D
:10B1B000FF3803D1BDF84400ADF80E000499042017
:10B1C000CDE9000103AB4A4641461B98FFF7ACFBB3
:10B1D00062E7072E01D0152E7ED1B5F8011021832C
:10B1E000ADF81C10B5F80320628309B1914201D972
:10B1F0000120EFE60121A172A4F808B084F80EB096
:10B20000052E07D0C0B2691DE26905F00DFD0028CA
:10B210007FF4DEAE4FF6FF70208401A806AA09A9CC
:10B22000CDF800B080E886032878214600F03F037F
:10B230001D9A1B98FFF790FB8246208BADF81C00EF
:10B2400088E10120032EC7D14021ADF82410B5F8C4
:10B2500001102183ADF81C100AAAB8F1000F00D02C
:10B260000023CDE9020304921D98CDF804800090DC
:10B2700038880022401E83B21B9800F0DAFF8DF858
:10B28000180050BB0B2189F80010BDF8280038E0E9
:10B290004FF0010C052E9FD18020ADF82400B5F8A9
:10B2A00001102183B5F803002084ADF81C10B0F51F
:10B2B000007F01D907208DE640F47C42228412A849
:10B2C000B8F1000F00D00023CDE90330CDE9018CA7
:10B2D0001D980090388801E09CE007E0401E83B292
:10B2E0001B9800F0A6FF8DF8180028B18328A7D17D
:10B2F0000220C7E0480000200D2189F80010BDF8A9
:10B300004800401C25E1C80900EB40020EEB82001A
:10B31000B04203D948067DD558461AE1B5F8011068
:10B32000ADF81C102A78520608D506228DF8302078
:10B330002A78120605D58DF830B02FE107228DF856
:10B3400030200323CDE9023BDDF878C0CDF810B002
:10B350001D9AA6EB00080092CDF804C01FFA88F3EE
:10B3600000221B9800F03CFD8DF818008DF830B0DD
:10B37000297849060DD52088C00506D5208BBDF853
:10B380001C10884201D1C4F824B058468DF818B07A
:10B39000DFE0832801D14FF0020A4FF48070ADF84E
:10B3A0002400BDF81C002083A4F820801E98606251
:10B3B000032060841321C9E0052E2BD3B5F80110BA
:10B3C000ADF81C10A28F32B3A2F57F43FE3B29D00B
:10B3D00008228DF830200523CDE9023BDDF878C046
:10B3E000CDF810B01D9A80B2CDF804C040F40043EF
:10B3F0000092B5F803201B9800F0F2FC4FF40071A6
:10B400008DF818008DF830B0ADF82410832813D0D3
:10B4100010B301E0DBE005E0A08FA0F57F41FE392D
:10B4200007D0D9E00B228DF830204FF6FE72A287AC
:10B43000D1E7A4F83CB0CFE000942B4631461E9AE9
:10B440001B98FFF770FB8DF8180008B183284BD1CB
:10B45000BDF81C0020834BE700942B4631461E9A12
:10B460001B98FFF760FB8DF81800E8BBE18FA06B1D
:10B470000844831D8DE888034388828801881B98CF
:10B48000FFF753FC824665E095F80180022E6FD1EC
:10B490005FEA080002D0B8F1010F7FD109208DF8D2
:10B4A000300007A800908DF83480434600222146E2
:10B4B0001B98FFF71CFC8DF835008DF836B050B99D
:10B4C000B8F1010F11D0B8F1000F04D1A08FA0F591
:10B4D0007F41FF3909D0A08F38B14FF480608DF8DB
:10B4E00030B0ADF824000EE034E00CA91B98FBF757
:10B4F00091FD82464FF480608DF830B0ADF82400A5
:10B50000BAF1020F06D0FB480068807928B18DF8A7
:10B51000180027E0A4F8188042E0BAF1000F03D029
:10B5200081208DF818003BE007A8009043460122D7
:10B5300021461B98FFF7DBFB8DF8180021461B986E
:10B54000FFF7BDFB9DF8180020B9192189F80010FC
:10B55000012038809DF8300020B10CA91B98FBF722
:10B5600059FD8246BAF1000F33D019E0062031E5CB
:10B5700014E02078000711D5012E0FD10A208DF894
:10B580003000E088ADF8340004201B9907F05CF926
:10B590000820ADF824007FE5480618D54FF0040ACE
:10B5A0002088BDF8241008432080BDF824008005C1
:10B5B0000BD5A18FA1F57F40FE3806D11E98E06221
:10B5C00028982063A6864FF0030A504697E404208B
:10B5D00000E59DF8180078B1012089F8000029786D
:10B5E00089F80110BDF81C10A9F802109DF8180088
:10B5F00089F80400052038802088BDF8241088438D
:10B600002080E2E72DE9FF4F8846087895B00121B8
:10B6100081404FF20900249C0140ADF820102088A1
:10B62000DDF88890A0F57F424FF0000AFF3A02D083
:10B6300029B1000703D5012019B0BDE8F08F239E82
:10B640004FF0000B0EA886F800B018995D460988E7
:10B65000ADF83410A7498DF81CB0179A0A718DF80F
:10B6600038B0086098F8000001283BD0022809D0C3
:10B6700003286FD1307820F03F001D303070B8F8CB
:10B680000400E08098F800100320022904D13178EA
:10B6900021F03F011B31317094F84610090759D54C
:10B6A00005ABB9F1000F13D0002102AA82E80B000C
:10B6B0000720CDE90009BDF83400B8F80410C01E19
:10B6C00083B20022159800F0B4FD0028D1D101E02A
:10B6D000F11CEAE7B8F80400A6F80100BDF8140070
:10B6E000C01C04E198F805108DF81C1098F80400AF
:10B6F000012806D04FF4007A02282CD00328B8D1B4
:10B700006BE12188B8F8080011F40061ADF8201051
:10B7100020D017281CD3B4F84010814218D3B4F8B5
:10B720004410172901D3814212D1317821F03F0111
:10B73000C91C3170A6F801000321ADF83410A4F83B
:10B74000440094F8460020F0020084F8460064E1CA
:10B7500005257DE176E1208808F1080700F4FE6008
:10B76000ADF8200010F0F00F1BD010F0C00F03D088
:10B770003888228B9042EBD199B9B878C00710D0A5
:10B78000B9680720CDE902B1CDF804B00090CDF83A
:10B7900010B0FB88BA883988159800F021FB002882
:10B7A000D6D12398BDF82010401C80294ED006DC4D
:10B7B00010290DD020290BD0402987D124E0B1F5E4
:10B7C000807F70D051456DD0B1F5806F97D1DDE0AD
:10B7D000C80601D5082000E0102082460DA907AA5E
:10B7E0000520CDE902218DF83800ADF83CB0CDE957
:10B7F000049608A93888CDE900015346072221465E
:10B800001598FFF7A9F8A7E09DF81C2001214FF03B
:10B810000A0A002A9BD105ABB9F1000F00D0002025
:10B82000CDE902100720CDE90009BDF834000493EA
:10B83000401E83B2218B0022159800F0FAFC8DF88F
:10B840001C000B203070BDF8140020E09DF81C2077
:10B8500001214FF00C0A002A22D113ABB9F1000FDD
:10B8600000D00020CDE902100720CDE900090493A3
:10B87000BDF83400228C401E83B2218B159800F055
:10B88000D8FC8DF81C000D203070BDF84C00401C19
:10B89000ADF8340005208DF83800208BADF83C0061
:10B8A000BBE000E028E03888218B88427FF450AF6D
:10B8B0009DF81C004FF0120A00281AD1606A98B156
:10B8C000B878C0073FF444AFBA680720CDE902B2A8
:10B8D000CDF804B00090CDF810B0FB88BA88159868
:10B8E00000F07EFA8DF81C00132030700120ADF8B6
:10B8F000340092E0480000203988208B8142D5D165
:10B900009DF81C004FF0160A0028A06B08D0E0B389
:10B910004FF6FF7000215F46ADF808B0019027E0B8
:10B9200068B1B978C907C1D1E18F0DAB0844821D58
:10B9300003968DE80C0243888288018809E0B87874
:10B94000C007BFD0BA680DAB03968DE80C02BB8868
:10B95000FA881598FFF7E9F905005ED0072D72D037
:10B9600076E0019005AA02A92046FFF71FF90146DB
:10B97000E28FBDF80800824201D00029F1D0E08FAB
:10B98000A16B084407800198E08746E09DF81C0001
:10B990004FF0180A40B1208BC8B138882083214667
:10B9A0001598FFF78CF938E004F118000090237E19
:10B9B000012221461598FFF79AF98DF81C000028FE
:10B9C000EDD1192030700120ADF83400E7E70525EE
:10B9D00021461598FFF773F93AE0208800F40070CB
:10B9E000ADF8200050452DD1A08FA0F57F41FE3944
:10B9F00001D006252CE0D8F808004FF0160A48B10F
:10BA0000A063B8F80C10A1874FF6FF71E187A0F88A
:10BA100000B002E04FF6FF70A087BDF8200030F4C0
:10BA20007F611AD0782300220420159906F06CFE5D
:10BA300098F8000020712088BDF82010084320806D
:10BA40000EE000E007252088BDF820108843208004
:10BA5000208810F47F6F1CD03AE021888143218038
:10BA60009DF8380020B10EA91598FBF7D3FA0546CA
:10BA70009DF81C000028EBD086F801A00120307052
:10BA8000208B70809DF81C0030710520ADF83400CB
:10BA9000DEE7A18EE1B118980DAB0088ADF8340057
:10BAA0002398CDE90304CDE90139206B0090E36AC6
:10BAB000179A1598FFF7F2F9054601208DF838001E
:10BAC0000EA91598FBF7A6FA00B10546A4F834B004
:10BAD00094F8460040070AD52046FFF796F910F083
:10BAE000760F04D114F8460F20F004002070189847
:10BAF000BDF83410018028469EE500B585B00428C5
:10BB000006D102208DF8000088B26946FBF782FA60
:10BB100005B000BD10B5384C0B782268012B02D05F
:10BB2000022B2AD111E013780BB1052B01D104238C
:10BB3000137023688A889A802268CB88D380226811
:10BB40000B891381498951810DE08B88938022688C
:10BB5000CB88D38022680B8913814B8953818B89D1
:10BB60009381096911612168FBF754FA2268002169
:10BB70000228117003D0002800D0812010BD83203E
:10BB800010BD806B002800D001207047817801290A
:10BB900009D10088B0F5205F03D042F60101884248
:10BBA00001D10020704707207047F0B587B000240E
:10BBB00015460E460746ADF8144010E00698018879
:10BBC0002980811DCDE9024107210194049400914F
:10BBD000838842880188384600F002F930B906AA05
:10BBE00005A93046FEF7E2FF0028E7D0822800D101
:10BBF000002007B0F0BD00004800002010B58B7891
:10BC000083B102789A4205D10B885BB102E08B794F
:10BC1000091D4BB18B789A42F9D1B0F801300C88EC
:10BC2000A342F4D1002010BD812010BD072826D0EA
:10BC300012B1012A27D103E0497801F0070102E09F
:10BC40004978C1F3C20105291DD2DFE801F00318CC
:10BC5000080C12000AB10320704702207047042824
:10BC60000DD250B10DE0052809D2801E022808D35C
:10BC700003E0062803D0032803D0052070470020E6
:10BC800070470F20704781207047C0B2820610D4E1
:10BC900000060CD5FA48807A421ED31702EB537285
:10BCA000012303EBE20201FB002080B2704708464B
:10BCB00070470020704770B513880B800D782B06F5
:10BCC0002AD5EF4B9B7A834204D845F010000870C8
:10BCD000002070BD946800F0070604EBD0042478BF
:10BCE000F44064F304150D701478D17804F0030463
:10BCF00041EA042140F20124B1FBF4F504FB1511E3
:10BD000092685B1E00FB0120D91703EB51710122E1
:10BD100002EBE101084470BD906870BD37B5144670
:10BD2000BDF8041011809DF804100A0622D5C1F355
:10BD30000013D3490122A568897A81420CD8FE28D4
:10BD400014D1491EC81701EB507002EBE0015A42B2
:10BD50002846F7F746F909E005EBD00100F00705A2
:10BD60000878AA409043AB4018430870207820F030
:10BD7000100020703EBD2DE9F0410746C81C0E465C
:10BD800020F00300B04202D08620BDE8F081BC4D17
:10BD9000002034462E60AF802881AA72E8801AE025
:10BDA000E988491CE980810614D4E17800F0030099
:10BDB00041EA002040F20121B0FBF1F201FB120147
:10BDC0002068FFF762FF2989084480B22881381A69
:10BDD0003044A0600C3420784107E1D40020D4E73F
:10BDE0002DE9FF4F89B01646DDE9168A0F469946C0
:10BDF00023F44045084600F00CFB04000FD00998DE
:10BE000003F06AFA0290207800060AD59C48817AED
:10BE10000298814205D887200DB0BDE8F08F01203F
:10BE2000FAE7224601A90298FFF745FF8346002062
:10BE30008DF80C004046B8F1070F1AD001222146B8
:10BE4000FFF7F4FE0028E7D12078400611D5022044
:10BE50008DF80C00ADF81070BDF80400ADF81200BC
:10BE6000ADF814601898ADF81650CDF81CA0ADF8D8
:10BE700018005FEA094004D500252E46A846012790
:10BE80000CE02178E07801F0030140EA012040F263
:10BE90000121B0FBF1F2804601FB12875FEA4940C5
:10BEA00009D5B84507D1A178207901F0030140EA0E
:10BEB0000120B04201D3BE4201D90720ACE7A81946
:10BEC0001FFA80F9B94501D90D20A5E79DF80C00AE
:10BED00028B103A90998FBF79BF800289CD1B84525
:10BEE00007D1A0784FEA192161F30100A07084F80E
:10BEF00004901A9800B10580199850EA0A0027D0DA
:10BF0000199830B10BEB06002A46199911F0C4FFBD
:10BF10000EE00BEB06085746189E099803F01FFB2E
:10BF20002B46F61DB5B239464246009502F07DFF1C
:10BF3000224601A90298FFF7BEFE9DF804002246A2
:10BF400020F010008DF80400DDE90110FFF7E6FE97
:10BF5000002061E72DE9FF4FDFF824918246174664
:10BF6000B9F80610D9F8000001EB410100EB81049B
:10BF700040F20120B2FBF0F185B000FB11764D4696
:10BF8000DDF84C8031460698FFF77FFE29682A8944
:10BF90008B46611A0C3101441144AB8889B28B4243
:10BFA00002D8842009B038E70699CDB2290603D516
:10BFB000A90601D58520F5E7B9F806C00CF1010CFA
:10BFC0001FFA8CFCA9F806C0149909B1A1F800C0A9
:10BFD000A90602D5C4F8088007E0104480B2A9F889
:10BFE0000800191A01EB0B00A0602246FE200699FA
:10BFF000FFF794FEE77026712078390A61F301009B
:10C00000320AA17840F0040062F30101A1702070AF
:10C010009AF802006071BAF80000E08000262673EA
:10C02000280602D599F80A7000E00127A80601D574
:10C030004FF000084D4600244FF007090FE0CDE90E
:10C0400002680196CDF800900496E9882046129B7C
:10C05000089AFFF7C5FE0028A4D1641CE4B2BC42D4
:10C06000EDD300209EE72DE9F047804600F0D1F99E
:10C07000070007D000264446014D40F2012918E090
:10C08000200600200120BDE8F087204600F0C1F91D
:10C090000278C17802F0030241EA0222B2FBF9F30E
:10C0A00009FB13210068FFF7F0FD3044641C86B2E1
:10C0B000A4B2E988601E8142E7DCA8F10100E880B3
:10C0C0002889801B288100203870DCE710B51446D1
:10C0D00031B1491E218003F0FFF8A070002010BD8F
:10C0E000012010BD10B5D34904460088CA8890428B
:10C0F00001D3822010BD096800EB400001EB8002F3
:10C100005079A072D08820819178107901F00301D4
:10C1100040EA0120A081A078E11CFFF7CCFD20615E
:10C120002088401C2080E080002010BD0121018279
:10C1300070472DE9FF4F85B04FF6FF788246A3F890
:10C14000008048681F460D4680788DF806004868D4
:10C150000088ADF8040000208DF80A00088A0C88D9
:10C16000A04200D304462C8241E0288A401C288249
:10C17000701D6968FFF742FDB8BB3988414501D1A0
:10C18000601E38806888A04236D3B178307901F0DB
:10C19000030140EA012901A9701DFFF72FFD20BB13
:10C1A000298941452CD0002231460798FFF73EFDF2
:10C1B000D8B92989494518D1E9680391B5F80AC069
:10C1C000D6F808B05046CDF800C003F0C8F9DDF845
:10C1D00000C05A460CF1070C1FFA8CFC4B46039921
:10C1E000CDF800C002F0E4FD50B1641CA4B22046BA
:10C1F00000F00FF90600B8D1641E2C828220D1E62F
:10C200007C807079B871F088B8803178F07801F06E
:10C21000030140EA01207881A7F80C90504603F012
:10C220005BF8324607F10801FFF745FD3861002051
:10C23000B8E62DE9FF4F87B081461C469246DDF8EF
:10C2400060B0DDF85480089800F0E3F805000CD0E9
:10C25000484603F041F82978090608D57549897AD6
:10C26000814204D887200BB0D7E50120FBE7CAF351
:10C2700009062A4601A9FFF71EFD0746149807285C
:10C280001CD000222946FFF7D1FC0028EBD12878EA
:10C29000400613D501208DF808000898ADF80C0071
:10C2A000BDF80400ADF80E00ADF81060ADF8124016
:10C2B00002A94846FAF7ACFE0028D4D12978E878DC
:10C2C00001F0030140EA0121AA78287902F0030273
:10C2D00040EA0220564507D0B1F5007F04D9611E1F
:10C2E000814201DD0B20BEE7864201D90720BAE773
:10C2F000801B85B2A54200D92546BBF1000F01D0B5
:10C30000ABF80050179818B1B9192A4611F0C4FDBE
:10C31000B8F1000F0DD03E4448464446169F03F046
:10C3200030F92146FF1DBCB232462B46009402F084
:10C33000B5FD002097E72DE9F04107461D4616465A
:10C34000084600F066F804000BD0384602F0C4FF3F
:10C350002178090607D53749897A814203D8872091
:10C3600013E5012011E522463146FFF7A4FC65B133
:10C370002178E07801F0030140EA0120B0F5007F68
:10C3800001D8012000E0002028700020FDE42DE904
:10C39000F04107461D461646084600F03AF80400EC
:10C3A0000BD0384602F098FF2178090607D52149BD
:10C3B000897A814203D88720E7E40120E5E4224618
:10C3C0003146FFF7ABFCFF2D14D02178E07801F067
:10C3D000030240EA022040F20122B0FBF2F302FB2A
:10C3E000130015B900F2012080B2E070000A60F37A
:10C3F000010121700020C8E410B50C4600F009F8D6
:10C4000028B1C18821804079A070002010BD012092
:10C4100010BD0849CA88824209D340B1096800EBBF
:10C4200040006FF00B0202EB8000084470470020D0
:10C43000704700002006002010B50C4602F051F8AD
:10C4400080B3204600F05BFE68B322780F2A09D043
:10C45000102A07D0022A05D0032A03D0142A2ED08E
:10C46000FFDF1DE0A0781E282DD00EDC0C2824D084
:10C4700008DC092827D2DFE800F013261726261E3D
:10C480001E1A1C0012281ED11BE0302819D01ADDFC
:10C49000A0F13A00032816D2DFE800F011150B00D6
:10C4A000002010BD13E010E043F20200F9E7042081
:10C4B000F7E70D20F5E70F20F3E70820F1E711205B
:10C4C000EFE70720EDE70320EBE7FFDFE8E7FFDF1B
:10C4D000E6E700F014BE70B50346002002466FF098
:10C4E0002F050EE09C5CA4F130060A2E02D34FF01B
:10C4F000FF3070BD00EB800005EB4000521C204473
:10C50000D2B28A42EED370BD30B50A240AE0B0FB45
:10C51000F4F304FB13008D18303005F8010C521EA3
:10C520001846D2B2002AF2D130BD30B500234FF602
:10C53000FF7510E0040A44EA002084B2C85C604041
:10C54000C0F30314604005EA00344440E0B25B1CD1
:10C5500084EA40109BB29342ECD330BDF0B516464E
:10C560000B880122B240134215D113430B800446BD
:10C57000051D018840880F18092F00D3093F401C72
:10C58000092800D9FFDF781C092800D9FFDF60885F
:10C59000401C6080EE55F0BDF0B506880446051DD0
:10C5A0000F46701C81B22180092901D309392180ED
:10C5B0006088012800D2FFDF701C092800D9FFDF46
:10C5C00060880122401E6080A85D398882409143C6
:10C5D0003980F0BD2DE9F0410E468046DDE9065078
:10C5E00089781746090612D420F8045D4380404636
:10C5F00002F0C7FF040000D1FFDF2D1D2046A9B2C5
:10C6000002F024F900B9FFDF404600F01AFC06EB07
:10C610004701087C401C0874BDE8F0817CB50546E4
:10C620001220187048780C46801C587008205880DA
:10C63000108898805088D88090881881D088588138
:10C640000C20CDE900030523062221462846FFF7EA
:10C65000C1FFF02300222946012006F055F860783A
:10C66000801C60707CBD2DE9F84F0F469A469146BC
:10C670000546032102F068FE0446808CDFF86085E1
:10C68000002618B198F80000B84221D1284602F0DF
:10C6900078FF050000D1FFDF09F10401284689B2C7
:10C6A00002F084F8060013D002F032FC077028462E
:10C6B00031466A4602F06BFB009800210A46018071
:10C6C000817000F081FC0098C01DCAF8000030E0C5
:10C6D00098F80000B84225D104F1220534F8301F43
:10C6E000012000FA07F911EA090F00D0FFDF2088C6
:10C6F00040EA090020802C8805F10409641E092CF9
:10C7000000D309342C806888401C092800D9FFDF39
:10C71000601C092800D9FFDF6888401C688009F880
:10C72000047006E03A4604F1300104F12200FFF7FC
:10C7300015FF092188F800103046BDE8F88F38B59C
:10C740000546032102F000FE0446807800F07F00D9
:10C75000012814D002226B4606212846121DFFF73D
:10C7600082FF00280AD0A07800F07F00012808D0BE
:10C77000228921462846009B00F084FA38BD082211
:10C78000E9E704F1080221462846009BFFF746FF2F
:10C7900038BDFEB514460D46064602AB06220721FB
:10C7A000FFF761FF80B1029B0120072218705C70C7
:10C7B0000220588000249C800620CDE90003052338
:10C7C00029463046FFF706FFEC70FEBD10B5044663
:10C7D000032102F0B9FD0146C2782046BDE81040B1
:10C7E000D7E7FF4909200870704770B50C46154619
:10C7F0003421204611F0E9FB0120607020781221DD
:10C8000020F00F00207004F1100011F0DEFB05B9DC
:10C81000FFDF2978A07861F30600A07070BD704733
:10C820000146012006F010B83EB58DB2032128461E
:10C8300002F08AFD040000D1FFDF2078002220F002
:10C840000F00207002208DF800004FF6FF70ADF849
:10C850000200ADF8040069462846F7F79AFA3EBD93
:10C86000F0B50C4600260078012117463546B1EB9D
:10C87000101F00D0FFDFFFDF3D800CB126806580F8
:10C880000020F0BD2DE9FC4788461D46174681462D
:10C8900003210A9E02F058FD040000D1FFDFCDE91C
:10C8A00000563B46424621464846FFF793FEBDE808
:10C8B000FC8738B50546A0F57F40FF381CD02846D8
:10C8C00002F04DFE040000D1FFDF204602F03EFAE8
:10C8D000002810D001466A46204602F058FA009817
:10C8E000B0F80500052807D10321284602F02CFDE9
:10C8F000C07808B1002038BD012038BD2DE9FF41C6
:10C900000546408802F02BFE040000D1FFDF03AA99
:10C910002046696800F0ADF9039C001F34F8032F2E
:10C92000618882420AD104290AD0052917D0062934
:10C9300004D16888211D6B68F8F74FFFBDE8FF81BF
:10C940001646241D2A4621463046F5F72BFD0828B9
:10C95000F4D12A4621463046FAF7B9FEEEE71646EC
:10C960006888032102F0F0FC014600208DF80000E9
:10C97000042EE3D36279002AE0D0237943F3000048
:10C98000401C05D14F789742D8D10F783F07D5D0BA
:10C99000142B3CDA4FF002074FF6FF78012B34D00E
:10C9A000122B02D0132B32D11DE00C2E2FD18B78FD
:10C9B00003F07F03012B2AD0087820F00F00401CE1
:10C9C00008706079487001208DF800002089ADF86A
:10C9D00002006089ADF80400A089ADF80600E08986
:10C9E000ADF8080028E0062E11D1087820F00F00DD
:10C9F00008706988012005F027FF8DF80070ADF8F8
:10CA000002802089ADF8040016E0062E05D000282B
:10CA100094D06888FFF7BDFE90E7087820F00F00FB
:10CA200008706988012005F00FFF8DF800702089DB
:10CA3000ADF80200ADF8048068882A466946F7F729
:10CA4000A8F97BE7F8B50D460646032102F07CFC09
:10CA5000040012D0207800F00F00012810D06B469F
:10CA60000C2206213046FFF7FEFD58B12A4621462A
:10CA70003046009BFFF7D2FD08E043F20200F8BD0C
:10CA80001120F8BD2868A0606868E060207820F078
:10CA90000F00401C20700020F8BDF8B50D4606467A
:10CAA000032102F051FC040006D0207800F00F00B2
:10CAB000012804D00820F8BD43F20200F8BD062288
:10CAC0006B4611463046FFF7CEFD30B12A4621466F
:10CAD0003046009B00F0D6F800E02581207820F059
:10CAE0000F0020700020F8BD2DE9F04F0F4691B0E7
:10CAF0008046032102F028FC0446404602F041FD36
:10CB00004FF00009CDF82090CDF82490ADF8349086
:10CB10000546CDF82890CDF82C90CDF80890CDF8AA
:10CB20000C90CDF8109004B9FFDF02AE05B9FFDF1D
:10CB3000B2467F1EFFB219D328460CA9002201F08D
:10CB40008EFF9DF83060092E00D3FFDF04EB460115
:10CB50003246087C401E08740DA908A8FFF7FEFCA9
:10CB60001AF80610491C0AF80610E2E704F1300032
:10CB700006900E381A4FDFF86CB0051D059010E0D6
:10CB8000DDE90501FFF708FD06463870092800D3E6
:10CB9000FFDF5BF8261040468847608C405DB0425E
:10CBA00002D0A08C0028EBD109200E4E387024361C
:10CBB00020E00DA908A8FFF7EFFC054604EB4507A8
:10CBC000787CC00716D02946204600F054F808B9F2
:10CBD00087F811901AF8057056F8250028B903E077
:10CBE00050000020B8E30100FFDF56F82520394649
:10CBF00040469047BDF822000028DAD111B0BDE8C8
:10CC0000F08F10B5032102F09FFB040000D1FFDF7D
:10CC1000122104F1100011F0D8F9A07840F0800042
:10CC2000A07010BD70B50D46032102F08DFB04000D
:10CC300000D1FFDF092D00D3FFDF2946204600F099
:10CC40001AF8002803D004EB45020121517470BD8D
:10CC500070B50D46032102F077FB0446294600F02B
:10CC60000AF820B9208E0121A940084000D00120F7
:10CC700070BD02F08CB800EB4100007C002800D0B1
:10CC8000012070471CB513241C704C785C70022482
:10CC90005C809A800622CDE900230523FFF79AFCE9
:10CCA0001CBD000010B509F066FB042803D009F094
:10CCB00062FB052802D108F03DF828B90AF01EFCF5
:10CCC00020B107F005F808B1012010BD002010BD0B
:10CCD0000178406819B190F8691059B901E001F084
:10CCE00073BC90F8FC1029B190F8FC00042801D026
:10CCF000012070470020704770B50C46054606219C
:10CD000002F022FB606008B1002006E007212846FF
:10CD100002F01AFB606018B101202070002070BD85
:10CD2000022070BD2DE9FC470C4606466946FFF718
:10CD3000E3FF00287DD19DF8000050B106F05AFFB6
:10CD4000B0427CD0214630460CF078FC002873D1EC
:10CD50002DE007F03BFDB04271D0214630460BF08C
:10CD60008DFA002868D1019D95F8C00022E00120CD
:10CD700000E00020804695F835004FF0010A4FF0A2
:10CD80000009F0B195F8360080071AD584F80190B3
:10CD900084F800A084F80290A68095F83710A1715D
:10CDA000298F2181698F618185F8359044E0019D4B
:10CDB00095F8FC0050350028DBD1687E0028D8D0DB
:10CDC000D5E7304602F0DDFB070000D1FFDF384633
:10CDD00001F0F9FD40B184F801900D212170A68089
:10CDE000E08084F802A027E0304602F0B8FB07009C
:10CDF00000D1FFDFB8F1000F21D0384601F074FEFA
:10CE0000B8B19DF8000038B90198D0F8E400418825
:10CE1000B14201D180F80090304606F0A5FD84F8BB
:10CE200001900A21217084F80290A680A97EA17148
:10CE300000E004E085F819900120BDE8FC8700209F
:10CE4000FBE71CB56946FFF757FF00B1FFDF6846F7
:10CE500001F0C8FBF94900208968A1F8C2001CBD97
:10CE60002DE9FC4104460E46062002F017FA05465D
:10CE7000072002F013FA2844C7B20025A8463E4412
:10CE800017E02088401C80B22080B04202D3404688
:10CE9000A4F8008080B2B84204D3B04202D200208D
:10CEA000BDE8FC816946FFF727FF0028F8D06D1C1C
:10CEB000EDB2AE42E5D84FF6FF7020801220EFE7CA
:10CEC00038B54FF6FF70ADF800000DE00621BDF853
:10CED000000002F04BFA04460721BDF8000002F002
:10CEE00045FA0CB100B1FFDF00216846FFF7B8FF3B
:10CEF0000028EBD038BD2DE9F047D1A10F79D1F84A
:10CF0000008006F09FFD0EF007F8CF4C4FF00409AB
:10CF10001020A4F8389060874FF6FF76A4F854608C
:10CF2000A4F85660002584F8315004F82E5BC649F9
:10CF30002570A5713E39A573C1F87B8081F87F709B
:10CF40007B31481E0BF040FB25751B20E0824FF41F
:10CF5000A47121836083A1830321A17784F81F90AA
:10CF600020846084B848A1843E3805704680B34868
:10CF70000C300570B448103805704680BDE8F08765
:10CF800070B5AE4C0D466060217006F0D5FCFFF721
:10CF900097FFFFF7B0FF207808F035FF07F004FD9A
:10CFA000217860680BF02FFA20780DF02DFB2846D1
:10CFB00009F08EFF06F028FE217860680CF019FC5D
:10CFC000BDE870400DF0A8BF10B501240AB10020E3
:10CFD00010BD21B1012903D00024204610BD02213B
:10CFE0000FF08FF9F9E72DE9F047040000D1FFDFDA
:10CFF000954D002695F8310058B1667014202070C8
:10D0000095F83200A07095F83300E07085F8316033
:10D0100068E0287840B12C22A91C204610F03CFF83
:10D020000F2020702E705DE095F82E0060B1012079
:10D03000E07095F82F00A07095F830006070102017
:10D04000207085F82E604DE07F48022156308246E0
:10D05000FFF706FF00B1FFDFB5F85690062002F09B
:10D060001DF90746072002F019F93844C7B2781CA9
:10D0700000F0FF08B5F85600B84212D1204607F07C
:10D0800031FB50BB95F8340070B3667012202070ED
:10D090002021A01C10F077FF0220A07085F83460DA
:10D0A00020E040451AD1204606F072FDE0B120781C
:10D0B000122817D1A0783C2814D1A088072102F0AB
:10D0C00043F9050000D1FFDF288806F04DFCA08859
:10D0D000072102F04BF900B1FFDF03E02146FFF723
:10D0E00021FE08B1012049E702215046FFF7B8FEB2
:10D0F00018B9B5F856104945BCD100203EE772E793
:10D1000010B5514C207828B10A21BDE810400F20FD
:10D1100001F000BAFFF7C6FD08B10C2002E00DF0E7
:10D1200041FF00202071012060710A21E170207010
:10D1300010BD70B5444D0446287828B1BDE8704054
:10D1400032210F2001F0E6B9207818B1012801D072
:10D15000122010E001F0EBF920B10EF06EF808B1EA
:10D160000C2008E0207801F0CAF904F11703E21D51
:10D17000611C0DF06FFF2871012068713221E97088
:10D18000287070BD70B5304C0546207828B1BDE8D8
:10D1900070400B210F2001F0BDB9287818B101288B
:10D1A00001D012200EE0FFF77DFD08B10C2009E050
:10D1B000287801F0A4F9691C0DF0BBFE08B100202D
:10D1C00000E007202071012060710B21E1702070C8
:10D1D00070BD10B51C4C217829B13021BDE810403C
:10D1E0000F2001F097B900880EF02AF8302110B115
:10D1F0000020207100E0217101206071E170207039
:10D2000010BD70B5104C0546207828B1BDE87040BF
:10D2100031210F2001F07EB901F089F908B10C200D
:10D2200005E0287800F001000EF004F800202071DD
:10D23000012060713121E170207070BD5400002028
:10D24000FFFFFFFF1F0000006A06002010B5FE4C24
:10D25000207828B13421BDE810400F2001F05AB9E0
:10D2600001F065F920B10DF0E8FF08B10C2002E0F3
:10D270000DF047FF00202071012060713421E17022
:10D28000207010BDF048017819B10F21084601F057
:10D2900041B9002101710F218170C170FF2181719D
:10D2A0004FF6FF710181E94949680A7882728A88DC
:10D2B00082814988C181012141710170704710B597
:10D2C000E14C207828B12B21BDE810400F2001F05F
:10D2D00021B90821A01D04F0A5FF00202071012024
:10D2E00060712B21E170207010BD70B5D64C217893
:10D2F00029B1BDE870403F210F2001F00BB990F932
:10D300000000042816D0032814D098B1011D11D0B4
:10D3100010F1080F0ED010F10C0F0BD010F1100F00
:10D3200008D010F1140F05D010F1280F02D01220F0
:10D33000207103E0002505F0A1FD25713F20E0707C
:10D3400001206071207078E710B5BF4C217829B1B9
:10D350002A21BDE810400F2001F0DCB8A31D0122F6
:10D3600000F110010EF031FD002020710F20A0709F
:10D370002A20E07001206071207010BD70B5B24CA1
:10D380000546207828B1BDE8704042210F2001F009
:10D39000C1B808F0F0FF052804D0284608F020FDA9
:10D3A000002000E00C202071012060714221E1701A
:10D3B000207042E770B5A44C0546207828B1BDE83E
:10D3C000704050210F2001F0A5B808F08CFD80B10D
:10D3D0000AF087F868B12878012800D000200DF005
:10D3E0001EF900202071012060715021E170207031
:10D3F00023E70C20F6E770B5934C0546207828B15A
:10D40000BDE8704040210F2001F084B801F08FF892
:10D4100038B10C202071012060714021E170207032
:10D420000BE72946002006F00EFB0020F2E770B55E
:10D43000854C0546207828B1BDE870403E210F207C
:10D4400001F068B808F04FFD50B10AF04AF838B161
:10D45000287809F061FD287807F0A3FC002000E09F
:10D460000C202071012060713E21E1702070E4E603
:10D4700070B5754C0546207828B1BDE8704017217D
:10D480000F2001F047B801F052F838B10C2020719C
:10D49000012060711721E1702070CEE6294601203D
:10D4A00006F0D1FA0020F2E738B5674D0446287837
:10D4B00028B1BDE8384049210F2001F02BB8A079F0
:10D4C000E179884213D021791F2910D861791F2969
:10D4D0000DD8002211460FF0F1FF40B90022E0798B
:10D4E00011460FF0EBFF10B9207A072801D912205E
:10D4F00012E04FF6FF70ADF8000009F0FFFF90B9A1
:10D5000008F039FF78B900216846FFF7A9FC50B14F
:10D51000204605F0AFFB00202871012068714921E9
:10D52000E970287038BD0C20F6E72DE9FC47464C21
:10D53000054694F82E0020B12821102000F0EAFFC3
:10D540007BE4282084F83000012184F82E10A8788C
:10D550004FF000091A2825D00EDC162831D2DFE85A
:10D5600000F030303030302130303030303030303A
:10D5700030303030302121212A2822D00BDCA0F19C
:10D580001E000C281DD2DFE800F01C1C1C1C1C1CFB
:10D590001C1C1C1C1C0D3A38042812D2DFE800F0B9
:10D5A000110211022888B0F5706F0AD21F20884638
:10D5B00084F82F0028886946FFF79EFB18B10220E7
:10D5C00019E0122017E09DF80000019F002806D006
:10D5D00007F5AF77019E05D106F1DD0604E007F1FE
:10D5E000DC07F7E706F25F166846FFF771FB08B144
:10D5F000387818B10C2084F82F001EE487F80080DA
:10D60000A878307084F82F90684600F0EBFF14E49F
:10D610007CB50D4C0546207820B125210F2000F067
:10D6200079FF7CBD28886946FFF766FB0200064843
:10D630004FF00001A0F13E0012D00222227140F80A
:10D64000461F0171E18003E06A06002054000020BB
:10D650000F20A0702520E0700120607120707CBD3B
:10D66000019A134612F1500282F83E109E68C0F8EB
:10D6700046601E7B80F84A6092F83E60002EF3D12F
:10D680002888E080DFE710B540B10478406813B126
:10D69000B0F8480003E0B0F84A0000E0FB201B2986
:10D6A00008D3814206D8B2F5A47F03D340F64800E0
:10D6B000824201D9122010BD002010BD2DE9FC418D
:10D6C000FE4D0446287828B1BDE8FC414C210F20CE
:10D6D00000F020BF4FF0010885F805801F21297157
:10D6E0000F21A9704C21E9702188E98085F800801C
:10D6F00020886946FFF700FB08B102200DE022896F
:10D70000E18801236846FFF7BEFF30B9A28861882F
:10D7100000236846FFF7B7FF10B12871BDE8FC8110
:10D720009DF800103A20019E002749B186F88181BA
:10D73000019991F8BC1106F5C076C1B1287114E0C9
:10D7400086F8F180019991F81011F0360029F5D191
:10D750002F71E08870802089B0806088F080A08878
:10D76000308101980122416A0DE07770D6E72F7170
:10D77000E08870802089B0806088F080A088308147
:10D7800001980022416A30460EF033FC86F8008092
:10D79000EBE770B5C94D044686B0287830B106B0C5
:10D7A0004D21BDE870400F2000F0B4BE012068712B
:10D7B00000262E710F21A9704D21E9702870208854
:10D7C00003A9FFF799FA18B10220287106B034E5D1
:10D7D0009DF80C0040B100220498E188B0F8483070
:10D7E000994203D9C91A02E00122F5E70021E98034
:10D7F0006388B0F84A108B4201D9591A00E0002121
:10D800002981009601960296E188ADF802102189DF
:10D81000ADF804106188ADF80610A188ADF80810C5
:10D82000416A68460EF0E5FB2089BDF80410401AF5
:10D830006881A088BDF80810401AA881E088BDF86A
:10D840000210401AE988884200DC0846E8806088B7
:10D85000BDF80610401A2989884200DC0846288154
:10D86000B4E72DE9F041954C0546207828B1BDE894
:10D87000F0411D210F2000F04DBE1F20207101201E
:10D8800060711D21E170207008F075FD0C260428E0
:10D890003CD005283AD0A9791220012904D019B129
:10D8A000022901D0032926D1297809B1012922D1E1
:10D8B000E97929B1012903D0022901D003291AD11C
:10D8C000698843F6FD720B1F3020934213D2AB8858
:10D8D0001B1F93420FD22187A88860870027A87951
:10D8E00007F099F990B1E87907F0ECF92878012868
:10D8F00004D030B10CE02071BDE8F081002102209D
:10D9000001E00021012007F00CFA08B12671F3E7CD
:10D910002771F1E770B5694C217829B1BDE87040F5
:10D920001E210F2000F0F6BD1F2121710121617120
:10D930001E22E270217002781221012A00D01AB949
:10D94000407818B1012801D0217176E400260C2519
:10D95000012A08D008F00FFD052802D008F09DF933
:10D9600040B1257169E407F06DF9618F208F08F0EF
:10D97000C7FAF5E7267160E42DE9F0474F4F80467E
:10D98000B0F84A00B7F8445092460E46854200D39C
:10D99000054600F0BBFD0446B7F84600A04200D2A1
:10D9A0000446B7F84800B8F84810B946884200D392
:10D9B00008460746084600F0A9FDB9F84A1081421A
:10D9C00000D208464FF4A4711B2F01D0884203D126
:10D9D0001B2D0DD08C420BD0F58034817780B08028
:10D9E00052463046D8F824100EF003FB0120307068
:10D9F000BDE8F0872DE9F04F85B00546AFF2C07164
:10DA00002E4ED1E9009196F82E00884630B12121A2
:10DA1000102000F07FFD05B0BDE8F08F1F2086F8D4
:10DA20002F00212086F830004FF0010B86F82EB031
:10DA3000284600F0E6FD002811D108F09CFC0528DE
:10DA40000CD008F098FC042808D096F8340028B9C7
:10DA500006F0BCFEA0F57F41FF3901D00C20C8E0E4
:10DA6000164801AA3E380190154802901348062135
:10DA70001038039004A801F037FC04007ED0032185
:10DA80000DF0D1FFB6F84E00A4F84800B6F85000EB
:10DA9000A4F84A0096F84D00009096F84C30B6F87D
:10DAA0005020B6F84E10208801F0E2FC00B1FFDFF4
:10DAB000208805F058FF218804E000006A06002055
:10DAC0006000002004F10D0000F040FDFCA004F116
:10DAD0001107006800900321684604F02EFB002027
:10DAE00069460A5C3A54401CC0B20328F9D3288A1C
:10DAF0006080688AA080A88AE080B6F8520008F0AA
:10DB00006FFA0146A062204608F074FA4FF0000A4E
:10DB100084F856A084F857A05746687900F0EFFCC7
:10DB20006076D5F80600C4F81A006889E083C4F866
:10DB3000089084F80C8084F8ECB0012204F1F00124
:10DB40002046FFF719FF8DF800700121684604F0A8
:10DB5000F4FA9DF8000000F00701C0F3C10211447F
:10DB6000C0F3401008448DF80000401D20760928BD
:10DB700001D2083020760021204600E00FE00DF0B1
:10DB800052FF287B07F047F858B107F05BF8697936
:10DB90002879AA1D07F0A1F807000ED01AE0092085
:10DBA00027E0208805F0E0FE2088062101F0DEFB5A
:10DBB00000283FF453AFFFDF50E72146032007F072
:10DBC000B0F8070006D16A882988204608F047F98E
:10DBD00007000BD0208805F0C7FE2088062101F041
:10DBE000C5FB00B1FFDF86F82F7014E7504684F8BC
:10DBF000E0A086F82F000EE738B5B24C207820B1AF
:10DC000022210F2000F086FC38BD1F202071012545
:10DC100065712220E070257094F8340010BB08F084
:10DC2000AAFB052805D006F0D1FDA0F57F41FF39FC
:10DC300018D000202071684608F0A4F90028E3D12C
:10DC40000098008805F090FE00980621008801F0F9
:10DC50008DFB00B1FFDF9C4884F834500078FCF75E
:10DC60002DFA38BD0C20207138BD2DE9F041954DBD
:10DC7000044695F82E0028B1BDE8F041232110207C
:10DC800000F048BC1F2085F82F00232085F83000C5
:10DC9000012085F82E00618840F67B438A1F3020E2
:10DCA0009A4251D2A288961F9E424DD291424BD8A1
:10DCB000E188B1F5FA7F47D2218940F67746A1F194
:10DCC0000A03B34240D2B1EBD20F3DD96189A28998
:10DCD000914239D84FF000082088062101F034FB2A
:10DCE00006004FF0020707D000F06EFC20B1D6F816
:10DCF000E400017839B902E085F82F70FCE5D6F828
:10DD00001C11097809B13A201EE005218171D6F86D
:10DD1000E4004146A0F80880D6F8E420A0885081AD
:10DD2000D6F8E420E0889081D6F8E4202089D081DC
:10DD3000D6F8E400028943899A4204D88279082AF5
:10DD400001D89A4203D3122085F82F00D4E5228807
:10DD50004280D6F8E400077085F82F10CCE5FEB5B8
:10DD6000584C0646207820B124210F2000F0D2FB29
:10DD7000FEBD012565712420E070257030460DF050
:10DD8000BFFF08B1002000E0122020710028EFD171
:10DD90004C4884F83C503E38316840F87B1F31795C
:10DDA0000171002684F83C606946062001F057FAAC
:10DDB00000B1FFDF684601F030FA60B9BDF80470C9
:10DDC000029880F8EC50684601F027FA18B9BDF8BF
:10DDD0000400B842F4D12671FEBD2DE9F041394D61
:10DDE000064695F82E0028B1BDE8F0412C21102000
:10DDF00000F090BB1F2085F82F002C2085F8300004
:10DE0000012085F82E003088062101F09DFA0400DB
:10DE100007D000F0D9FB20B1D4F8E410087830B96D
:10DE200001E0022026E0D4F81C01007808B13A2075
:10DE300020E08C200027005D10F0010F19D0D6F8EB
:10DE400002004860D6F80600886054F8E40F718933
:10DE500010228181206806F10C010E3010F01CF8B0
:10DE600021680320087021683088488085F82F7069
:10DE700042E50C2085F82F003EE52DE9F041114DDB
:10DE800004460C26287828B1BDE8F04118210F205F
:10DE900000F040BB09F032FB012788BB6179032900
:10DEA00034D8A079012831D8A07B03282ED8607BF4
:10DEB00060B307282AD822792020052A26D205E037
:10DEC000112233006A06002054000020DFE802F02F
:10DED000040D03030400A0202288824216D3608828
:10DEE000824213D8B0F5804F10D8084605F0F7FEEF
:10DEF00030B1207985F83600204605F05AFF0646F5
:10DF00002E716F711820E8702F70F5E41226F7E774
:10DF100010B5FE4C217829B11A21BDE810400F2020
:10DF200000F0F8BA01781F2902D91220207106E00A
:10DF3000002121710278411C104605F0A5FF012047
:10DF400060711A21E170207010BD10B5EF4C21787E
:10DF500029B12021BDE810400F2000F0DBBA017884
:10DF60001F2902D91220207106E0002121710278B8
:10DF7000411C104605F077FF012060712021E170FF
:10DF8000207010BD2DE9FC41E04C217829B1BDE89D
:10DF9000FC411B210F2000F0BDBA012767710C2145
:10DFA000217100780026012804D0002860D01220BA
:10DFB00020716EE005F05DFE00286AD009F09EFA3F
:10DFC000002866D105F09EFE94F8360050B1012875
:10DFD00008D0042806D0002008F0A1FF00B1FFDF20
:10DFE000267156E005F006FEA0F57F41FF3950D1BD
:10DFF0000022072101A801F077F9050049D0C448A3
:10E000000321856028460DF0DBFB284606F073F8F7
:10E01000B4F84E00A5F84800B4F85000A5F84A003E
:10E02000B4F852004C3409F086F80146A862002288
:10E03000284608F064FA6078009014F8043B2888B9
:10E0400034F8022934F84E1901F012FA00B1FFDF5A
:10E05000288805F088FC284608F061FF00B1FFDF42
:10E060002671002205F5C0712846FFF785FC10E0F7
:10E0700008F042FA054608F08AFE50B9267145B10B
:10E08000288805F071FC2888072101F06FF900B19C
:10E09000FFDF1B20E0702770BDE8FC812DE9F04117
:10E0A0009A4C0646207828B1BDE8F0412D210F207A
:10E0B00000F030BA3088072101F046F905004FF032
:10E0C000010720D095F8610140B995F85C0011284E
:10E0D00001D0122802D195F89E0150B10C20207178
:10E0E0000F20A0702D20E0703088E08067712770CD
:10E0F0000DE41022B11C05F5B1700FF0CDFE85F8CE
:10E1000061710020EBE70220E9E770B57F4C05461E
:10E11000207828B1BDE870402E210F2000F0FAB918
:10E120002888072101F010F9022178B190F86121C7
:10E130002AB990F85C20112A04D0122A02D00C20AF
:10E14000207104E080F861110020F9E721710F20AF
:10E15000A0702E20E0702888E0800120607120707F
:10E1600009E42DE9FC47694C0646207828B138219E
:10E170000F2000F0CFF9BDE8FC8770884BF68032A5
:10E18000122190420AD848B14FF000083088694601
:10E19000FEF7B2FD20B10220207110E021710EE0E7
:10E1A000019800F15009851C2F887288394648462D
:10E1B0000DF0D4FA2888B842F6D184F80480012002
:10E1C00060713821E1702070D5E77CB54F4C054671
:10E1D000207820B145210F2000F09CF97CBD2888D3
:10E1E0006946FEF789FD38B1022020710120607177
:10E1F0004521E17020707CBD01987F22014680F8A6
:10E20000582080F85920002280F85A20A87801F878
:10E210002C0FE8784870287988702271E6E71CB5E1
:10E220003A4C217821B151210F2000F073F91CBD27
:10E2300000886946FEF760FD48B102202071012088
:10E2400060715121E1700F21A17020701CBD0198F7
:10E2500090F8690000B1012000212171A071EEE762
:10E260001CB52A4C217821B113210F2000F052F95E
:10E270001CBD00886946FEF73FFD08B1022005E09D
:10E28000019890F82C10012902D00C20207106E092
:10E29000582100222271095C21720088E08001204F
:10E2A00060711321E1700F21A17020701CBD2DE958
:10E2B000F041164C0546207828B1BDE8F0414621D2
:10E2C0000F2000F027B92888072101F03DF801232D
:10E2D000D8B182886D88C688418803EB4207BD4269
:10E2E0001DD342F210777E43BF107943B6FBF1F1A4
:10E2F000491E89B24FF4FA76B14200D931468D42B7
:10E3000000D22946491C521C04E014E06A06002091
:10E3100054000020B1FBF2F15143491E8AB290F83B
:10E320008A1101B90284E2800020207163714620C5
:10E33000E0702370E2E40220F7E770B5D44C0546A4
:10E34000207828B1BDE8704048210F2000F0E2B8E5
:10E350002888072100F0F8FF90B1A97811F0010199
:10E3600080F8CF1004D090F8CD1009B108F0EDFE80
:10E3700000202071012060714821E1702070EFE6DB
:10E380000220F6E7C2490A781AB14E210F2000F0A8
:10E39000C1B802789AB142788AB142881B2A0ED35A
:10E3A00082881B2A0BD3C288022A08D3B84A036882
:10E3B000423242F80A3F40685060002000E01220DC
:10E3C0000871012048714E22CA700870704770B5FC
:10E3D000AF4C0546207828B1BDE870404F210F2092
:10E3E00000F098B8287800F0010007F0F6FD2878D2
:10E3F00000F0010008F06BFE002020710120607128
:10E400004F21E1702070ABE670B5A14C0546207835
:10E4100028B1BDE8704052210F2000F07BB8688819
:10E4200007F0DEFD0646688808F085FE864200D3C8
:10E43000304629880023C900503189B20122E631D3
:10E44000884206D901F19602401AB0FBF2F0401C56
:10E4500082B2E2800120237160715221E17020704C
:10E460007EE670B58A4D0446287828B1BDE8704034
:10E470004A210F2000F04EB800F059F808B10C20E6
:10E480000DE0601C0DF014F8207800F0010005F09C
:10E4900035FC207800F0010006F0D0FB0020287148
:10E4A000012068714A21E970287059E670B5784CEE
:10E4B0000546207828B1BDE8704047210F2000F0C4
:10E4C00029B809F01BF808B10C2003E0287805F002
:10E4D000EBFC00202071012060714721E170207069
:10E4E0003EE610B50178532907D26A4A52F8211046
:10E4F00019B1801C8847012010BD002010BD18B143
:10E50000022801D00120704700207047C000703001
:10E5100080B270475E4A92F83130002B06D182F803
:10E52000320082F83310012082F83100704710B5B4
:10E5300007F021FF042807D007F01DFF052803D0AE
:10E5400008F0DCFF002800D0012010BD2DE9FE43BB
:10E5500000250F4680460A260421404603F062FE4D
:10E5600040460DF09EFB062000F098FE044616E0A3
:10E570006946062000F073FE0BE000BFBDF8040002
:10E58000B84206D00298042241460D300FF058FCE4
:10E5900050B1684600F041FE0500EFD0641E002C2B
:10E5A00006DD002DE4D005E040460DF083FBF5E7E5
:10E5B00005B9FFDFD8F800000DF0DAF8761E01D0BB
:10E5C0000028C9D0BDE8FE8390F8691041B990F8E1
:10E5D000C01029B190F8C000042801D00120704774
:10E5E00000207047017801290AD1416891F8CD20B7
:10E5F000002A05D0002281F8CD20406808F0A5BD92
:10E60000704710B5038843F6FD711A1F8A4223D262
:10E610004288141F8C421FD29A421DD8C28940F6EC
:10E620007B43911F994217D2018A8C1F9C4213D2BF
:10E630008A4211D8428AB2F5FA7F0DD2828A40F618
:10E640007744A2F10A03A34206D2B2EBD10F03D959
:10E65000C18A028B914201D9302010BD017911B1DC
:10E66000012910D107E0417929B1012903D00229FC
:10E6700001D0032907D1007B38B1012805D0022839
:10E6800003D0032801D0122010BD002010BD0000CF
:10E690006A06002000E4010020B100234360021D4F
:10E6A00001810260081D7047026800212AB1938829
:10E6B0001268194489B2002AF9D100234360021D6F
:10E6C00001810260704730B4026800230AB3026817
:10E6D00093888B421EBF1368002B1046F7D1B2F807
:10E6E00004C013468C4508BF116811D001F108041D
:10E6F000A5B20024AC4538BF00230AD3ACEB010C13
:10E7000011440C60A1F804C00268126802600A603B
:10E71000016030BC1846704700230B608A80026895
:10E720000A6001607047000008440830424301F16C
:10E730004A00104480B27047F0B51D460446A81840
:10E74000059B083000FB03F205F14A00104486B235
:10E75000B14238BFFFDF002727606760A760E7602E
:10E7600027616761A761E76127624FF6FF70676203
:10E77000A082A6F1280080B265776080B0F5004FD6
:10E7800088BFFFDF608805F13C01884238BFFFDFAA
:10E790006088401B3C3880B220801B2838BF1B207B
:10E7A0002080A777F0BD8161886170472DE9F04F27
:10E7B0000D46C188044600F12808008921F4004371
:10E7C00020F4004221F4004620F400474FF0010AF3
:10E7D0004FF000099A4208D100F4004001F40041D2
:10E7E00088421CBF0020BDE8F08FB7420BD9617F83
:10E7F000B81B401A083885421BDC08EB06000021D4
:10E80000058041801EE06088617F801B401AB0F166
:10E81000080B0ED4BBF11B0FB8BFFFDF5D45D4BFA3
:10E8200029461FFA8BF1681A0204120C18BFBA426B
:10E8300004DD84F817900020BDE8F08F08EB060097
:10E840000180428084F817A0BDE8F08F2DE9F041E7
:10E85000044600F12802C08820F40043E07D00282F
:10E8600008BFBDE8F081D0180288438813448B426A
:10E870003CBF0020BDE8F081002791429CBF018091
:10E88000478013D9891A0D042D0C45800ED0E088DD
:10E89000A61D20F40040854288BFFFDF30884FF47A
:10E8A000004121EA0000284330800AE0627F0088AE
:10E8B00002F108031044083081B26288A01D00F004
:10E8C000A8FBE7750120BDE8F08130B4B0F804C0C2
:10E8D000C488034600F128052CF400402844A445D0
:10E8E00003D10020188230BC7047B3F80CC00488F4
:10E8F000A44509D34088ACEB040CA0EB0C0084B217
:10E900000CEB0500C01E06E0A4EB0C045D7FA4B276
:10E91000AC446044401DB1F800C0A44588BF0C80E1
:10E92000B3F80CC0BCF1000F0CBF4FF0010C4FF05E
:10E93000000C82F800C00988198230BC70472DE9AC
:10E94000F041044600F12801808820F40040451879
:10E95000208A002808BFBDE8F081A08910B9A0690D
:10E96000807F2871A089218A084480B2A0812988EB
:10E970006A881144814238BFFFDF28886D88A289E8
:10E980004119002791421AD175B1A088261D20F4A3
:10E990000040A84238BFFFDF30884FF4004121EA31
:10E9A00000002843308009E0627F1044083081B2C3
:10E9B00002F108036288201D00F02BFBA78127824B
:10E9C0000120BDE8F0812DE9F0474189B0F80480CD
:10E9D0000027044600F1280A414518BF4FF40049BA
:10E9E0003AD000BF21F40040504446886EB160899F
:10E9F00004F10A0520F40040B04238BFFFDF288848
:10EA000029EA00003043288021E0637F008803F179
:10EA1000080C18446389083023F4004562882844B0
:10EA200080B204F10A0190420BD2121A92B20CF198
:10EA30001B0C62452CBF03F4004229EA030004D2F8
:10EA400004E0801A80B229EA030210430880781C8F
:10EA5000618987B24145C5D13846BDE8F0872DE9C7
:10EA6000F047B0F808800B46044600F12801B0F8E2
:10EA70000A90808828F4004C01EB0C05804504BF07
:10EA80000020BDE8F087002A1CBF681D106023B17C
:10EA9000627F691D18460FF0FFF92F886D888DB1D0
:10EAA000E81987B2208904F1080620F40040A84242
:10EAB00038BFFFDF30884FF4004121EA00002843CF
:10EAC00030800AE0607F6288C119083100F10803D4
:10EAD00089B204F1080000F09CFAC84504BF2089FF
:10EAE00060813846BDE8F0878188C08881420CBFCC
:10EAF0000120002070470189808881420CBF0120DD
:10EB00000020704730B48488C28800F1280324F4C0
:10EB1000004C22F40041634494421BD08289048A51
:10EB200015191C885A88A3189D4216D312B18A421F
:10EB300010D212E0437F0CF1080C1A19624440888D
:10EB400092B2801A80B22333984201D211B104E00C
:10EB50008A4202D130BC0020704730BC012070478F
:10EB60002DE9F007B0F806C0048900F12807024635
:10EB70002CF400457E1924F400492CF4004A0020AE
:10EB800024F400434FF00108D1450AD104F40044B5
:10EB90000CF4004C644504D05082BDE8F00700201E
:10EBA0007047AB4208D992F81DC05B1BA3EB0C0366
:10EBB000A3F10804002308E0B2F802C0547FACEBD4
:10EBC000050CACEB040CACF10804002CE4DBB2F84F
:10EBD0000EC0BCF1000F0DD0B6F800C075884DB165
:10EBE0005B1B10778B42D7DBD0893844A0EB0C003D
:10EBF000C01E09E0A4EB0C0410778C4208DB507FA8
:10EC0000D38918443044401D5182BDE8F007704755
:10EC10008B42A8BF82F81C80E6DABDE72DE9F05FE1
:10EC2000044600F1280AC088934620F400400AEB0D
:10EC30000005608A894608B1484502D20020BDE837
:10EC4000F09FE08980B1B5F800806E8808EB06017E
:10EC5000884218BFFFDF207F4FF0000750EA06010F
:10EC600008D0002840D04AE04FF00008A17F464677
:10EC70002971F0E7E08948B1617F01444819B4F88F
:10EC80001F10A0F8051094F82110C171E18908EB5C
:10EC900009004944E18128806F80BBF1000F19D041
:10ECA000607F298800F108030144083189B2628835
:10ECB000A01D00F0AEF9E781A07F401CA077A07DE9
:10ECC00000281CBFE088A082A7756782E775012035
:10ECD000BDE8F09F607FE18908442844B0F8051042
:10ECE000A4F81F10C0792EE0E089B4F81F1050443A
:10ECF000A0EB080020F8031D94F82110817006EBAA
:10ED0000090086B2E089BBF1000F4844E081A5F814
:10ED100000806E800ED0E088A51D20F40040B04237
:10ED200038BFFFDF28884FF4004121EA000030435C
:10ED30002880C0E7E0895044A0EB080030F8031DAC
:10ED4000A4F81F10807884F82100BEE7818800F1C4
:10ED5000280221F4004C6244B0F814C0C388614515
:10ED600018BF99420FD0818969B9806968B101895A
:10ED70008388994209D021F4004128300844117950
:10ED80000079884201D1002070471046704700F199
:10ED90002803407F01F1050C6044106008880028BA
:10EDA00004BFD81E106008884988084480B27047A4
:10EDB0002DE9F04115460A4600F128061C46407F21
:10EDC000531D034410885788069900281CBFC01C97
:10EDD00080B226D088429CBF081A80B213D9401A4C
:10EDE000A042A8BF20461FFA80F85818424629467C
:10EDF0000FF026F8002818BFBDE8F0814544A4EBC9
:10EE0000080084B2002001198F423CBF4FF0FF3050
:10EE1000BDE8F081304422462946BDE8F0410FF0BC
:10EE20000FB8FA1C97B2F61ED4E72DE9F04100F1B5
:10EE300028071D46407F4B1D0344164608880024C2
:10EE4000B1F80280069A00281CBFC01C80B21FD0F7
:10EE500090429CBF101A80B20DD9801AA842A8BF58
:10EE6000284684B29918224630460FF015F8281B20
:10EE700085B2264400204119414506D839182A4652
:10EE800030460FF009F8601984B22046BDE8F081E1
:10EE900008F103011FFA81F8FF1ED9E72DE9F041BF
:10EEA00016460A4600F128071D46407F531D0344BD
:10EEB00010880024B2F80280069900281CBFC01CEC
:10EEC00080B21FD088429CBF081A80B20DD9401A68
:10EED000A842A8BF284684B25818224631460EF0F0
:10EEE000DBFF281B85B2264400204119414506D886
:10EEF00038442A4631460EF0CFFF601984B22046CE
:10EF0000BDE8F08108F103021FFA82F8FF1ED9E77D
:10EF1000401D704770B5044600F12801C288808802
:10EF200020F400431944904208D0A289002A04BF6B
:10EF3000228A002A02D1A28A904201D1002070BD0B
:10EF4000B1F800C04D8885B1261D20F40040A842CC
:10EF500038BFFFDF30884FF4004121EA000028432A
:10EF6000308000202082012070BD607F0CF10801FC
:10EF700000F10803084481B26288201D00F049F8BE
:10EF8000EFE70021C18101774182C175817570472A
:10EF900003881380C289002A04BF00207047C288FA
:10EFA00000F1280322F400421A440A60C089704725
:10EFB00010B50446808AA0F57F41FF3918BFFFDFF6
:10EFC000E088A082E089002818BF0120A07510BD4C
:10EFD0004FF6FF71818200218175704710B504469C
:10EFE000808AA0F57F41FF3908BFFFDFA07D28B9E7
:10EFF000A088A18A884204BF002010BD012010BD56
:10F000008188828A914205BF807D002800200120EE
:10F01000704710B4B0F800C02CF40044214489B209
:10F020004FF4004491420AD2521A92B21B339A42D0
:10F030002CBF0CF4004224EA0C0104D204E0891A2B
:10F0400089B224EA0C021143018010BC704770B5EC
:10F0500016464FF6FC72C91C01EA0205D8B10446F7
:10F06000C01C20F00301A14200D0FFDF201D0121C0
:10F0700008E00246284401D2034600E00023491C70
:10F08000C9B21360B142F4D916B104F1040001E031
:10F090004FF00000206005FB06F000F1040070BD99
:10F0A000024600201168002902D008460968116054
:10F0B000704702680A60016070474FF6FC73C91C14
:10F0C0001940101A001F90FBF1F0C0B270474FF6C4
:10F0D000FC73C91C1940001D01FB020070470000B1
:10F0E0002DE9F041C14D04469046A8780E46A04255
:10F0F00000D8FFDF05EB8607B86A50F8240000B19E
:10F10000FFDFB868FFF7CCFF05000CD0B86A082E07
:10F1100040F8245000D3FFDFB5484246294650F856
:10F120002630204698472846BDE8F0812DE9F04773
:10F130001E460400074602EB060091468A46C5B209
:10F1400027D000218846FF2800D9FFDFE01C20F0EF
:10F150000300A04200D0FFDFB24500D9FFDFA34883
:10F1600080F800A080F801908570C5700571457128
:10F170008671DFF87CA280F8079000260AF1400A29
:10F180008146FF1C27F003000746B8F1000F03D0AB
:10F1900005E04FF00101D5E709EB860188603AF8F8
:10F1A000161019F8062001D04FF00000FFF74FFFAE
:10F1B000761CF6B20744082EE3D3FF1C27F00300A9
:10F1C0002A460646B8F1000F0DD000200221FFF7B5
:10F1D0003EFF4346002130440F46C846C01C20F085
:10F1E00003021BB110E0C9F84800EFE708EB810605
:10F1F0000020B26206E000BFD6F828C04CF82070AC
:10F20000401CC0B2A842F7D3491CC9B202EB85002A
:10F210000829E3D3001BBDE8F08710B5044603F0CE
:10F220007DFB08B1102010BD2078704A618802EB88
:10F23000800092780EE0836A53F8213043B14A1C73
:10F240006280A180806A50F82100A060002010BD7B
:10F25000491C89B28A42EED86180052010BD70B584
:10F2600005460C46084603F059FB08B1102070BD56
:10F27000082D01D3072070BD25700020608070BD6F
:10F280000EB56946FFF7EBFF00B1FFDF6846FFF7F9
:10F29000C4FF08B100200EBD01200EBD10B504460C
:10F2A000082800D3FFDF5148005D10BD3EB505467C
:10F2B00000246946FFF7D3FF18B1FFDF01E0641CAB
:10F2C000E4B26846FFF7A9FF0028F8D02846FFF708
:10F2D000E5FF001BC0B23EBD44498978814201D997
:10F2E000C0B27047FF2070472DE9F04190460C46B0
:10F2F0000546062901D0072C10D13C4FB86CFFF70A
:10F30000CFFE02004FF6FF7604D00221B86CFFF763
:10F31000D4FE00E030462880B04201D1002003E74F
:10F3200042462146FFF7DCFE040002D1288800F0A7
:10F330004FF82046F8E6A0F57F43FF3B01D00829AF
:10F3400001D300207047CBE6A0F57F42FF3A0BD0F7
:10F35000082909D2254A9378834205D902EB810115
:10F36000896A51F820007047002070472DE9F0416C
:10F3700005460C46A5F57F4143F20200FF3902D055
:10F38000082C01D30720CFE618494FF000088A78EF
:10F39000AA42F8D901EB8406B26A52F82570002F10
:10F3A000F1D013483946203050F8242028469047A1
:10F3B000B16A062C41F8258001D0072C02D12846DD
:10F3C00000F006F83946B068FFF773FE0020ABE6A0
:10F3D00010B5064CC2B20221A06CFFF778FE0146C0
:10F3E000A06CBDE81040FFF764BE0000C40600201A
:10F3F0004CE5010070B50E461D46114600F0D5F8EB
:10F4000004462946304600F0D9F82044001D70BD5E
:10F410002DE9F04190460D4604004FF0000610D053
:10F420000027E01C20F00300A04200D0FFDFE5B180
:10F4300041460020FFF730F90C3000EB850617B18C
:10F4400013E00127EDE7624F04F10C00A9003C60D6
:10F450002572606000EB8500206060680EF0B5FDED
:10F46000386841460068FFF717F93046BDE8F0817B
:10F470002DE9FF4F564C804681B020689A4693464E
:10F4800000B9FFDF2068027A424503D9416851F88C
:10F49000280020B143F2020005B0BDE8F08F5146CC
:10F4A000029800F082F886B258460E9900F086F86D
:10F4B00085B27019001D87B22068A14639460068E0
:10F4C000FFF701F904001FD0678025802946201D21
:10F4D0000E9D07465A4601230095FFF72DF9208817
:10F4E000314638440123029ACDF800A0FFF724F9F1
:10F4F0002088C1193846FFF756F9D9F8000041684D
:10F50000002041F82840C7E70420C5E770B5304C1B
:10F510000546206800B9FFDF2068017AA9420ED9AC
:10F52000426852F8251051B1002342F825304A882C
:10F530000068FFF7F1F8216800200A7A08E043F23A
:10F54000020070BD4B6853F8203033B9401CC0B284
:10F550008242F7D80868FFF7A7F8002070BD70B5A1
:10F560001B4E05460024306800B9FFDF3068017A81
:10F57000A94204D9406850F8250000B1041D204676
:10F5800070BD70B5124E05460024306800B9FFDF2B
:10F590003068017AA94206D9406850F8251011B1A7
:10F5A00031F8040B4418204670BD10B50A460121FD
:10F5B000FFF7BAF8C01C20F0030010BD10B50A46D2
:10F5C0000121FFF7B1F8C01C20F0030010BD0000BE
:10F5D0006800002070B5044600780E4601281AD055
:10F5E000072802D00C281AD115E0A06821690578F7
:10F5F0000B2D0CD0052003F027F9052D0FD0782313
:10F6000000220520D4F8101003F07EF807E07823DC
:10F6100000220620F8E70520216903F015F931469C
:10F620002046BDE8704001F0ADB910B500F13902D7
:10F63000C3799478411D64F003042340C371DB0750
:10F640000DD04B79547923404B710B7912791340CB
:10F650000B718278C9788A4200D9817010BD00226E
:10F660004A710A71F5E74178012900D00C21017037
:10F6700070472DE9F74F86B000208C690D468DF854
:10F68000040009780127FA4816464FF0070A4FF0A0
:10F6900011094FF00A0B2A2978D2DFE811F02A006D
:10F6A000110352036903A803B303CC03FA030F0445
:10F6B0003B04620481049A04D504E60405051005A0
:10F6C0003005540577059C05C605E005EE050F06D7
:10F6D0002706300663068506D6060D071B074B076F
:10F6E0006A0779078A07C407FB072708E407E807C2
:10F6F000ED0714B120781D2829D0D5F808805FEADD
:10F70000080043D001208DF80400686A05900320AA
:10F710008DF808008DF809B0286A0390A8880028A1
:10F72000EFD098F8001091B10F2910D27ED2DFE807
:10F7300001F07D144CDCFDFCFBFAF9F8F7089FF6AC
:10F74000F500022822D124B120780C2801D000270E
:10F7500070E302208DF80400ACE10620696A03F032
:10F7600073F8A8880728EDD1204601F006F9022891
:10F7700009D0204601F001F9032808D9204601F0FC
:10F78000FCF8072803D20120207005E011E2002CCC
:10F79000B7D020780128D5D198F80400C11F0A29D4
:10F7A00003D300BF85F81CB089E2A070D8F8001020
:10F7B000A163B8F80410A18798F8060084F83E0009
:10F7C000012028700320207046E00728BAD1002CC1
:10F7D00097D020780D28B5D198F8031094F83B20E5
:10F7E000C1F3C000C2F3C002104201D00E2000E0FD
:10F7F0000F20890707D198F805100142D2D198F857
:10F8000006100142CED194F83D2098F8051020EA68
:10F8100002021142C6D194F83E2098F80610904397
:10F820000142BFD198F80400C11F00E045E20A2957
:10F83000B8D2617F814201D90620C2E3D8F8001016
:10F840006160B8F80410218198F80600A0720120C8
:10F8500028700E20207003208DF80400686A05903F
:10F8600004F139000290601D03901730049067E2A4
:10F87000412890D1204601F080F8042802D1E07898
:10F88000C00704D1204601F078F80F289ED1A88C3B
:10F89000EF6880B24FF0400AD4F82480FFF75FFE93
:10F8A00039460827424653460097FFF7BEFA0E2016
:10F8B0008DF80400686A0590606A0290002101A832
:10F8C000FFF788FE2078042806D0A07F38B10128F1
:10F8D00005D0032806D0AEE3052020700BE284F8A3
:10F8E000009034E71220207066E01128C1D1204634
:10F8F00001F043F8042802D1E078C00719D020466F
:10F9000001F03BF8062805D1E078C00711D1A07FAF
:10F9100002280ED0204601F030F808E0AFE07DE08C
:10F920009AE16EE14EE106E1E5E0CBE01CE0112852
:10F930009FD1102208F1010104F148000EF0ACFA49
:10F94000607801280DD012202070E078C00703D025
:10F95000A07F88B301282FD085F800B08DF804B0BF
:10F96000F0E384F800A027E011288FD1204601F0B1
:10F9700004F8082804D0204600F0FFFF132885D1A2
:10F980002869D8B16869C8B104F17800102208F17B
:10F99000010107460EF080FA2078082812D01420C2
:10F9A0002070E078C0070FD0A07F022818D06178BF
:10F9B000022912D00328CFD10420FDE300208DF8C6
:10F9C0000400F6E00920EBE70B20287029690120EC
:10F9D0004870206CC1E9010792E208B1012870D19A
:10F9E0000B202870296981F801A0606A4860206AAC
:10F9F000C1E9020778E2206CE2780068C2F34402B1
:10FA0000521ED04000F0010040F0800000E00020D5
:10FA10000874E06A48617CE20746F9E31128D0D116
:10FA2000204600F0AAFF0A2802D1E078C00704D1DE
:10FA3000204600F0A2FF1528C3D1102208F10101D1
:10FA400004F148000EF028FA20780A2812D0162077
:10FA500020701220287029690920487004F158008C
:10FA60004860203088601038C860206C0861ACE3C2
:10FA700094E601000B202070E4E22870D9E102280E
:10FA80009FD1204600F079FF042804D3204600F0DF
:10FA900074FF082809D3204600F06FFF0E2890D38A
:10FAA000204600F06AFF12288BD2A07F022888D15E
:10FAB0008DF80490686A059098F801008DF80800A8
:10FAC000FBE36CE20228AAD1204600F056FF002892
:10FAD0006FD0204600F051FF0128F9D0204600F0F9
:10FAE0004CFF0C28F4D005208DF8080098F8010090
:10FAF0008DF8090065E71128FCD1002CFAD0207898
:10FB00001728F7D16178E06A022912D05FF000016E
:10FB100001EB4101182606EBC1011022405808F103
:10FB200001010EF0B9F90520696A00F019FF26708D
:10FB30000DE60121ECE70B28DCD1002CDAD020788F
:10FB40001828D7D16178E06A02292CD05FF0000133
:10FB500001EB4101102202EBC1014158B8F801004C
:10FB600008806078E16A022820D0002000EB400283
:10FB7000142000EBC2000958404650F8032F0A60D9
:10FB8000406848600520696A00F0EAFE6078022853
:10FB900010D04FF000002044407A20F001000CD13A
:10FBA0004FF001010BE04FF00101D1E74FF00100F0
:10FBB000DCE77FE24FF00100EDE74FF00001214468
:10FBC000487279E3112895D1002C93D02078192818
:10FBD00090D16078E16A022811D0002000EB400249
:10FBE0001C2000EBC2001022085808F101010EF0A1
:10FBF00053F90520696A00F0B3FE1A20F5E00120F0
:10FC0000ECE7082898D1002C98D020781A2893D1B6
:10FC1000E06A98F80120017862F347010170E16A17
:10FC2000D8F8022041F8012FB8F806008880052096
:10FC3000696A00F095FE6078022807D04FF0000056
:10FC40002044407A20F002012BD033E04FF0010035
:10FC5000F6E7204441722FE31128B4D1002CB4D030
:10FC600020781B28AFD16178E06A02291CD00021DE
:10FC700001EB4101202202EBC1011022405808F1A2
:10FC800001010EF009F90520696A00F069FE60784B
:10FC900002280CD04FF000002044407A20F00401EC
:10FCA00008D14FF00100D4E74FF00101E0E74FF039
:10FCB0000100F1E74FF00000CBE785F81CA0FAE364
:10FCC0003078012884D11C2204F11C0071680EF0E8
:10FCD00028F9E079C10894F83B0001EAD001E07806
:10FCE00061F30000E070217FF1BB217803290AD085
:10FCF000C0073FF4F9AD032028708DF804B0686A9E
:10FD0000059041209EE3607FA17888423FF694AD44
:10FD100002272771E179204621F0E001E171617A43
:10FD200021F0F0016172A17A21F0F001A172FFF7D8
:10FD30007CFC2F708DF804B0686A05908DF808A0DF
:10FD4000F2E33078112888D18DF804A0696A059112
:10FD5000B1680391ADF808A0084661680160218987
:10FD60008180A17A817100E06AE004202070A4E221
:10FD700030781128A6D18DF804A0686A0590301D4E
:10FD800002AB07C883E807004120ADF80800084629
:10FD90000C210170A88CD6F80C8080B24027D4F8D2
:10FDA0002090FFF7EEFB41464FF008084A463B46DD
:10FDB000CDF80080FFF772F8002101A8FFF70AFCD8
:10FDC000E07820F03E00801CE0702078052801D00B
:10FDD0000F200AE0A07F00283FF4C3AD0128FBD02C
:10FDE00003287DD184F80080B1E42070AFE430783E
:10FDF0000328A8D170680168A1664068E066052004
:10FE0000287035E2317803299DD171680A6822672C
:10FE100049686167216C51B9A17F19B1012901D0ED
:10FE2000062029E185F800A02064606401E085F8DF
:10FE300000A00327F3E33178022984D1317909B195
:10FE4000297737E1A17F022910D00329EFD161780A
:10FE5000012910D0A17994F83A2001290FD020640B
:10FE6000E178C90713D0012A0ED010E0B06800284D
:10FE7000E7D020640BE0A27994F83A10EDE7B1687E
:10FE80000029DED02164EBE7F0680028D9D0606457
:10FE9000CDE78DF804B0696A0591E1785846C90745
:10FEA00009D06178022903D1A17F29B1012903D0AA
:10FEB000A17F032900D00820287012E23078112891
:10FEC000BFD1B068286209202870E0782969C0078E
:10FED0000FD081F801A0206A4860606A886000E065
:10FEE000ABE004F16800C860A07F02287FF48FAD0A
:10FEF00081E501204870206C486004F1680088604A
:10FF000004F13800C860201D0861206B4861606BF7
:10FF100088611FE2E1783078C90701D0062100E04E
:10FF20000A2188428DD12078072817D084F80090C4
:10FF30008DF804A0686A0590286A0390ADF80890CF
:10FF4000032100F8011B102271680DF0A5FF0021AC
:10FF500001A8FFF73FFB00202862C2E408202070C0
:10FF6000E6E730781128ABD18DF804A0686A0590D7
:10FF7000B0680390ADF80890042100F8011B10222E
:10FF800004F168010DF088FF002101A8FFF722FBB2
:10FF90002078092801D0132027E784F800B016E064
:10FFA000E1783078C90701D0062100E00A218842B3
:10FFB00086D1102204F1480071680DF041FF10B1A4
:10FFC00004202877A2E3207809283FF4C5AC0C2050
:10FFD00053E5E078C10735D0A17F012902D002297D
:10FFE0001BD02CE00D202870296981F801B06078C1
:10FFF000012809D0206A4860606A886004F16800BE
:020000040001F9
:10000000C8601030086104E5606A4860206A886052
:1000100004F17800C8601038F4E7C0F344011429F3
:100020000DD24FF0006101EBB0104FEAB060E0700C
:100030006078012801D0102055E40620D5E66078CC
:1000400001288AD00E2018E5307809288BD185F850
:1000500000B010208DF80400686A05907068029066
:10006000002101A8FFF7B6FAE9E7E078C00706D05B
:10007000A07F01281FD10F2028700420F8E0152050
:100080002870296902204870206C48606078012837
:1000900005D004F1780088601038C8605AE104F196
:1000A000680088601030F8E730780228CED13079C7
:1000B00008B1287728E3102028700F20D8E0307886
:1000C0001328F7D185F800902969082048707068D6
:1000D0004860607801280DD004F168008860103015
:1000E000C860206B0861606B486104F1580088614A
:1000F000A06A21E004F1780088601038F0E73078D9
:100100000728D7D1607801281AD1A078A16A0A18E7
:10011000C0F1100110460DF036FF12202870296939
:100120000920487004F15800486020308860103879
:10013000C860206C086141E0C861E06A086209E1BA
:100140001320C9E0CBE030780828B3D1102204F1A5
:10015000480071680DF074FE08B10B2031E720787B
:100160000B28EDD02046FFF760FAA078A16A0A18A4
:10017000C0F1100110460DF006FF1620287008206F
:100180008DF80400686A0590002049E03078112855
:1001900090D1B0682862142028702969092048701D
:1001A00004F158004860103088601030C860606CFE
:1001B00008616078012800E09EE006D004F1390073
:1001C0004861206B8861606BB6E7601D4861606BB9
:1001D0008861206BB0E73078082892D18DF804A0B0
:1001E000686A0590286A0390ADF808900D2100F820
:1001F000011B102271680DF04FFE002101A8FFF7CE
:10020000E9F9002028626178012902D01520ECE587
:1002100069E21621297008218DF80410696A059198
:100220000290A0788DF80C007EE130780B288CD1FC
:10023000162028706078022802D12046FFF7F5F9D1
:10024000A07871680A18C0F1100110460DF09BFEED
:1002500008208DF80400686A05907068E0E730783F
:100260000F2895D1E079C0077BD01720287009208E
:100270008DF80400686A059056E13078102887D11F
:100280001422311D04F11C000DF04BFEE16A208D9B
:10029000A1F80900E16AA078C871E179E26A01F089
:1002A00003011172E16A627A0A73E16AA07A81F845
:1002B00024006078012876D0B3E13EE2607802281D
:1002C00001D0012000E000202044407AC0070BD07C
:1002D000E078C00708D1192028708DF804B0686A4A
:1002E00005908DF808901FE11E2071E630781128E6
:1002F00074D1B06828621A2028700520B8E73078D9
:1003000003286BD16078E26A022801D0012000E066
:10031000002000EB4001142000EBC101515872682D
:1003200013680B6052684A601B212970D5E90412DA
:1003300005234B70636A4B606778E36A022F01D034
:10034000012700E0002707EB470700EBC70018581C
:10035000C1E90202686A4862069800F02AFBFFF7CA
:100360005BBB87E130780E2838D16078E26A0228DA
:1003700001D0012000E0002000EB4000102101EB43
:10038000C00002231058093271680CF06FF91C206C
:100390002870296904204870206A4860E06A0930A2
:1003A0008860FA4879E65AE130780D2816D16178EC
:1003B000E06A022901D0012100E0002101EB4101A6
:1003C000182707EBC101A278405871680DF064FD51
:1003D0006178E06A022902D0012101E0A9E0002150
:1003E00001EB410107EBC1014058A1780844C1F17C
:1003F00010010DF0C8FD8DF804A0686A0590286A08
:100400000390ADF80890062101706278E16A022A33
:1004100001D0012200E0002202EB420207EBC202FF
:10042000401C895810220DF037FD002101A8FFF76C
:10043000D1F8002028621D2028708DF804B0686A69
:1004400005900B208DF808006EE03078112870D1EF
:100450008DF804A0686A0590B06803900B20ADF891
:100460000800039880F800A06278E16A022A01D0AF
:10047000012200E0002202EB4202102303EBC20241
:1004800089580988A0F801106178E26A022901D030
:10049000012100E0002101EB4103142101EBC30124
:1004A00051580A6840F8032F49684160002101A8AB
:1004B000FFF790F818E729E16078022801D00120C1
:1004C00000E000202044407A800701D51F2003E788
:1004D00021207DE5307811282BD18DF804A0686AA1
:1004E0000590B0680390ADF8089008270770617810
:1004F000E26A022901D0012100E0002101EB410361
:100500001C2101EBC301401C515810220DF0C4FC0A
:10051000002101A8FFF75EF8202028708DF804B0B4
:10052000686A05908DF80870314601A8FFF752F807
:1005300015E775E03078112872D18DF804A0686A4B
:100540000590B06803900820ADF8080003980921D1
:100550000170E169097849084170E16951F8012F9A
:10056000C0F802208988C180002101A8FFF732F875
:10057000AEE76078022801D0012100E0002121448B
:10058000497A490701D52220A6E6012849D068E02A
:100590003078112844D1B068286223202870296956
:1005A00004204870206A4860E06A09308860784812
:1005B00073E530780D2833D16178E06A022901D0E3
:1005C000012100E0002101EB4101202707EBC101DF
:1005D0001022405871680DF05FFC8DF804A0686A25
:1005E0000590286A0390ADF8089080F800B0627812
:1005F000E16A022A01D0012200E0002202EB42025D
:1006000007EBC202401C895810220DF045FC002166
:1006100001A8FEF7DFFF002028626078B5E791E0CF
:1006200037E02420D4E4607802280BD00020204456
:10063000407AC10702D0E178C90705D0810705D506
:100640001920A9E40120F2E71720A5E4400701D50D
:100650001B20A1E41C2020706078012801D0182004
:10066000B6E42720B4E4282028700B2000E6307878
:10067000122849D12920ABE42078012844D00C2845
:1006800042D02046FEF7EFFF0C208DF80400686A88
:10069000059039E030784FF02608112805D0122057
:1006A0003070032785F800804CE08DF804A0686A5C
:1006B0000590B06803900220ADF80800039805216A
:1006C0000170297F4170002101A8FEF783FF0B20F4
:1006D0008DF80400686A0590314601A8FEF77AFF9C
:1006E000074685F80080012F0ED02BE001208DF801
:1006F0000400686A059004208DF80800287F8DF8B2
:1007000009000020287712E0287F80B11D2020708A
:10071000252028708DF804B0686A059002208DF8B5
:100720000800314601A8FEF755FF07460AE00CB164
:10073000FE2020709DF8040020B1002101A8FEF7E2
:1007400049FF0AE409B03846BDE8F08F2DE9F04FC3
:1007500085B00C464E69002190468DF804100127A3
:100760002278BA464FF00209072022B1012A51D05F
:10077000022A20D1CAE0217901290BD0022916D002
:10078000032911D0042916D11CE000008CE60100D9
:10079000FE2F0000707801280CD10620616A02F05B
:1007A00029F8002807D11CE01D20307019E071786D
:1007B000022901D0052798E031780C2929D18DF83C
:1007C000040010E0B07F022823D13078011F0429F3
:1007D00004D30A39032901D31D281AD120890228FC
:1007E00017D38DF8049084F800A020899DF8041098
:1007F000884203D20A208DF800003FE0112108341E
:1008000088F8001094E80E00C8E901120327C8F820
:100810000C306AE098F80020112A66D18DF80000AB
:10082000626A0492D8F80850029522794FF00B0BB7
:10083000012A06D0022A29D0032A11D0042A54D131
:1008400059E0ADF8049085F800B0207E4F4600F0E6
:100850001F00687000216846FEF7BCFE377043E059
:10086000ADF8049005202870207E68704E46002167
:100870006846FEF7AFFE26708DF800B0606A0490FF
:1008800041466846FEF7A6FE07462EE0ADF8040096
:1008900085F800A0207F6870607F00F00100A870DC
:1008A000A07F00F01F00E870E27F2A71C0071FD010
:1008B00094F8200000F00F00687194F8210000F017
:1008C0000F00A87100216846FEF784FE2868B06317
:1008D000A888B087A87986F83E00A069407870772C
:1008E0002879B0700D2030700027384605B02BE70E
:1008F000A9716971E6E7ADF804900E202870207E9A
:10090000687000216846FEF765FEEDE7FE20307056
:100910008DF800A0606A049004208DF80400207E09
:100920008DF80500EDE700B50023012285B005280C
:1009300010D006280CD102208DF8002004918DF8EB
:10094000040000BF8DF8053000216846FEF742FE26
:1009500005B000BD8DF8002004918DF80420F1E76A
:1009600070B50C46054601F06FFF21462846BDE8EC
:1009700070407823002201F0C7BE08B100787047AC
:100980000C20704770B50C0005784FF000010CD0BA
:1009900021702146F4F7C9FB74482178405D8842F4
:1009A00001D1032070BD022070BDF4F7BEFB002012
:1009B00070BD027B032A05D000220A704B780B2BF6
:1009C00002D003E0042070470A770A62027B93009A
:1009D000521C0273C15003207047F0B585B00F461A
:1009E00005460124287B05EB800050F8046C7078E4
:1009F000411E0C290AD25D493A46123101EB8000B2
:100A0000314650F8043C2846984704460CB1012C66
:100A100011D1287B401E10F0FF00287301D0032461
:100A2000E0E70D208DF80000706A04900021019627
:100A30006846FFF7A7FF032CD4D005B02046F0BDD1
:100A400070B515460A46044629461046FFF7C5FF0D
:100A5000064674B12078FE280BD1207E30B10020EC
:100A60002870294604F10C00FFF7B7FF2046FEF777
:100A7000FAFD304670BD704770B50E4604468821B9
:100A80000DF0A3FA0225012E03D0022E04D005207A
:100A900070BD0120607000E065702046FEF7E3FD48
:100AA000A577002070BD28B1027E1AB10A4600F178
:100AB0000C01C5E70120704730B5044687B00D46EC
:100AC000062001F0C1FE2946052001F0BDFE207878
:100AD000FE2806D000208DF8000069462046FFF76A
:100AE000E2FF07B030BD7FB50E4600218DF80C1037
:100AF00041780B2903D00C2903D0002405E0846938
:100B000000E044690CB1217E91B16D460146284652
:100B1000FFF74FFF032809D1324629462046FFF749
:100B20008FFF9DF80C10002900D0042004B070BD88
:100B300004F10C05EAE710B590B00C4607900B489D
:100B40000421801E08900A488DF8191009900F9210
:100B5000694606A8FFF7C7FF002805D110222046E6
:100B600001990DF099F9002010B010BD9EE501002B
:100B70008CE6010070B50D46040011D085B121014D
:100B800028460DF000FA10224E4928460DF084F94F
:100B90004C4801210838018044804560002070BD28
:100BA000012070BD70B5474E00240546083E10E098
:100BB0007068AA7B00EB0410817B914208D1C17B55
:100BC000EA7B914204D10C2229460DF039F930B16B
:100BD000641C30888442EBDB4FF0FF3070BD204650
:100BE00070BD70B50D46060006D02DB1FFF7DAFFD7
:100BF000002803DB401C14E0102070BD314C083C81
:100C000020886288411C914201D9042070BD61682E
:100C1000102201EB001031460DF03EF92088401CF7
:100C200020802870002070BD70B514460D0018D0CB
:100C3000BCB10021A170022802D0102811D105E01A
:100C4000288870B10121A170108008E02846FFF7C4
:100C5000A9FF002805DB401CA070A8892080002087
:100C600070BD012070BD70B5054614460E000BD056
:100C700000203070A878012808D005D91149A1F1C9
:100C800008010A8890420AD9012070BD24B1287851
:100C900020702888000A5070022008700FE064B1AC
:100CA0004968102201EB0011204610390DF0F4F8CC
:100CB000287820732888000A607310203070002084
:100CC00070BD0000740000202DE9F04190460C46F4
:100CD00007460025FE48072F00EB881607D2DFE8FD
:100CE00007F00707070704040400012500E0FFDF01
:100CF00006F81470002D13D0F548803000EB880101
:100D000091F82700202803D006EB4000447001E052
:100D100081F8264006EB44022020507081F82740DD
:100D2000BDE8F081F0B51F4614460E460546202A60
:100D300000D1FFDFE649E648803100EB871C0CEB71
:100D4000440001EB8702202E07D00CEB46014078CF
:100D50004B784870184620210AE092F825304078F8
:100D600082F82500F6E701460CEB4100057040785B
:100D7000A142F8D192F82740202C03D00CEB440478
:100D8000637001E082F826300CEB4104202363708D
:100D900082F82710F0BD30B50D46CE4B4419002225
:100DA000181A72EB020100D2FFDFCB48854200DD4A
:100DB000FFDFC9484042854200DAFFDFC548401CDA
:100DC000844207DA002C01DB204630BDC148401CBC
:100DD000201830BDBF48C043FAE710B5044601688B
:100DE000407ABE4A52F82020114450B102200844F3
:100DF00020F07F40F1F7E1FE94F90810BDE81040C3
:100E0000C9E70420F3E72DE9F047B14E803696F8A4
:100E10002D50DFF8BC9206EB850090F8264038E0B4
:100E200009EB85174FF0070817F81400012806D0C2
:100E3000042816D0052816D0062800D0FFDF00F0C1
:100E400056FF07EB44014A7806EB850181F826201E
:100E500091F82720A24202D1202281F8272028B130
:100E600005E0022000E003208046E8E762B62A465B
:100E700021460120FFF728FF9948414600EB041066
:100E800002682046904796F82D5006EB850090F8B2
:100E90002640202CC4D1BDE8F08710B58C4C202111
:100EA000803484F8251084F8261084F82710002058
:100EB00084F8280084F82D0084F82E10411EA160CB
:100EC00044F8100B2074607420736073A07385491C
:100ED000E07720750870487000217D4AB4F1100455
:100EE00002F81100491CC9B22029F9D30120F1F7F9
:100EF00052FD0020F1F74FFD012084F82200F9F7A0
:100F0000AFF87948F9F7BBF8764CA41E2070774803
:100F1000F9F7B5F86070BDE81040F1F7C9BC10B53D
:100F2000F1F7EBFC6F4CA41E2078F9F7C1F860785C
:100F3000F9F7BEF8BDE8104000F003BF202070476D
:100F40002DE9F34F624E0025803606EB810A89B009
:100F50009AF82500202822D0691E02916049009548
:100F600001EB00108146D0E90112C0680391CDE980
:100F70000420B08BADF81C00B07F8DF81E009DF8EA
:100F80001500C8B10227554951F820400399E219CC
:100F9000114421F07F41019184B102210FE0012031
:100FA000F1F7F9FC0020F1F7F6FCF1F7C4FC00F0D2
:100FB000C8FE86F82F508AE00427E4E700218DF868
:100FC0001810022801D001281BD1039839190144B7
:100FD0000998081A20F07F4033280BD903208DF898
:100FE00015000398C4F13201401A20F07F403224EA
:100FF00003900CE096F8240018B901F029F80028B5
:101000004DD0322C03D214B100F08FFE01E000F07D
:1010100098FE344A107820B393465278039B121BF3
:1010200000219DF81840984601281BD0032819D0AC
:101030005FF000008DF81E00002A04DD981A03906E
:1010400001208DF818009DF81C0000B102210398C2
:10105000274A20F07F40039003AB099800F07DFE03
:1010600010B110E00120E5E79DF81D0018B99BF8CC
:101070000000032812D08DF81C50CDF80C808DF89C
:1010800018408DF81E509DF8180058B103980123A0
:10109000C11900221846F1F7D1FC06E000200BB080
:1010A000BDE8F08F0120F1F776FC99F90C200123BF
:1010B00000200199F1F7C2FC012086F82F008AF880
:1010C000285003482022694680300CF02AFF11E0A6
:1010D00010090020FF7F841E0020A107E0E5010029
:1010E0001007002086000020B7250100070E010030
:1010F000FFFF3F000120D2E72DE9F05FDFF88C848D
:10110000064608EB860090F82550202D1FD0A8F148
:1011100080002C4600EB8617A0F50079DFF870B44C
:1011200005E0A24607EB4A004478202C0AD0F1F7EC
:10113000D1FC09EB04135A4601211B1D00F00DFEE2
:101140000028EED0AC4202D0334652461AE0F1F706
:10115000C1FC98F82F206AB1D8F80C20411C891ADC
:101160000902CA1701EB12610912002902DD0020F1
:10117000BDE8F09F3146FFF7E3FE08B10120F7E735
:1011800033462A4620210420FFF7CCFDEFE72DE966
:10119000F041FE4C2569F1F79DFC401B0002C11790
:1011A00000EB1160001200D4FFDF94F8220000B1C0
:1011B000FFDF012784F8227094F82E00202800D148
:1011C000FFDF94F82E60202084F82E00002584F89C
:1011D0002F5084F8205084F82150EE482560007884
:1011E000022833D0032831D000202077A068401C8B
:1011F00005D04FF0FF30A0600120F1F7CCFB0020BC
:10120000F1F7C9FBF1F7C7FCF1F7BFFCF1F793FB6E
:101210000CF0F0F9E048056005604FF0E0214FF474
:101220000040B846C1F88002F1F74FFD94F82D70E8
:101230003846FFF761FF0028FAD0D448803800EB29
:10124000871010F81600022802D006E00120CCE733
:101250003A4631460620FFF737FD84F8238004EB39
:10126000870090F82600202804D0CA48801E4078C5
:10127000F8F724FF207F002803D0F1F77CFC2577C6
:1012800065774DE50146C14810B590F82D20002442
:10129000803800EB821000BF10F814302BB1641CB2
:1012A000E4B2202CF8D3202010BDBC4800EB041081
:1012B000016021460120FFF707FD204610BD10B553
:1012C000012801D0032800D171B3B04A92F82D3023
:1012D000AE4C0022803C04EB831300BF13F8124095
:1012E0000CB1082010BD521CD2B2202AF6D3A94A54
:1012F00048B1022807D0072916D2DFE801F0150609
:10130000080A0C0E100000210AE01B2108E03A2117
:1013100006E0582104E0772102E0962100E0B521A3
:1013200051701070002010BD072010BD994810B5F5
:101330004078F1F742FC80B210BD10B5202811D2E0
:10134000924991F82D30A1F1800202EB831414F838
:1013500010303BB191F82D3002EB831212F81020BF
:10136000012A01D0002010BD91F82D200146002057
:10137000FFF7AAFC012010BD10B5F1F7ABFBBDE8EB
:101380001040F1F71ABCF0B5804F04782025803F5B
:10139000264607EB831303E0254603EB45046478F8
:1013A000944202D0202CF7D108E0202C06D0A6428F
:1013B00006D103EB46025278027007E00020F0BD30
:1013C00003EB440003EB45024078507019B10878F4
:1013D000A04200D10D700120F0BD10B542680B682D
:1013E0009A1A1202D41702EB1462121216D4497A16
:1013F00091B1427A82B96A4A006852F821101268A3
:1014000019441044001D891C081A0002C11700EB82
:1014100011600012322801DB012010BD002010BD38
:101420002DE9F047814659485C4E00EB8100984613
:1014300090F825402020107006F50070154600EB4E
:1014400081170AE006EB04104946001DFFF7C5FFAF
:1014500028B107EB44002C704478202CF2D1297875
:1014600088F8001013E000BF06EB0415291D48465C
:10147000FFF7B3FF68B988F80040A97B99F80A0024
:10148000814201D8002006E507EB44004478202C77
:10149000EAD10120FFE42DE9FC410E460746002475
:1014A0003E4D08E09DF8000005EB001081683846CD
:1014B00000F067FC01246B4601AA31463846FFF76D
:1014C000AFFF0028EED02046BDE8FC8170B5044691
:1014D0002E4801258038A54300EB841100EB8510D0
:1014E00040220CF0D9FC294800EB850100EB840078
:1014F000D0F82500C1F82500284670BD2DE9FC4133
:101500008446224815468038089C00EB85170E4615
:1015100017F81400012803D0022801D00020D3E7D7
:101520000B461B4A0121604600F017FCA0B101AB3D
:101530006A4629463046FFF773FF68B19DF80420DC
:101540009DF8001011488A4200EB850608D02B4612
:101550000520FFF7E7FB0BE02A462146042014E0B4
:10156000202903D007EB4100407801E096F82500E0
:1015700007EB440148709DF80000202816D007EBC7
:10158000400044702A46214603200BE090090020C9
:10159000FFFF3F008600002000F5004010070020FC
:1015A000E0E50100FFF790FB01208DE706F8254FED
:1015B0000120F070E6E7FA4901EB0010001D0CE491
:1015C0007CB51D46134604460E4600F1080221462E
:1015D0001846F1F7FFFA94F908000F2804DD1F38C8
:1015E00020722068401C206096B10220ED4951F81D
:1015F0002610461820686946801B20F07F40206036
:1016000094F908002844C01C1F2803DA012009E0CF
:101610000420EBE701AAF1F7DDFA9DF8040010B110
:101620000098401C00900099206831440844C01C78
:1016300020F07F4060607CBD2DE9FE430C460746EC
:10164000097860799072207998461546507241B1B8
:10165000781D20F07F46D44890F82E00202808D02E
:101660000AE0D4E90223217903B02846BDE8F0431B
:10167000A6E7CE4840780644217900222846A36890
:10168000FFF79EFF3146284600F07BFBD4E902328B
:1016900021796846FFF794FF41462846019CFFF7F1
:1016A000FAFE2B4622460021384600F056FB002861
:1016B00003D13946284600F064FBBDE8FE832DE9DE
:1016C000FE43804600F019FB28B1002798F800007F
:1016D00018B10020F1E70127F8E7B34C4FF00009FB
:1016E00094F82D6084F8239000251FB93046FFF749
:1016F000EDFE0646F1F7EEF933466A464146FFF73E
:101700009BFF94F82E0020280CD021690098401AE5
:101710000002C21700EB1260001203D5684600F009
:1017200030FB012594F823000028D9D1F1F7D2F934
:101730006B469F4A002100F010FB0028BDD027B95E
:1017400031466846FFF7A7FE054325B16846FFF717
:1017500044FBC8F808000120AFE72DE9FF5F8A4687
:10176000814600F0CAFA904C48B19AF80000002770
:1017700010B1012800D0FFDF4FF0010810E094F80D
:101780002E000127202800D1FFDF9AF80000002852
:10179000F2D0FFDFF0E700BFB8F1000F00D162B672
:1017A00094F82D50002084F823003FB92846FFF715
:1017B0008DFE054694F823000028EDD1F1F78AF953
:1017C00006462B4601AA5146FFF736FF3B462A46FE
:1017D00001A93046CDF80090FFF790FE064604EBD5
:1017E000850090F828B000F082FA804694F8230033
:1017F0000028D1D16A490DF1040C01EB09109CE8D5
:101800000E0000F1040080E80E00D6B13BEA0700AC
:101810000CD094F82E00202808D12846FFF76CFC45
:1018200020B99AF8000028B10128B5D0284600F068
:1018300057FA05E094F82D2049460420FFF744FAB2
:101840000126B8F1000F00D162B666B194F82D0000
:1018500004EB800090F82600202804D05348801E16
:101860004078F8F72BFC304604B081E42DE9F05FB6
:101870004D4C814694F82D004FF000080125474655
:1018800005B962B604F8237FA07AFFF71FFE06466B
:1018900014F823090028F3D14348803800EB86115F
:1018A00011F81900032837D1334604EB830A4A465E
:1018B0009AF82500904201D1012000E000208346E3
:1018C0000AF125000021FFF75EFD014610EA0B0F2B
:1018D00003D001228AF82820A777E9B13246494689
:1018E0000120FFF7F1F99AF828A000F000FA054668
:1018F00094F823000028C3D1BAF1000F07D094F860
:101900002E00202803D13046FFF7F6FB20B13046E9
:1019100000F0E6F94FF0010805B962B6404627E449
:101920000020F1F711B80120F1F70EB81F48801E12
:10193000007870472DE9F0411B4C94F82E002028C8
:101940001FD194F82D6004EB860797F82550202DC1
:1019500000D1FFDF1449803901EB861000EB450010
:10196000407807F8250F0120F87084F823002946F5
:1019700084F82E50324602202234FFF7A5F90020C9
:1019800020707EE42DE9F041054E074C012588B119
:1019900001282BD0022874D0032873D0FFDF70E415
:1019A00010070020E0E501009009002086000020DB
:1019B000FFFF3F0000F0B9F9FFF7BCFF207E00B148
:1019C000FFDF84F821500020F0F7E5FFA168481CF4
:1019D00004D0012300221846F1F730F814F82E0F36
:1019E000217806EB01110A68012154E0FFF7A2FFFC
:1019F0000120F0F7D0FF94F8210050B1A068401CFE
:101A000007D014F82E0F217806EB01110A68062181
:101A100041E0207EDFF880830027012803D00228E0
:101A20001ED0FFDF2DE4A777F1F7A5F898F80000A6
:101A3000032801D165772577607DD84951F82000CA
:101A400094F8201051B948B161680123091A0022A5
:101A50001846F0F7F3FF0220207612E4277610E410
:101A600084F8205000F061F9A07F60B198F801007F
:101A700061680123091A00221846F0F7DFFF257676
:101A800002E00BE011E0277614F82E0F217806EB28
:101A900001110A680021BDE8F0411047BE48801ED0
:101AA0000078BDE8F041F8F709BBFFF743FF14F8F1
:101AB0002E0F217806EB01110A680521EBE710B51E
:101AC000B74C94F82E00202800D1FFDF14F82E0F19
:101AD0002178B44A02EB01110A68BDE810400421E4
:101AE00010477CB5AE4C054694F82E00202800D156
:101AF000FFDFA068401C00D0FFDF94F82E00A9494A
:101B000001AA01EB0010694690F90C002844F1F796
:101B100061F89DF904000F2801DD012000E000209C
:101B2000009908446168084420F07F41A16094F85E
:101B30002100002807D002B00123BDE87040002238
:101B40001846F0F77BBF7CBD30B5974A0B1A541C82
:101B5000B3EB940F12D3451AB5EB940F0ED3934207
:101B600003D9101A43185B1C08E0954204D9511A96
:101B70000844401C434201E0FFDF0023184630BD0B
:101B80000123002201460220F0F758BF0220F0F79F
:101B900002BFF0F79FBF2DE9FC47814D044695F841
:101BA0002E00202800D1FFDF642C4AD37F4A002179
:101BB000121B71EB010044D395F82E20A84628464D
:101BC000DFF8E09190F82D7009EB0215D8F80000CD
:101BD00001AA20446946F0F7FDFF9DF904000028A2
:101BE00002DD0098401C0090A96800986A680E18F1
:101BF000B21A22F07F42B2F5800F22D208EB8702A0
:101C0000454692F82520202A07D009EB0212526897
:101C1000511A21F07F41814213D3A868401C05D09E
:101C20000120F0F7B8FE4FF0FF30A860286820448C
:101C3000286026F07F402861012085F82300BDE858
:101C4000FC870020FBE72DE9F041554C074694F84E
:101C50002D00A4F1800606EB801010F8170000B9E3
:101C6000FFDF94F82D5006EB851606E004280CD013
:101C700005280AD0062808D020BF16F8170001282A
:101C8000F4D101254FF0000807E02A46394601202B
:101C9000FFF71AF8F1E705B962B604F8238FA07AC6
:101CA000FFF714FC064614F823090028F3D104EBCF
:101CB000860000F1270133463A462630FFF763FBE2
:101CC00000F015F8054694F823000028E3D184F8C5
:101CD0002D60012084F82300002D00D162B650E66B
:101CE0002F4981F82D00012081F823007047EFF380
:101CF000108000F0010072B670472D480068C005E2
:101D0000C00D10D0103840B2002806DA00F00F00E5
:101D100000F1E02090F8140D03E000F1E02090F8CD
:101D20000004400970470820704710B51C4C94F817
:101D30002400002804D1F7F7AFFF012084F8240025
:101D400010BD10B5164C94F82400002804D0F7F705
:101D5000CCFF002084F8240010BD10B51C685B681F
:101D6000241A181A24F07F4420F07F40A14206D89C
:101D7000B4F5800F03D2904201D8012010BD00209D
:101D800010BDD0E90032D21A21F07F43114421F076
:101D90007F41C0E90031704786000020E0E5010086
:101DA0009009002010070020FF7F841EFF1FA1075D
:101DB00004ED00E0F0B5734AD2F80032724D002411
:101DC00001212E7856B9714E3460704F03263F1DA5
:101DD0003E606E4F04260C373E602970C2F8004208
:101DE000D1601160694C4834D16425688542FBD3C9
:101DF0005160D160C2F80032F0BD2DE9F0410446D7
:101E000080074FF000054FF0010604D560480560DB
:101E1000066024F00204E0044FF0FF3705D55D486A
:101E20004660C0F8087324F48054600003D55A4813
:101E3000056024F08044E0050FD55248C0F80052F8
:101E4000C0F8087351490D60091D0D604F4A042107
:101E50000C321160066124F48074A00409D54F4847
:101E60004660C0F80052C0F808734D48056024F47D
:101E70000054C4F38030C4F3C031884200D0FFDF87
:101E800014F4404F14D047484660C0F808734648E1
:101E90008660C0F80052C0F8087344490D600A1DFE
:101EA00016608660C0F808730D60166024F4404424
:101EB00020050AD53E4846608660C0F80873C0F821
:101EC00048733C48056024F400640BF06DFB3A480D
:101ED000044200D0FFDFBDE8F08170B5202500226C
:101EE0004FEA020320FA02F1C90719D051B201F0FA
:101EF0001F060124B4404E09B60006F1E026C6F8DC
:101F00008041C6F88042002906DA01F00F0101F194
:101F1000E02181F8143D03E001F1E02181F8003473
:101F2000521CAA42DED370BD70B5174C0D466060DE
:101F3000FFF763FF6068FFF7D0FF2846F7F7A1FFC0
:101F40000AF070FF00F0D5F80BF02EFB0BF079FAD9
:101F5000F8F786F8BDE870400BF012B810B50A4CDF
:101F60006068FFF74AFF6068FFF7B7FF0BF01CFBE4
:101F7000F8F751F80020606010BD034840687047D2
:101F80000A2070470080004088000020048500403F
:101F9000FC1F004000C0004004E5014000D00040AC
:101FA00004D5004000E0004000F0004000F5004093
:101FB00000B0004008B50040FEFF0FFD70B51F499E
:101FC0000A68BAB100231D4601244A68521C4A60BF
:101FD000092A00D34D600E7904FA06F20E68164203
:101FE0000AD072B60B6893430B6062B64968016011
:101FF000002070BD052070BD5B1C092BE5D3FFDF01
:10200000F8E74FF0E0214FF48000C1F8000270477C
:10201000EFF3108111F0010F72B64FF0010202FAD6
:1020200000F20648036842EA0302026000D162B689
:10203000E7E70248002101604160704790000020FE
:1020400001208107086070470120810748607047C0
:1020500012480068C00700D0012070470F48001FD9
:102060000068C00700D0012070470C4808300068A5
:10207000C00700D001207047084810300068704742
:1020800006490C310A68D20306D5096801F003013C
:10209000814201D101207047002070470C040040AC
:1020A000C84911F8210F4978884201D3401A02E04B
:1020B000C1F121010844C0B27047C249233111F86F
:1020C000210F4978884201D3401A02E0C1F1210171
:1020D0000844C0B27047BB49463111F8210F497816
:1020E000884201D3401A02E0C1F121010844C0B284
:1020F0007047B54910B5802081F80004B14900202F
:10210000233101F8210F4870AE4901F8210F4870C2
:10211000AC49463101F8210F4870AC480BF0DAF8B1
:10212000AA48401C0BF0D6F8F0F7DEFDBDE81040E1
:1021300000F03DB920207047B2E770B50C46054667
:102140000026FFF7ADFF01469E48A14212D30022B0
:10215000641EE4B20DD390F82210435C491CC9B24E
:1021600005F8013B80F822102129F1D180F82220C6
:10217000EEE7012600F01BF9304670BD20207047C5
:102180009BE770B50C4605460026FFF796FF014613
:102190008C482330A14212D30022641EE4B20DD336
:1021A00090F82210435C491CC9B205F8013B80F845
:1021B00022102129F1D180F82220EEE7012600F03B
:1021C000F6F8304670BD202101700020704710B530
:1021D0000446FFF780FF2070002010BD70B50C464C
:1021E0000546FFF778FF014676484630A14213D3F3
:1021F0000022641EE4B20DD390F82210435C491C07
:10220000C9B205F8013B80F822102129F1D180F8EC
:102210002220EEE7002401E042F2070400F0C7F8B4
:10222000204670BD70B50C460546212900D9FFDF58
:1022300067480068103840B200F0A0F8C6B20D2020
:1022400000F09CF8C0B2864204D2FFDF02E000BF7B
:10225000F0F79AFD21462846FFF76FFF0028F7D0D8
:1022600070BD2DE9F047DFF86481564CA8F10108F4
:102270000746233498F80000DFF84891002604F15F
:10228000230A38B994F8221094F82100212200F092
:1022900084F890B14D4699F8221099F82100212236
